:020000040800F2
:10000000000002204DFA0008D18D0008D38D0008B1
:10001000D58D0008D78D0008D98D0008000000009C
:10002000000000000000000000000000DB8D000860
:10003000DD8D000800000000DF8D0008E18D000864
:1000400091FA000891FA000891FA000891FA000864
:1000500091FA000891FA000891FA0008E58D00086D
:1000600091FA000891FA000891FA0008DD5A000898
:1000700091FA000891FA000891FA000891FA000834
:1000800091FA000891FA000891FA000891FA000824
:1000900091FA000891FA000891FA0008B58F00085B
:1000A00091FA000891FA000891FA000891FA000804
:1000B000098E0008198E000891FA000891FA0008CC
:1000C00091FA000891FA000891FA000891FA0008E4
:1000D00091FA000891FA0008C990000891FA000806
:1000E00091FA000891FA000891FA000891FA0008C4
:1000F00091FA000891FA000891FA000891FA0008B4
:1001000091FA000891FA000891FA000891FA0008A3
:1001100091FA000891FA000891FA000891FA000893
:1001200091FA000891FA000891FA000891FA000883
:1001300091FA000891FA000891FA000891FA000873
:1001400091FA000891FA000891FA00080D8E000853
:1001500091FA000891FA000891FA000891FA000853
:1001600091FA000891FA000891FA000891FA000843
:1001700091FA000891FA000891FA000891FA000833
:0801800091FA000891FA000851
:10018800CCAB0508000000204C0C0020500C0020CF
:10019800B0810020064B07481A68074B1A60074BC6
:1001A80000221A70064B01221A7000F0A0BF00BF8F
:1001B800F4630020BC0E002008640020E0630020E7
:1001C800085E002008B5034800F091FF024B0022AA
:1001D8001A7008BD4C110020085E002008B5054BB8
:1001E800012200201A7003F07DFF0348BDE8084093
:1001F80000F07DBFA0640020F01100202DE9F0413F
:10020800144C204602F0B3FA00201349134A02F0B6
:1002180065F81349134A0746002002F05FF81249AF
:10022800124A0646002002F059F8D22105463A46FD
:1002380023460A2002F06AF9D22132462346FA20E0
:1002480002F064F95A20D2212A462346BDE8F0413B
:1002580002F05CB904100020F69B0508CD010008E7
:10026800FF9B0508E5010008079C05089D0100089B
:1002780008B5054B012200201A7003F033FF03482C
:10028800BDE8084000F033BFA0640020F011002052
:10029800044B054800221A70044B02221A7000F021
:1002A80026BF00BFE063002004100020085E002085
:1002B80008B5034800F01BFF024B00221A7008BD66
:1002C8004C110020085E00202DE9F041144C204616
:1002D80002F04DFA00201349134A01F0FFFF1349B9
:1002E800134A0746002001F0F9FF1249124A064650
:1002F800002001F0F3FFD22105463A4623460A20A2
:1003080002F004F9D221324623465A2002F0FEF8C0
:10031800AA20D2212A462346BDE8F04102F0F6B8C9
:10032800BC0E0020F69B0508B9020008109C0508C1
:1003380099020008199C050879020008002008B5F0
:1003480003F0D0FE064B00221A70064B1B78022BD6
:100358000CBF05480548BDE8084000F0C8BE00BF0E
:10036800A0640020085E002004100020BC0E0020BD
:1003780010B5084C204602F0FAF900200649074A51
:1003880001F0ACFFD22102462346E620BDE810402A
:1003980002F0BCB838130020229C05084503000869
:1003A80010B5074C4FF6E071206801F0EBFA2068B1
:1003B800044901F095FABDE8104002F011BC00BFF5
:1003C800500C00202B9C050810B5074C4FF6E07127
:1003D800206801F0D7FA2068044901F081FABDE8E5
:1003E800104002F0FDBB00BF500C0020409C0508E7
:1003F80010B5094C07F044FC20684FF6E07101F095
:10040800C1FA2068054901F06BFA02F0E9FBBDE882
:10041800104007F02ABC00BF500C0020559C05086E
:1004280038B507F0EBFB55EC104B07F0FDFB0EF071
:10043800CFFC19A3D3E900230EF030FD02460B468A
:10044800204629460EF054FE114C0FA3D3E9002391
:10045800C4E902010EF022FD04F1100502460B4624
:1004680028460C4913F03AF94FF6E07003F00EFEF7
:1004780000236E209E212A4603F036FF01232376AF
:1004880038BD00BFAFF30080000000A2941A6D428F
:10049800500C0020699C05081F85EB51B81E1940B7
:1004A80038B507F0A5FB0D4C0D4904F1100553ECC8
:1004B800102B284684ED080B13F010F94FF6E07066
:1004C80003F0E4FD00236E203A212A4603F00CFFD6
:1004D800012384F82830BDE8384061E7500C00203B
:1004E800729C050838B507F083FB0D4C0D4904F1E3
:1004F800100553EC102B284684ED0C0B13F0EEF886
:100508004FF6E07003F0C2FD00236E206C212A46EE
:1005180003F0EAFE012384F83830BDE8384053E799
:10052800500C0020729C05082DE9F8433A4C4FF610
:10053800E071206801F026FA2068384901F0D0F906
:1005480002F04EFB002003F0CDFD94F838300BB9D3
:10055800FFF726FF94F828302F4D53B928684FF637
:10056800E07101F00FFA28682D4901F0B9F902F09D
:1005780037FB237E0BB9FFF727FF274C94F8283069
:10058800002B43D094F83830002B3FD0D4E90867CB
:10059800D4E90C89304642464B4639460EF0CAFA31
:1005A8000022204B0EF07AFC02460B4600201E4922
:1005B8000EF09EFD4246C4E910014B4630463946CE
:1005C8000EF096FD0022194B0EF0B4FA02460B46C7
:1005D800002015490EF08CFD0DA3D3E900230EF081
:1005E800A9FA227E0023C4E9120184F8383084F87D
:1005F800283002B123760E4A137007F041FB07F04A
:1006080034FB0C48BDE8F84300F071BDBDE8F88341
:100618000000000000805140500C0020789C050824
:100628008D9C050800005E40000049400000F03F36
:10063800085E00204C1100202DE9F74F464D474E2B
:1006480000244FF6FF78284602F091F841462246EA
:10065800234643480094019401F058F90427306573
:10066800224623464FF6E0713E480097019401F078
:100678004DF941463060224623463B480097019495
:1006880001F044F9414670652246234637480097F1
:10069800019401F03BF92346B065414622463448AF
:1006A8000097019401F032F93249F065324A204648
:1006B80001F014FE3149324A0746204601F00EFE89
:1006C8003049314A8046204601F008FE2F49304A19
:1006D8008146204601F002FE2E492F4A83462046D5
:1006E80001F0FCFD21468246326D2B46204601F082
:1006F8000DFF214632682B467D2001F007FF6E2151
:10070800B26D2B460A2001F001FF3C21F26D2B4609
:100718000A2001F0FBFE69213A462B46E62001F04B
:10072800F5FE372142462B46E62001F0EFFE9B21DD
:100738004A462B46E62001F0E9FE52462B46C821E0
:10074800E62001F0E3FEAA20C8215A462B4603B052
:10075800BDE8F04F01F0DABEA8100020500C0020D0
:10076800A29C05088D9C0508799C0508A99C05088C
:10077800C29C0508DC9C0508ED040008E39C0508FC
:10078800A9040008EB9C0508290400084A9E0508EE
:10079800F9030008F39C050831050008014B93EDA7
:1007A800100B7047500C0020014B93ED120B704753
:1007B800500C0020014B93ED020B7047500C0020A9
:1007C800294B2A48062210B51A704FF6E07400F03B
:1007D8008EFC0020214607F06BFC3120214607F0F3
:1007E80067FC6320214607F063FC9520214607F04B
:1007F8005FFC1F34C7204FF4FC6107F059FC20460A
:1008080003F044FC052001210023194A03F06CFD84
:10081800052020210023174A03F066FD05205221F8
:100828000023154A03F060FD84210520134A0023A4
:1008380003F05AFD4FF4FC6003F028FCB6210520B4
:100848000F4A002303F050FD204603F01FFC0D4A19
:1008580000238720DC2103F047FD0B4B00221A60A0
:100868000A4B01221A7010BDA064002080140020D9
:10087800FA9C0508319D0508299D0508FE9C050878
:1008880045A20508009D0508F8630020E0630020E4
:100898003B4B3C48072270B51A704FF6E07400F0E5
:1008A80026FC0020214607F003FC3120214607F0F2
:1008B800FFFB6320214607F0FBFB9520214607F04C
:1008C800F7FB4FF6FF752146C72007F0F1FB2846D6
:1008D80003F0DCFB0520012100232B4A2B4E03F0FB
:1008E80003FD052020210023294A03F0FDFC0520F3
:1008F80052210023274A03F0F7FC05208421002316
:10090800254A03F0F1FC0520B6213246002303F006
:10091800EBFC40F213144FF4FC6003F0B7FB2046E5
:1009280001211E4A002303F0DFFC204620211C4A37
:10093800002303F0D9FC204652213246002303F05D
:10094800D3FC20468421174A002303F0CDFCB621AE
:10095800154A0023204603F0C7FC284603F096FBFF
:10096800124A00237D20DC2103F0BEFC104B00223C
:100978001A60104A012313700F4A137070BD00BF2C
:10098800A064002080140020059D05082EA10508FC
:10099800099D05080D9D0508109D0508199D050868
:1009A800159D0508149D0508189D05081D9D050839
:1009B800F8630020E0630020206D002038B52D4B3F
:1009C8002D4805241C704FF6E07500F090FB0020C0
:1009D800294607F06DFB2720294607F069FB4F20C1
:1009E800294607F065FB7720294607F061FB9F2021
:1009F800294607F05DFB2946C7201F3507F058FB3D
:100A0800284603F043FB0121002320461B4A03F03C
:100A18006BFC162100232046194A03F065FC3E2191
:100A280000232046174A03F05FFC66210023204676
:100A3800154A03F059FC8E2100232046134A03F07F
:100A480053FCB621124A0023204603F04DFC2846E9
:100A580003F01CFB0F4A00237D20DC2103F044FC3B
:100A68000D4B00221A600D4A012313700C4A1370B3
:100A780038BD00BFA0640020801400202EA1050806
:100A8800289D05082C9D0508309D0508349D0508FE
:100A9800389D05083C9D0508F8630020E0630020A8
:100AA800206D0020F8B53B4B3B483C4F3C4E0422A0
:100AB8001A704FF6E07400F01AFB0020214607F088
:100AC800F7FA3120214607F0F3FA6320214607F0B0
:100AD800EFFA9520214607F0EBFA4FF6FF7521460D
:100AE800C72007F0E5FA284603F0D0FA05200121CF
:100AF80000233A4603F0F8FB052020210023294A69
:100B080003F0F2FB052052210023274A03F0ECFBF7
:100B1800052084210023254A03F0E6FB0520B621A1
:100B28003246002303F0E0FB40F213144FF4FC605C
:100B380003F0ACFA204601213A46002303F0D4FB27
:100B4800204620211A4A002303F0CEFB20465221DA
:100B58003246002303F0C8FB20468421154A0023AF
:100B680003F0C2FBB621144A0023204603F0BCFB65
:100B7800284603F08BFA114A00237D20DC2103F07C
:100B8800B3FB0F4B00221A600E4A012313700E4A62
:100B98001370F8BDA0640020801400205D9D050836
:100BA8002EA10508489D0508589D05084D9D050876
:100BB800529D0508579D05085C9D0508609D050820
:100BC800F8630020E0630020206D0020F8B5324B68
:100BD8003248334F334E03221A704FF6E07400F058
:100BE80086FA0020214607F063FA6320214607F0C1
:100BF8005FFAB3204FF4FC6107F05AFA2146C72088
:100C08001F3407F055FA204603F040FADC21002390
:100C18007D20254A03F068FB204603F037FA0520BB
:100C2800012100233A4603F05FFB052052210023EF
:100C38001E4A03F059FBB62100230520324603F073
:100C480053FB40F213154FF4FC6003F01FFA002326
:100C5800284601213A4603F047FB522128463246EE
:100C6800002303F041FBB621114A0023284603F074
:100C78003BFB204603F00AFA0E4A00230520A22176
:100C880003F032FB0C4B00221A600C4A012313704C
:100C98000B4A1370F8BD00BFA06400208014002028
:100CA8007A9D05082EA105086B9D0508759D050808
:100CB800799D0508399D0508F8630020E063002048
:100CC800206D002008B5074B074802221A7000F073
:100CD8000EFA07F0C7F8054B00221A60044B0122F0
:100CE8001A7008BDA064002080140020F86300205A
:100CF800E0630020002008B503F0F4F9064B002259
:100D08001A70064B1B78022B0CBF05480548BDE836
:100D1800084000F0ECB900BFA0640020085E002085
:100D280004100020BC0E00202DE9F14F2D4C204668
:100D380001F01DFD00202C492C4A01F0CFFA2C4966
:100D48002C4A8146002001F0C9FA2B492B4A074654
:100D5800002001F0C3FA2A492A4A0646002001F079
:100D6800BDFA2949294A0546002001F0B7FA284961
:100D7800284A8046002001F0B1FA2749274A8246CE
:100D8800002001F0ABFAD22183464A462346E620EA
:100D980001F0BCFB28203A462346014601F0B6FB89
:100DA800462132462346282001F0B0FB64212A461A
:100DB8002346282001F0AAFB822142462346282008
:100DC80001F0A4FB524623462820A02101F09EFBF7
:100DD80028205A46BE21234601B0BDE8F04F01F055
:100DE80095BB00BFF0110020229C0508FD0C0008EF
:100DF8007E9D0508CD0C00086B9D0508D50B0008E5
:100E0800609D0508AD0A0008899D0508C509000808
:100E1800949D050899080008009D0508C907000861
:100E280008B5002003F05EF906F0B4FE06F02EFCCB
:100E3800064B00221A70064B01221A7007F094F92B
:100E48000448BDE8084000F052B900BFA064002083
:100E5800085E0020BC0E002008B5002003F042F90F
:100E680006F098FE064B00221A70064B02221A70F2
:100E780007F07AF90448BDE8084000F038B900BF27
:100E8800A0640020085E00200410002008B500209F
:100E980003F028F9034B044803221A70BDE8084000
:100EA80000F025B9085E0020A810002010B50B4CF2
:100EB80006F070FE04F0A4F806F0DDFE07F054F921
:100EC80020684FF6E07100F05DFD2068044900F0ED
:100ED80007FDBDE8104001F083BE00BFB00C002044
:100EE8009E9D05080088C83880B2042810B505D929
:100EF8000A480B4A0B4B7F2102F09AF80A4CC0B201
:100F080004F006F920684FF6E07100F03BFD206818
:100F18000649BDE8104000F0E3BC00BFB29D0508DB
:100F2800ACD50308D29D0508B00C0020039E050827
:100F38002DE9F04F5248534D85B0002401F017FCBD
:100F48004FF6FF71224623464F480094019400F063
:100F5800DDFC042607464FF6E071224623464B483F
:100F68000096019400F0D2FC4FF6E07180462246CC
:100F7800234647480096019400F0C8FC4FF6FF71DD
:100F880081462246234643480096019400F0BEFC61
:100F9800234628604FF6FF7122463F480096019489
:100FA80000F0B4FC3D4968603D4A204601F096F9DE
:100FB8003C493D4A8246204601F090F93B493C4A6B
:100FC8008346204601F08AF93A4902903A4A204677
:100FD80001F084F93A4603902146294B204601F056
:100FE80095FA21464246264BC82001F08FFA0A217D
:100FF8004A46234BC82001F089FA2A68204B64210D
:10100800782001F083FA78206A681D4B014601F0C8
:101018007DFAC82505262827E0B203F0ABFF274A4A
:101028000146284601F05AF994FBF6F106FB1141F6
:1010380079431E31024689B20020114B0134013533
:1010480001F064FA042CADB2E6D1D2215246052053
:101058000B4B01F05BFAD2215A464C20084B01F0A9
:1010680055FAD221029A064B9C2001F04FFA039AB6
:10107800034BEC20D22105B0BDE8F04F01F046BA91
:101088004C110020B00C0020139E05081D9E050879
:101098002A9E0508359E0508799C0508499E05087D
:1010A800B50E0008519E0508950E00085A9E0508C1
:1010B800610E0008639E0508290E0008ED0E000861
:1010C80008B500F005FAFFF799F8FFF7B5FAFFF74A
:1010D800FBF8FFF729FEFFF72BFFFFF749F900F0B0
:1010E8008BFA00F0D9F8BDE8084000F0A1B910B5B6
:1010F800044628B90F48104A104B452101F098FFC3
:101108000F4B1868844213D010B1C3690021984767
:10111800002002F0E7FF002002F0CEFF4FF6FF703C
:1011280002F0B4FFE369204601219847044B1C6094
:1011380010BD00BF6C9E0508BBD50308889E050836
:10114800B80C00200048D2E74C1100204FF6FF7081
:1011580070474FF6FF70704713B5002944D04FF21F
:10116800DE7002F0BFFF002003F086F80F2002F0C7
:101178008DFF1E4C1E4A412101230A2003F0B4F8BA
:10118800042003F079F8236828209621042B21DC19
:101198000123184A03F0A8F801A90DF106022068F6
:1011A80003F02AFB0F2002F071FFBDF80400BDF820
:1011B800061014382822002380B202F097FFBDF8E9
:1011C8000610BDF80400143989B22822012302F060
:1011D8008DFF09E0084A012303F086F81E20A521A7
:1011E800064A012303F080F81CBD00BFBC0C002098
:1011F800989E0508AB9E0508C79E0508DD9E050854
:1012080037B51E4C2368042B05462BDC01A80DF1CD
:10121800060103F0EFFABDF80630BDF804201849BE
:10122800042008F00DF92368002B04DA1548164A43
:10123800164B592105E0042B05DD1248124A144BC0
:101248005A2101F0F5FE04EB8302BDF804100133C6
:101258009180BDF806102360052BD18008D1201D90
:1012680003F04AFB00230B482360FFF740FF03E02D
:1012780028460121FFF770FF3EBD00BFBC0C0020CF
:10128800F49E0508399F0508CDD503085B9F05081E
:10129800729F05089412002037B50B4C204601F0C8
:1012A80066FA0A4B0A49009300250120094A0A4BAD
:1012B800019501F004F9294602462346284603B061
:1012C800BDE8304001F022B9600F0020611100082C
:1012D800551100085B110008091200084FF6FF704D
:1012E80070474FF6FF7070471FB54FF6E07002F079
:1012F800F9FE002002F0C0FF0F2002F0C7FE002117
:10130800294A2A4C01230A2002F0EEFF002002F0AD
:10131800BDFE042002F0B0FF0A201921244A01234F
:1013280002F0E2FF2521234A01230A2002F0DCFF14
:101338001F2002F0ABFE01230A2037211E4A02F0CB
:10134800D3FF237873B301231E2096211B4A02F092
:10135800CBFF62881A49684612F0C0F901231E20A3
:10136800A2216A4602F0C0FFA2881649684612F018
:10137800B5F9AE216A4601231E2002F0B5FF0F2001
:1013880002F084FE6088A188143880B228220023E5
:1013980002F0ACFEA1886088143989B228220123A2
:1013A80002F0A4FE1FBD00BFA09F0508D40C0020BA
:1013B800B29F0508D29F0508F29F050815A00508E9
:1013C80027A0050834A0050801B18DE7704713B5BB
:1013D8000DF1060101A803F0C1F9144B01221A709E
:1013E8005988BDF80420891A0E311C2919460AD8D3
:1013F8009C88BDF80600201A0E301C2803D899686E
:101408000131996001E000238B60084B996801293C
:1014180005DD00229A601A70FFF794FE05E05A80F5
:10142800BDF806209A80FFF75FFF1CBDD40C002092
:1014380037B50B4C204601F09AF90A4B0A4900933C
:1014480000250120094A0A4B019501F038F8294680
:1014580002462346284603B0BDE8304001F056B89E
:1014680094120020D1130008E5120008EB120008BE
:10147800D713000838B50D4B0D4D00241C700D4BCB
:101488001C700D4B4FF0FF321A600C4B1A680C4B56
:1014980020461A6002F026FE0A4B1B78022B0CBF6E
:1014A80009480A48FFF723FE2C7038BDA0640020C5
:1014B800206D0020E0630020F8630020F463002022
:1014C80008640020085E002004100020BC0E0020E4
:1014D80010B50B4C204601F04AF90020014622467F
:1014E80000F074FA00200749074A00F0F7FED221FD
:1014F800024623464FF48270BDE8104001F006B85A
:101508008014002041A005087D14000810B5064C81
:101518004FF6FF71206800F035FA044B206819680F
:10152800BDE8104000F0DCB9E00C0020CC0200203F
:1015380008B5002002F0D6FD054B1868054B196860
:1015480000F0CEF90448BDE80840FFF7D0BD00BF61
:10155800E00C0020C80200204C11002008B5FFF75D
:10156800D5FF0020014606F00BFABDE8084001F05F
:1015780037BB0088A0F5C87080B2092808B505D91E
:101588000748084A084B8F2101F052FD074B188085
:10159800074BFF21197006F0F3F9BDE80840B5E7DD
:1015A80048A00508DFD503086BA00508241500200E
:1015B800261500200088A0F5967080B2092808B585
:1015C80005D90848084A094B832101F031FD084B29
:1015D8001880084B0121197006F0D2F9BDE80840BF
:1015E80094E700BF48A00508F4D503086BA00508D8
:1015F80024150020261500202DE9F34100243A483F
:101608003A4D01F0B4F8224623464FF6FF713848A8
:101618000094019400F07AF90426224623460746EE
:101628004FF6FF7133480096019400F06FF9234696
:10163800286022464FF6FF712E480096019400F06C
:1016480065F92D4968602D4A204600F047FE2C496F
:101658002C4A0646204600F041FE214680463A467E
:101668002046214B00F052FF2A681F4B20462821B4
:1016780000F04CFF3246D2211B4B5A2000F046FFA7
:10168800AA20D2214246184B00F040FF0F254FF404
:10169800967440F2351620461B491C4A00F01EFE7F
:1016A80001340246782128460F4BA4B2233500F0B6
:1016B8002DFFB442ADB2EED10F254FF4C87440F2FD
:1016C800991620461249134A00F008FE01340246D2
:1016D8009B212846044BA4B2233500F017FFB442DF
:1016E800ADB2EED1BDE8FC81DC130020E00C002097
:1016F8009CA005088A9C0508A8A00508651500088F
:10170800B1A0050839150008BAA00508BD150008DC
:10171800BCA005087B15000808B508B143682BB9BB
:101728000348044A044B9B2101F082FC586908BD18
:10173800BEA0050808D60308E0A0050808B5FFF70D
:10174800EBFF8068123080B208BD08B5FFF7E4FFF0
:101758004068063080B208BD2DE9F84F0446884637
:10176800FFF7DAFF6689E589074606F1030905F1FF
:101778000F0AB8F1000F1FD01F2002F087FC204687
:10178800FFF7DCFF83462046FFF7DFFF29460346C5
:101798005FFA8BF2F0B202F0ADFC042002F06CFDAF
:1017A8000B364FF6FF70033502F070FCB0B2A9B2E9
:1017B8003A68012302F098FD3D69204641464A46B1
:1017C8005346A847BDE8F88F13B504460DF1060146
:1017D80001A802F0C3FF2046FFF79EFF6389BDF80A
:1017E8000410BDF80620C91AE389D21A0339C36860
:1017F8000F3A204698471CBDF7B5044614200D46FD
:1018080016461F4611F0F8FB089BC7600361064B9C
:101818000649074A80E8700000930190054B0020B4
:1018280000F04DFEFEBD00BF611700085317000809
:1018380045170008D1170008704708B508B1436874
:101848002BB90448044A054BAD2101F0F1FB586956
:1018580008BD00BFFFA0050820D60308E0A00508C2
:10186800F8B505460E46FFF7E8FF836B04461BB143
:1018780028463146984700E018466F8994F83C306E
:10188800ED890EB9034310D0208E02F0FFFB608E65
:1018980002F012FC94F8350002F0EEFC94F83430B3
:1018A80038462946224602F01FFD002384F83C30C2
:1018B800F8BD08B5FFF7C1FF90F83500BDE808404E
:1018C80002F0EFBC38B5FFF7B8FF044611F08CFF03
:1018D800054694F8350002F0DFFC684380B238BD55
:1018E80038B50D46FFF7A9FF29462E22044611F008
:1018F800ABFF50B1204629462E2211F0F7FF0023F6
:1019080084F82E30012384F83C3038BD2DE9F743A4
:10191800074640200E461546984611F06DFB0446D2
:1019280028B91148114A124B4E2101F081FB114B85
:10193800114A12498DE818000020114B00F0BFFD34
:1019480039468146FFF7CCFF9DF82830268684F873
:1019580035300B9B6586A363002384F8348084F8B4
:101968003C304846BDE8FE83FFA0050838D603088A
:101978001DA1050869180008BB180008CD18000843
:101988004118000810B50C46FFF757FF01230486DD
:1019980080F83C3010BD00BF4FF4A0707047C820DD
:1019A80070477047074B1B78022B07B508D1064BC9
:1019B8001B78022B04D001A80DF1060102F0CEFE1F
:1019C8000EBD00BF206D0020A064002073B50A4B37
:1019D80006460D461446009300200849084A094B5C
:1019E800019000F06CFD294602462346304602B0BD
:1019F800BDE8704000F08ABDAB190008A1190008C5
:101A0800A7190008AD19000813B502AB03E90600D1
:101A1800436843B1027C0124082A9C7004D11B69E5
:101A28002146984700E01C4620461CBD30B50028DA
:101A38002BD0058B002425E0036A1A7C012A05D1E6
:101A48005B681A888A421BD1187F30BD052A06D1E7
:101A58005B681A888A4213D193F82C0030BD032A98
:101A680006D15B681A888A420AD193F8250030BDEE
:101A7800062A05D15B681A888A4201D1D87A30BD16
:101A880001340430AC42D7D3002030BD08B1817591
:101A980001207047F8B504460D46D0B1E175D0F87D
:101AA80098309847012D0DD12746002606E0F869A1
:101AB80000F10802436906CA98470136238B0437A8
:101AC8009E42F4D3D4F898302046294698470120FE
:101AD800F8BDF8BDF8B50546084617460E4611F09C
:101AE80083FE013FB84234BF04463C463CB1284619
:101AF8003146224611F0FAFE00232B55F8BD2C7012
:101B0800F8BDF7B5044600200090019000296CD07C
:101B18000E8B68E000F1080351F823301D7C042D7A
:101B280004D15D682D88954247D0013000F1080343
:101B380051F823301D7C012D04D15D682D88954214
:101B48003BD0013000F1080351F823301D7C052DEE
:101B580004D15D682D8895422FD0013000F108032B
:101B680051F823301D7C032D04D15D682D889542E2
:101B780023D0013000F1080351F823301D7C022DD9
:101B880004D15D682D88954217D0013000F1080313
:101B980051F823301D7C072D04D15D682D8A9542AC
:101BA8000BD0013000F1080351F823301D7C062DBD
:101BB80008D15D682D88954203D103F108012046BC
:101BC80015E0013000F1080351F823502B7C082B55
:101BD80009D16F683F88974204D105F10801204672
:101BE8001A4605E00130B04294D3204669460822DF
:101BF80011F0B2FC2046FEBDF8B505460F46164664
:101C0800002830D04388032B2FD0202011F0F4F97E
:101C1800044600282BD040F80C5B39460C22FFF70D
:101C280059FF1820E66111F0E7F90646B8B102231A
:101C38000374012363760F4B446063600E4BA3600B
:101C4800002323766B8805EB830201339BB2012BBB
:101C580050606B800CD16A685268137608E02046A1
:101C680011F0D2F904E0064602E0002600E006463C
:101C78003046F8BDA85504084652040837B54568EB
:101C880002AB03E906003DB3037C0124042B85F86D
:101C9800314022D1688E02F0F9F995F8300002F04F
:101CA800EBFA95F8343043B9BDF80200BDF80610D8
:101CB800AA1C234602F018FB0FE0012B03D10848A9
:101CC80040F2395104E0022B07D1054840F2415156
:101CD800044A054B01F0ACF92C4620463EBD00BF36
:101CE80030A10508F82004082EA10508F8B5044617
:101CF8000F46164610B3838A0A2B20D0202011F0F5
:101D08007BF90546E8B14460102200F10800394625
:101D1800FFF7E0FE4FF6FF73A08A2B801F236B802E
:101D280000232B76831D013080B20128EE6144F830
:101D38002350A08207D1A3691876F8BDF8BD00200A
:101D4800F8BD0120F8BD0120F8BD2DE9F0411D4680
:101D58004B1C984280460C4617460CDD95420ADC1F
:101D6800013208F101035B1A521BC8B2D2B29BB20E
:101D7800294602F0BDF9A8F10208BDF81800C4EB25
:101D8800080802F083F901261FFA88F808E0A91963
:101D9800601C80B289B24246002302F0A7F90136DE
:101DA8007B1B9E42F3D3BDE8F081F8B5C7B2144659
:101DB80038461E460D4602F09FF9621E92B238461A
:101DC800294602F099F9304602F060F9022606E049
:101DD800A21B92B23846294602F08EF90136A64275
:101DE800F6D3F8BD70B5044600F11E003C2200236E
:101DF80080B20D4602F07AF91E3DA9B220463C2277
:101E08000123BDE8704002F071B970B5044601388D
:101E18000322002380B20D4602F068F9013DA9B201
:101E2800204603220123BDE8704002F05FB9F7B5F0
:101E3800089D2E7BEF7A1C463604AB7A06EB072604
:101E4800F618431A687B06EB00602D1800200190F5
:101E5800121B08462146009501F098FEFEBD30B5DC
:101E6800456885B004AB03E906007DB101242C73F5
:101E78006D68BDF80800BDF80A109DF80C209DF8A3
:101E88000E300095FFF7D3FF204600E0284605B046
:101E980030BD2DE9F04385B004AB03E90600446882
:101EA800BDF80860BDF80C70002C41D0012384F8FF
:101EB800263094F825300BB9A26800E06268FFB2BA
:101EC800BDF80A109DF80E30009230463A46FFF7EA
:101ED800AEFF04F10C08022002F0CEF9404611F0E2
:101EE80083FC054600B1451E0F3F0024153E1FFA2E
:101EF80087F90DE002F0CAF902F0CEF904FB10618F
:101F080089B248462022002302F008FA0134E4B2DC
:101F1800AC42EFD3002002F0B9F8B8B2B1B24246F1
:101F2800012302F0FBF9002002F0A6F9012000E0ED
:101F3800204605B0BDE8F0832DE9F04385B004AB39
:101F480003E906004568BDF80860BDF80C70002D6F
:101F58003CD001236B762B7EBDF80A10012B0CBFF9
:101F68006A68AA689DF80E300092FFB23A46304679
:101F7800FFF75DFF0C35022002F07EF9284611F0CC
:101F880033FC0E3F81460024163E1FFA87F80DE009
:101F980002F07CF902F080F904FB106189B2404636
:101FA8002022002302F0BAF90134E4B24C45EFD9FB
:101FB800002002F06BF8B8B2B1B22A46012302F051
:101FC800ADF9002002F058F9012000E0284605B0DC
:101FD800BDE8F0832DE9F04F85B00546DDF8409067
:101FE800029148469046039311F0FEFBDDF838A0B5
:101FF800DDF83CB00646294600242F4611E024B1FE
:10200800B4420CBF5B46534600E0039B01F1080550
:10201800ADB200932846029A4346FFF708FF013401
:102028002946B442EBDD002002F030F8022002F02D
:1020380023F97D1D08F10508A8B21FFA88F14A4660
:10204800012305B0BDE8F04F02F04EB970B5406805
:1020580086B006AB03E9060000282ED0012380F8DD
:102068002D308668164BF21A534243EB020390F860
:102078002C205AB1002B134D134B144A08BF1D4690
:10208800134B00F11C0418BF13460AE0002B0D4D3A
:102098000D4B0E4A18BF1D460D4B00F10C0408BF2E
:1020A8001346BDF81200BDF81410BDF816200096AE
:1020B80001950294FFF78EFF012006B070BD00BFA6
:1020C800682A0408A42604084A2C04088628040858
:1020D8002C2E040870B5446886B006AB03E90600E8
:1020E80004B301236377A668104B227FF11A4B4291
:1020F80043EB01030AB10BB904E01BB966680C4D48
:102108000C4B01E00C4D0D4BBDF81200BDF814103E
:10211800BDF8162000960C3401950294FFF75AFF7B
:10212800012000E0204606B070BD00BFB4350408A9
:10213800F0310408D23304089637040878390408C3
:102148002DE9F04385B004AB03E906004468BDF807
:102158000860BDF80A90BDF80C50BDF80E80002C40
:1021680000F08C800123A3740220676802F084F8D1
:102178004FF6FF7001F0A0FF002001F087FFEDB2DD
:102188005FFA88F8A6F1160189B230462A46434616
:102198000097FFF74CFE277A002F2ED1A28A2346FC
:1021A80000E00137974204D29969097E0433002977
:1021B800F7D002F06BF802F06FF8A9F116091FFAD0
:1021C80089F90E2101FB10914FF6FF7208F1010801
:1021D8005FFA88F389B2009248462A46FFF7B5FDB0
:1021E800022002F049F81F2001F050FFA38A002BBB
:1021F80038D0103DE8B2303E2CE0E3685C68A28A33
:102208002346013A002700E00137974204D2996932
:10221800097E04330029F7D002F038F802F03CF8C0
:102228000E2101FB10914FF6FF7208F101085FFAC9
:1022380088F389B2009248462A46FFF786FD0220B5
:1022480002F01AF81F2001F021FFA38A53B1103DB4
:10225800E8B21A3E0637B1B254F8272001230832F3
:1022680002F05CF8002002F007F84FF6FF7001F06A
:1022780023FF1F2001F00AFF012000E0204605B0DF
:10228800BDE8F0832DE9F04105463620884614461E
:102298001F4610F0B1FE0646E0B120F8025B414649
:1022A8002E22FFF717FCBDF8183086F834407386E5
:1022B8001820012386F8307086F8313010F09CFE23
:1022C800044618B104234660037404E0304610F055
:1022D8009BFE00E004462046BDE8F081F8B50646BE
:1022E80024200F46154610F087FE0446D8B10F4B40
:1022F800068083600E4B39464360102200F10C00C3
:10230800FFF7E8FB0126002318202562237766776C
:1023180010F072FE054610B14460067404E02046D1
:1023280010F072FE00E005462846F8BDB4350408F2
:102338000E300408F8B506462C200F46154610F056
:102348005BFE0446E8B120F80C6B39461922FFF70A
:10235800C1FB0D4BA562A3600C4B6360002384F89E
:1023680025301820012384F8263010F045FE054654
:1023780018B103234460037404E0204610F044FEBF
:1023880000E005462846F8BDE44E0408824B0408E0
:1023980010B50446142010F02FFE20B1002343800E
:1023A800014B0480036110BD011C000838B50546C7
:1023B800442010F021FE0446C0B10E4B0582436054
:1023C8000D4B0360012383740023037283820B4B3C
:1023D8000364182010F010FE054618B10723446066
:1023E800037404E0204610F00FFE00E0054628467E
:1023F80038BD00BF784704086E430408F51C000880
:102408002DE9F04105463420884614461F4610F051
:10241800F3FD064620B3144B05808360134B4146F9
:102428004360102200F10C00FFF754FB214606F12F
:102438001C001022FFF74EFB002386F82C301820D2
:102448000123376386F82D3010F0D6FD044618B105
:1024580005234660037404E0304610F0D5FD00E023
:1024680004462046BDE8F081682A0408C22404080E
:102478002DE9F041044614200D461646984610F002
:10248800BBFD0746B8B1069B048003610023C372F5
:1024980001234560068180F80A800373182010F034
:1024A800ABFD044618B106234760037404E03846C0
:1024B80010F0AAFD00E004462046BDE8F0812DE9B1
:1024C800F041044618200D461646984610F094FD33
:1024D8000746B8B101238370069B04800361079BFC
:1024E80045608660C0F80C804361182010F084FDB8
:1024F800044618B108234760037404E0384610F016
:1025080083FD00E004462046BDE8F0812DE9F34153
:1025180098461B8B1D2B05460C4617464FF00000AE
:1025280000F2B480B5F5A07F0090019000F2AE8073
:10253800F02900F2AB80127CADF80610511EADF800
:102548000250072900F28A80DFE801F045595E044D
:10255800456A14767B684E4A7A611A8893F8343053
:102568003A80013BDBB2012B7FD8ADF80240ADF8D1
:1025780006507AE005F11602ADF8002004F11602C3
:10258800ADF8042002AE434A16E903007A6107F168
:10259800080282E8030003F10802013348F82270B8
:1025A800A8F818307B681A8A187A3A8000286CD103
:1025B800FFF7FCFE3849436859603849DF60012657
:1025C800163D196002461E72A8B2E1B24346FFF7F3
:1025D8009DFF30465AE0012A0CBF314B314B7868D9
:1025E8007B6130F80C3B3B8011F0FEF8431CDB00AC
:1025F8001A34ED18ADF80440ADF8005035E07B68AA
:10260800294A1B687A6102E0284A7B687A611B883C
:1026180014353B80ADF800501434ADF8044024E084
:102628007B68234A7A611A883A801A899B7AAD189E
:10263800ADF80050E418F0E77E681E4B7B613388E4
:1026480038463B8073689847013D4519ADF80050FE
:10265800B36838469847013C0419DEE71648174A1C
:10266800174B40F21A3100F0E3FC02AA12E903000A
:1026780007F1080383E80300B8F8183003F10802EB
:10268800013348F82270A8F818300120BDE8FC8111
:10269800851C000849210008643F04085A3B0408C7
:1026A800DD20000855200008411F00089B1E000877
:1026B800671E0008111A000830A10508082104083F
:1026C8002EA10508F8B51646002834D01378002B3B
:1026D8002ED0028B002327E0046A257C042D21D10B
:1026E80065682F888F421DD195F8313053B16F8EB0
:1026F80001F0F2FC04F1080268866369204606CA04
:1027080098476F86A81C31462E22FFF7E3F995F803
:1027180031307BB104F108026369204606CA984744
:102728000120F8BD013304309342D5D30020F8BD11
:102738001846F8BD0120F8BD70B5B8B1068B04463F
:10274800002310E0256A287C04280AD16D682888AF
:10275800884206D11046A91C2E22FFF7BBF901209A
:1027680070BD01330434B342ECD3002070BD38B5DA
:10277800044620B3134BC361134BC0F89830134B76
:10278800C0F89C30124B00257822C0F8A03085751F
:10279800C5750583294600F1200010F01FFFD4F805
:1027A80098302046294698470A4A1388312B07D87B
:1027B800094941F8234001331380012038BD38BD51
:1027C800284638BD9D1A0008951A0008351A0008D1
:1027D8000B1B0008E80C0020281500202DE9F0410B
:1027E8000446002800F0B380078B02460025A8E0C5
:1027F800136A1E7C042E00F08780012E23D15868AE
:1028080003888B4240F09B8005F1080710F0FCFB21
:1028180054F827004FF00008C0F8048010F0F4FBCB
:10282800228B531E9D4208D00732238354F822106E
:1028380044F8271044F8228002E044F827802583D2
:102848003046BDE8F081052E5ED0032E5CD0022E06
:1028580013D15B68186803888B4270D14388013BA9
:102868009BB243800BB910F0CFFB05F1080654F872
:102878002630586810F0C8FB4EE0072E21D15E685C
:10288800338A8B425BD1002706E0BB1D013756F81F
:10289800230010F0B9FBFFB2B38ABB42F5D800277A
:1028A800B78205F1080654F82630586810F0ACFBDA
:1028B80054F8260033E044F8267025830120BDE84B
:1028C800F081062E1ED1586803888B4237D105F156
:1028D800080610F099FB54F826000027476010F00E
:1028E80093FB228B531E9D4209D00833013A54F8BA
:1028F8002310228344F8261044F82370DEE744F8B6
:1029080026701AE0082E1AD1586803888B4216D10F
:1029180010F07AFB05F1080654F8260000274760F6
:1029280010F072FB228B531E9D42C4D0073254F81C
:10293800221044F8261044F822702383BEE701359C
:102948000432BD42FFF454AF0020BDE8F081BDE879
:10295800F08170B5044600282AD0068B751E08360B
:1029680000EB86061EE056F8043D1A7C042A13D0B4
:10297800012A11D0052A0FD0032A0DD0022A02D12C
:102988005B681B6809E0072A02D15B68198A05E0C1
:10299800062A01D0082A04D15B6819882046FFF767
:1029A8001DFF013D681CDED100232383012070BD7B
:1029B80070BDF0B528B30023068B1A461EE0046AE2
:1029C800257C072D18D16468258A8D4214D1A78AE1
:1029D800002504EB83040DE004EB050C0435DCF85A
:1029E80018C09CF818C0BCF1010F03F1010301D114
:1029F800D8B2F0BDBB42EFD301320430B242DED3CD
:102A08000020F0BD70B508B3048B00231BE0026AF8
:102A1800157C072D15D15268158A8D4211D10023D6
:102A2800958A11461C46012007E013B9966930764D
:102A380001E08E69347601330431AB42F5D30120CD
:102A480070BD01330430A342E1D3002070BD2DE9ED
:102A5800F04128B30023078B1A461EE0046A257C40
:102A6800072D18D16468258A8D4214D1B4F814C092
:102A7800002504EB83040CE066190435B66996F862
:102A88001880B8F1010F03D106F10800BDE8F08104
:102A980001336345F0D301320430BA42DED300205B
:102AA800BDE8F0812DE9F04700282FD00023B0F8C9
:102AB80018C01D4627E0046A267C072E21D16468C9
:102AC800268A8E421DD1B4F81480002604EB8309AF
:102AD80015E009EB0604A7693C7E012C0DD192F89C
:102AE80000A0BAF1000F08D007F108001146102223
:102AF800FEF7F0FF2046BDE8F08701330436434572
:102B0800E7D3013504306545D5D30020BDE8F0870B
:102B1800F0B5B0B1068B002510E0046A277C062FBB
:102B28000AD1646827888F4206D123819DF8143022
:102B38006260A3720120F0BD01350430B542ECD3C8
:102B48000020F0BD10B500210446FEF7A3FF204683
:102B58000121BDE81040FEF79DBF38B598B1048B40
:102B6800024600230CE0106A058804328D4206D123
:102B780000F10802436906CA9847012038BD0133AD
:102B8800A342F0D3002038BD10B50C460021FEF753
:102B980081FF20460121BDE81040FEF77BBF13B539
:102BA80002AC04E90C00BDF80230834206D8BDF837
:102BB8000030834234BF0020012000E00020BDF82F
:102BC80006308B4206D8BDF804308B4234BF002152
:102BD800012100E00021002818BF0846C0B21CBD32
:102BE80038B5114B114A1988002319E052F8045FCF
:102BF800A87D012812D100240CE004F1080355F83F
:102C08002300037C082B03D1436800211B699847E4
:102C18000134A4B22B8BA342EFD838BD01339BB249
:102C28008B42E3D138BD00BFE80C002024150020FA
:102C3800704770B5094CA5787DB9094B1E78012EEF
:102C48000BD16368013363606268064B9A4204D90A
:102C5800284601F0D3FAA670656070BDE80C002024
:102C68003000002040420F00054A9060134602E001
:102C780099680139996091680029F9D1704700BFB6
:102C8800E80C0020F0B585B001F066FD002800F0E2
:102C98004981002502A80DF10A01ADF80850ADF8E8
:102CA8000A5001F05BFD03A80DF10E01ADF80C50C0
:102CB800ADF80E5001F09EFDBDF80C10BDF80820CF
:102CC8000091BDF80E10BDF80A3001912C46964DC2
:102CD8009649082006F0B4FBA878012803D101F032
:102CE8008DFAAC7019E1924B5B78012B40F015819D
:102CF800AB78002B40F011816B6029888D4A09E17F
:102D080052F8046FB07D012840F002810025FAE0F6
:102D180005F10803BDF8080056F82340BDF80A106D
:102D280004F108030CCBFFF73AFF002800F0E98014
:102D3800237C013B062B00F29F80DFE803F0042987
:102D4800159D1F9D4C006668012304F10805337723
:102D580095E80600636920469847002333772046A4
:102D6800636995E8060086E0636893F8252012F108
:102D7800FF3218BF012283F8252077E0636893F8B3
:102D88002C2012F1FF3218BF012283F82C206DE0AD
:102D98006268137E1568002B6ED16E882F4629460F
:102DA800184606E051F804EFDEF804E001338EF827
:102DB8001800B342F6D301231376002607E057F82C
:102DC800040F00F10802436906CA984701366B8868
:102DD8009E42F4D350E0656820892E68A37B227B4D
:102DE8000096A0F1160189B2FFF721F81420FFF729
:102DF8003BFF2B7AC3B9AF8A29461A461E4609E01B
:102E0800886990F818E00676BEF1010F08BF1346EE
:102E180004310132BA42F3D301220BB9AB6924E081
:102E2800053355F8233020E06368DB685A680023CF
:102E3800908A154619461F4609E0AE6996F818E0CB
:102E48003776BEF1010F08BF0B46043501318142C8
:102E5800F3D3411E8B4203D1053052F8203003E0F2
:102E680004D2073352F8233001221A7604F10802FB
:102E780006CA636920469847237C013B072B4CD838
:102E8800DFE803F00410074B0A0D123A63681B6A67
:102E980034E063689B6A2DE063681B6B2AE0636813
:102EA8001B6927E0636824E063681A7A7AB9988A0C
:102EB8001946013800E00132824204D28C69247E2E
:102EC8000431002CF7D0063253F8223011E0DB68C9
:102ED8005A68908A11460138002300E00133834282
:102EE80004D28C69247E0431002CF7D0063352F8C2
:102EF8002330DB69984710E06368DB682046984711
:102F08000BE00135ADB2338BAB423FF601AF04E0C5
:102F180001339BB28B427FF4F3AE01F063FC0F20C8
:102F2800FFF7A2FE05B0F0BDE80C002056A1050889
:102F38003000002024150020034B9A6812B19A68CB
:102F4800013A9A60704700BFE80C00202DE9F3476A
:102F58000120DFF8D080DFF8D09001460AF098FB16
:102F68000025012403234FF4807602274046694652
:102F78008DF8053000968DF804708DF806508DF8A0
:102F8800074009F0DDFF4046082122460AF058F8BC
:102F9800234BDFF898801A6844F2A243B2FBF3FA95
:102FA8000AF1FF3A204621461FFA8AFA0AF0A0FBE6
:102FB800C8F804A048464146A8F80050A8F80250AE
:102FC800A8F8085088F80A500AF02EFF7023A8F8CD
:102FD8000C300423A8F810300AF1FF3A6323642266
:102FE80003FB0AF3B3FBF2F39BB2C8F8143008F101
:102FF8000C014846A8F80E40A8F81870A8F81A500E
:10300800A8F81C60A8F81E500BF02CF8484621467A
:103018000AF09FFF484621460BF0A5FABDE8FC8759
:10302800E00200200000024000000140F80C0020EF
:1030380083B50E460746154910201C46154606F06E
:10304800FFF91020124906F0FBF91020114906F08B
:10305800F7F910200E4906F0F3F9002310200E4965
:10306800019306F0EDF9334610200C493A4606F074
:10307800E7F910200A492A4606F0E2F91020094922
:10308800224606F0DDF9019B0133E7E790A1050828
:1030980095A10508B5A10508C5A10508D5A105088C
:1030A800EAA10508FBA1050808B5164B1A6A013202
:1030B8001A621A6A012A1A4603D013484FF4A071FB
:1030C8000FE05862194602E04B6A013B4B62506AB6
:1030D8000C4B0028F8D11A6A012A06D00A4840F297
:1030E8004B110A4A0A4BFFF7A3FF1A6A013A1A6200
:1030F8001B6A2BB10448054A064B40F24D11F2E712
:1031080008BD00BFF80C00200CA205080A590408E5
:1031180036A2050847A205080C4B0D491A6844F267
:10312800A2436428B2FBF3F3D4BF20EAE070642022
:10313800013B9BB24B60013B58436422B0FBF2F069
:1031480080B2486103480C310AF00FBFE00200204A
:10315800F80C00200000014010B5134B93F828200C
:103168002AB11248124A134B4FF40A710EE0012299
:1031780083F8282066234FF0C042013BDBB2108061
:1031880033B90A480A4A0C4B40F23221FFF750FF84
:103198001488A4B28442F0D1084B1980024B002253
:1031A80083F8282010BD00BFF80C00200CA20508E9
:1031B8001459040858A205082EA105080000026049
:1031C80010B5FFF7C3FE6420FFF7A6FFE5204FF414
:1031D8000041FFF7C1FF00200121FFF7BDFF0120DB
:1031E8004FF48071FFF7B8FF02204FF4E061FFF75A
:1031F800B3FF032041F23001FFF7AEFF04200021A6
:10320800FFF7AAFF082040F20221FFF7A5FF0920D7
:103218000021FFF7A1FF0A200021FFF79DFF0C20E6
:103228000021FFF799FF0D200021FFF795FF0F20E0
:103238000021FFF791FF10200021FFF78DFF1120DB
:103248000021FFF789FF12200021FFF785FF1320D7
:103258000021FFF781FF102041F2B071FFF77CFFDA
:1032680037211120FFF778FF3220FFF71DFF1220CA
:1032780040F23B11FFF770FF3220FFF715FF1320D4
:103288004FF4C051FFF768FF0F212920FFF764FFB3
:103298003220FFF709FF20200021FFF75DFF2120E2
:1032A8000021FFF759FF30200021FFF755FF31209B
:1032B8000721FFF751FF322040F20311FFF74CFFBF
:1032C800352040F20741FFF747FF40F2044436201B
:1032D80040F60F11FFF740FF37202146FFF73CFF6C
:1032E80038204FF48061FFF737FF39202146FFF778
:1032F80033FF3C200021FFF72FFF3D204FF4806172
:10330800FFF72AFF50200021FFF726FFEF21512069
:10331800FFF722FF52200021FFF71EFF532040F243
:103328003F11FFF719FF60204FF41C51FFF714FFFE
:1033380061200121FFF710FF6A200021FFF70CFF31
:1033480080200021FFF708FF81200021FFF704FFFC
:1033580082200021FFF700FF83200021FFF7FCFEF9
:1033680084200021FFF7F8FE85200021FFF7F4FEF6
:1033780090201021FFF7F0FE92200021FFF7ECFECD
:1033880093200321FFF7E8FE95204FF48871FFF79B
:10339800E3FE97200021FFF7DFFE98200021FFF7CA
:1033A800DBFE072040F27311BDE81040D4E610B5EB
:1033B800FFF7CCFD6420FFF7AFFE21210720FFF7C0
:1033C800CBFE3220FFF770FE01210020FFF7C4FE7C
:1033D8003220FFF769FE23210720FFF7BDFE3220C8
:1033E800FFF762FE00211020FFF7B6FE40F6B83066
:1033F800FFF75AFE33210720FFF7AEFE3220FFF712
:1034080053FE112046F63001FFF7A6FE3220FFF7E3
:103418004BFE4FF4C0610220FFF79EFE3220FFF7FB
:1034280043FE122046F6EB41FFF796FE3220FFF7E7
:103438003BFE03204AF6A401FFF78EFE3220FFF779
:1034480033FE00210C20FFF787FE3220FFF72CFE09
:103458000D2040F60C01FFF77FFE3220FFF724FE17
:103468000E204FF42C51FFF777FE3220FFF71CFE99
:10347800B0211E20FFF770FE3220FFF715FE012055
:1034880042F63F31FFF768FE3220FFF70DFE0520B8
:103498000021FFF761FE3220FFF706FE002106201B
:1034A800FFF75AFE3220FFF7FFFD16204EF61C717B
:1034B800FFF752FE3220FFF7F7FD172040F2031105
:1034C800FFF74AFE3220FFF7EFFD00210B20FFF740
:1034D80043FE3220FFF7E8FD00210F20FFF73CFEF6
:1034E8003220FFF7E1FD41200021FFF735FE3220B1
:1034F800FFF7DAFD42200021FFF72EFE3220FFF70A
:10350800D3FD00214820FFF727FE40F23F14322068
:10351800FFF7CAFD21464920FFF71EFE3220FFF7BC
:10352800C3FD00214A20FFF717FE3220FFF7BCFD3C
:1035380000214B20FFF710FE3220FFF7B5FD442095
:103548004FF46F41FFF708FE3220FFF7ADFD002171
:103558004520FFF701FE3220FFF7A6FD2146462051
:10356800FFF7FAFD3220FFF79FFD302040F2077188
:10357800FFF7F2FD3220FFF797FD31204FF401717C
:10358800FFF7EAFD3220FFF78FFD32204FF401717B
:10359800FFF7E2FD40F202543220FFF785FD214695
:1035A8003320FFF7D9FD3220FFF77EFD342040F2AB
:1035B8000751FFF7D1FD3220FFF776FD35204FF494
:1035C8000171FFF7C9FD3220FFF76EFD36204FF479
:1035D8000171FFF7C1FD3220FFF766FD2146372054
:1035E800FFF7BAFDA4F500743220FFF75DFD214610
:1035F8003A20FFF7B1FD3220FFF756FD2F2041F2A8
:10360800BE21FFF7A9FD3220FFF74EFD21463B20E2
:10361800FFF7A2FD3220FFF747FD00212320FFF727
:103628009BFD3220FFF740FD00212420FFF794FD89
:103638003220FFF739FD25204FF40041FFF78CFDBC
:103648003220FFF731FD00214F20FFF785FD3220A2
:10365800FFF72AFD4E200021FFF77EFD3220BDE84E
:10366800104021E508B5124B93F829202AB11148DA
:10367800114A124B40F242210FE0012283F829201F
:10368800222166234FF0C042013BDBB2118033B9DF
:103698000848094A0A4B40F25B21FFF7C9FC108829
:1036A80080B22228F0D1024B002283F8292008BDDD
:1036B800F80C00200CA205082159040858A2050896
:1036C8002EA1050810B5224B49F22032032823D831
:1036D800DFE800F0021A0B111C8846F6280041F2B8
:1036E8002801944218BF01461AE01C8841F20800DC
:1036F80046F6080104E01C8841F2300046F6300125
:10370800944208BF01460BE0188846F62001904213
:1037180008BF4FF4815103E00E4840F2792113E0CD
:103728001B8848F68912934205D049F22032934209
:1037380007D1032000E01120FFF70EFDBDE810407F
:1037480090E7044840F28521034A044BFFF770FCD8
:10375800320000200CA20508365904082EA10508DD
:10376800014B18800A209FE4000002604FF0C0431C
:10377800188003F500331A881A88188880B27047B1
:103788002DE9F041022098B00121002409F080FFC2
:10379800012502268C488DF85C5016A98DF85E40EC
:1037A8008DF85F4016968DF85D6009F0C9FB18200A
:1037B800294609F06DFF2846294609F081FF214670
:1037C8000C22824809F03CFC29460C227F4809F06B
:1037D80037FC04210C227D4809F032FC05210C221B
:1037E8007A4809F02DFC07210C22784809F028FCBA
:1037F80008210C22754809F023FC09210C22734882
:1038080009F01EFC0A2171480C2209F019FC0B2151
:103818006E480C2209F014FC0E210C226B4809F0AA
:103828000FFC0F210C22694809F00AFC07210C2221
:10383800674809F005FC08210C22654809F000FCDE
:1038480009210C22624809F0FBFB0A210C2260487E
:1038580009F0F6FB0B210C225D4809F0F1FB0C2165
:103868000A465B4809F0ECFB0D210C22584809F088
:10387800E7FB0E210C22564809F0E2FB0C225448C3
:103888000F2109F0DDFB03274CF6B3734F4816935D
:1038980016A98DF85D708DF85E408DF85F408DF843
:1038A8005C6009F04DFB4FF6807316A948481693E3
:1038B8008DF85D708DF85E408DF85F408DF85C6026
:1038C80009F03EFB40F6B830FFF7EEFB22463146E2
:1038D8003D4809F0AAFB44F6FF70FFF7E5FB2A46CE
:1038E8003146394809F0A1FB40F6B830FFF7DCFB58
:1038F8004FF48053102709930DF13C084FF400232F
:1039080068460F9410941294139514941594009487
:103918000194029404940694079408940A940594D4
:103928000B940C9311960397CDF8348009F081F825
:1039380004236846119310941294139514941594C3
:103948000F96CDF8388009F074F82946204609F01A
:10395800F0F840F6B830FFF7A7FB2046FFF706FF60
:1039680004461C491C4D3846224605F069FD48F6B8
:1039780089139C421AD049F220339C420DD041F25F
:1039880089239C4212D03846144905F059FD144841
:10399800144A154BA621FFF74BFB3846134922461C
:1039A80005F04EFD2C80FFF70BFC0AE0FFF7FFFC4B
:1039B80048F689122A8010200D4941F2892305F022
:1039C8003FFD18B0BDE8F08100040240000C024041
:1039D800001002406DA205083200002084A20508EC
:1039E8000CA205084E5904082EA10508BBA205081B
:1039F800F0A205084FF0C04322221A8003F50033D5
:103A080082B01A8892B2ADF806201B889BB2ADF836
:103A18000630BDF8060080B202B07047134B1B8811
:103A280048F68912934210B504460BD049F2203269
:103A3800934213D1C1F1EF01202089B2FFF78CFB2B
:103A4800212006E0C1F1EF014E2089B2FFF784FB87
:103A58004F202146BDE81040FFF77EBB0448054AC9
:103A6800054B40F2F321FFF7E3FA00BF32000020D4
:103A78000CA20508575904082EA105082DE9F041A4
:103A88000D46C5F1F008411E5E18C2EB0802C5F1EB
:103A9800EF039BB292B2B6B29A422CBF90469846B8
:103AA8009A4234BF11461946864234BF3746074604
:103AB80040F23F13864238BF06469E4228BF1E4644
:103AC8001B4B1B8848F68912B8F1EF0F28BF4FF03F
:103AD800EF089342044610D049F2203293421FD196
:103AE8005020FFF739FB51204146FFF735FB5220A4
:103AF8003946FFF731FB53200AE041EA082189B231
:103B08004420FFF729FB45203946FFF725FB4620CF
:103B18003146FFF721FB20462946BDE8F0417DE705
:103B28000448054A054B40F2DD21FFF781FA00BF42
:103B3800320000200CA20508655904082EA10508CA
:103B480000200146F0224FF4A07397E7072040F2C7
:103B58007311FFF701BB07200021FFF7FDBA10B56D
:103B68001446FFF75BFFFFF77DFD2046BDE81040D8
:103B7800F6E508B5FFF752FF4FF0C04322221A803E
:103B880003F500331A88188880B208BDF8B580B2EA
:103B980002FB03F589B292B29BB2069C9DF81C60A9
:103BA800FFF76CFF0020FFF78DFD002709E034F8D0
:103BB800020B1EB1030A43EA002080B2FFF7D0FDD2
:103BC8000137AF42F3DBBDE8F840B9E72DE9F74F1D
:103BD80016469DF834200C9F01920546B2B280B279
:103BE8000C46984689B29BB2FFF748FF4FF0000B8E
:103BF8000020FFF767FDDA463DE0002D30DB09EBDA
:103C0800050340F23F1293422ADC002C28DB0BEB21
:103C18000403EF2B24DC19F00F0F04D1B9F1000FC6
:103C2800C8BF0AF1010A174B09EA0303002B03DA9C
:103C3800013B63F00F030133019A0AB1C3F10F038B
:103C4800012202FA03F337F81A2013401BB213B10A
:103C58000D4B588D01E00D4A508880B2FFF780FD6A
:103C680009F1010901E04FF00009C145C5DB0AF17E
:103C7800010A0BF1010BB345F5DB03B0BDE8F04FCA
:103C88005EE700BF0F000080F80C00203200002023
:103C98002DE9F04F85B004469DF83C0002920027BC
:103CA8008A46039088463E4640F23F1C9B463AE0CF
:103CB800002C2FDBE1452DDCBAF1000F2ADBB8F12F
:103CC800EF0F27DC2A0702D1002DC8BF01361B4998
:103CD8002940002903DA013961F00F010131039A03
:103CE8000AB1C1F10F010E9830F8162003FA01F15C
:103CF8000A4012B272B112494A8D019392B21FFA68
:103D080089F01FFA88F1CDF800C0FFF728FFDDF829
:103D180000C0019B013509F101095D45C8DB013689
:103D2800013708F10108029A974203DAA1460025F3
:103D38000123F2E705B0BDE8F08F00BF0F00008057
:103D4800F80C002082B0044BADF80600BDF8062040
:103D580092B25A8502B07047F80C002082B0044B2A
:103D6800ADF80600BDF8062092B25A8002B070473E
:103D78003200002070B50646FFF7E2FE0020FFF78C
:103D8800A1FCF02409E0013D3046ADB2FFF7E8FCA4
:103D9800002DF8D1013CA4B214B14FF4A075F2E79C
:103DA80070BD70B51D461446FFF738FE2846FFF76C
:103DB80089FC0025054E05E0708D80B2FFF7D0FC28
:103DC8000135ADB2A542F7D170BD00BFF80C002097
:103DD8002DE9F0410C4616461F461A4600230546B3
:103DE800FFF7DFFF611E711828463A46002389B2A3
:103DF800FFF7D7FF2846214632460123FFF7D1FFB8
:103E0800013D7F19B8B2214632460123BDE8F04191
:103E1800C7E770B580B202FB03F489B292B29BB2D5
:103E2800FFF72CFE0020FFF74DFC0025054E04E0AF
:103E3800708D80B2FFF794FC0135A542F8DBBDE830
:103E480070407DE6F80C0020F8B5561A0C46013192
:103E580089B21F460546FFF7E1FD0120FFF732FC56
:103E68004FF0C04322221A800E4A0F491388B6B277
:103E7800002304E01088013321F8020B9BB2B342FF
:103E8800F8D121462846FFF7C9FD0120FFF71AFCA3
:103E9800002404E03846FFF763FC0134A4B2B442BE
:103EA800F8D1F8BD00000260226D002070B5194BF2
:103EB800194AD98D92F9004064180025A4B2AC4281
:103EC80008BF0124C62C28BFC6240F2615704FF63C
:103ED800FF7288B09E85DC855A8519200A222B46F8
:103EE8002146FFF75EFF21463046FFF742FE224695
:103EF80003460A4968460FF0F1FB6A4604A80849D8
:103F08000FF0ECFB3220D22104AA2B4600F0ECF98A
:103F180008B070BDF80C0020A45D00202FA3050890
:103F280037A305082DE9F0431F2093B0FFF722FFC0
:103F38004FF47840FFF71EFF4FF6E0754FF4FC6032
:103F4800FFF718FF2846FFF715FF0020494CFFF739
:103F580011FF00200146642203464FF6FF79A4F8BA
:103F68002A90FFF71EFF00200A2164220346FFF76C
:103F780018FF00200146642201234FF47847658525
:103F8800FFF70FFF7720EF21C82200234FF4FC66CC
:103F98006785FFF706FFBD213222012340F23F105B
:103FA8006685FFF7FEFEA020322200237821678570
:103FB800FFF7F7FEA0207821322201234FF01F08D7
:103FC8006685FFF7EEFEA020782132220223A4F8AE
:103FD8002A80FFF7E6FEA020782132220323658598
:103FE800FFF7DFFE244B2549A3F8028002AD3C22EF
:103FF80028460FF0B1FAEB20C321052230230095A3
:104008000025A4F82A900195FFF7E0FD32210A2047
:1040180096220B466785FFF7DBFE32213C2096226D
:104028000B466685FFF7D4FE32210B4696226E209A
:10403800A4F82A80FFF7CCFEFFF78DFDFFF786FD79
:104048003220FFF769F82846FFF766F86420FFF783
:1040580063F80B4B03F110028DE8240028465A68D8
:104068001B682946FFF792FD1195119B01331193A7
:10407800FBE700BFF80C0020320000207A59040842
:10408800987D010800487047F415002082B0064B5F
:10409800ADF80600BDF8062092B21A80188880B2E2
:1040A80002B0FFF74FBE00BFF0150020014B188883
:1040B80080B27047F015002082B0064BADF80600BC
:1040C800BDF8062092B21A80188880B202B0FFF7B5
:1040D80045BE00BFF2150020014B188880B270471A
:1040E800F2150020FFF746BEFFF7C8BCFFF759BE20
:1040F800FFF76EBEFFF78DBE2DE9F04F4FEA42087D
:1041080000253D4C85B082468B46C8F1030817460A
:104118002E461FFA87F909EB0B0C228805EB0A03D8
:104128001FFA8CFC9BB26146184692B2CDF804C0C7
:104138000293FFF714FDC9EB0B0292B20392029BA4
:1041480022880399184692B2FFF709FDDDF804C0EA
:104158002288C5EB0A039BB26146184692B20293C5
:10416800FFF7FDFC029B22880399184692B2FFF7DD
:10417800F6FC05EB0B0292B2039209EB0A032288C4
:1041880003999BB2184692B20293FFF7E8FC029B90
:104198002288C5EB0B0C1FFA8CFC1846614692B2BC
:1041A800CDF804C0C9EB0A09FFF7D9FC22880399A6
:1041B8001FFA89F992B24846FFF7D1FC2288DDF848
:1041C80004C092B248466146FFF7C9FCB8F1000F37
:1041D80004DA08EB860808F1060805E0F31B08F185
:1041E8000A0808EB8308013F01360135BE42ADB22B
:1041F8008FD905B0BDE8F08FF015002008B9FFF79A
:10420800AABC012801D1FFF7A1BC70477047002064
:104218000146F0224FF4A073FFF730BC704708B591
:1042280005280CD8DFE800F012140305070909482F
:1042380008BD094808BD094808BD094808BD09481E
:10424800094A0A4B40F24111FEF7F2FE084808BD40
:10425800084808BD200000201000002008000020A9
:10426800000000203CA30508B65904082EA1050843
:10427800280000201800002010B50446FFF7CFFFE3
:10428800014B18601C7110BD38000020014B1879D3
:10429800704700BF3800002008B5FFF7C0FF8088CE
:1042A80008BD08B5FFF7BBFFC08808BDF7B51F46B6
:1042B8000B4B0C4E1D681446EA882B68203C54436F
:1042C800A4B2AE1B03EB440418BF0126AB888DE8EB
:1042D800500017B1FFF7DCFC01E0FFF777FCFEBDEB
:1042E80038000020280000202DE9F0410F469846AC
:1042F80015460446084E08E0204643463946FFF76F
:10430800D5FF33689B88E418A4B215F8012B002A5E
:10431800F2D1BDE8F08100BF3800002010B5044696
:1043280008462146BDE81040DEE7094B70B5044653
:1043380018790E461546FFF7B4FFC6F1F001091AC1
:1043480089B220462A460023BDE87040CCE700BF6A
:1043580038000020704700BF044B1A680AB9044AA5
:104368001A601A681018186010467047280D002047
:10437800B08100204FF0FF30704708B50248034A6B
:10438800034B3721FEF754FE5BA30508CC590408FC
:104398002EA105080120704710B504460A480221DD
:1043A80009F0FCFB0028F9D00748214609F0BFFBBB
:1043B8000548012109F0F2FB0028F9D00248BDE8C0
:1043C800104009F0B1BB00BF0038004010B51948D3
:1043D800022109F0E3FB0028F9D01648002109F072
:1043E800A6FB1448012109F0D9FB0028F9D011488F
:1043F80009F09AFB0402A4B2002301E001339BB246
:10440800002BFBD00B48022109F0C8FB0028F9D08B
:104418000848002109F08BFB0648012109F0BEFB82
:104428000028F9D0034809F07FFB2043C0F3CB00F4
:1044380010BD00BF003800402DE9F0478AB00AAF30
:104448000A20012109F024F94FF4604347F8143D8C
:10445800474EDFF824A1012400254FF0020830461A
:1044680039468DF81A508DF818808DF819808DF816
:104478001B4008F065FD30460D21052208F0E0FDDF
:1044880030460E21052208F0DBFD052230460F21BB
:1044980008F0D6FD21464FF4804009F01DF950463A
:1044A80009F0F8F94FF48273ADF802304FF4007355
:1044B800ADF80A303823ADF80C305046072369466A
:1044C800ADF81030ADF80050ADF80450ADF8065016
:1044D800ADF80850ADF80E5009F00EFA50462146D6
:1044E80009F0A5FAA9468DF81A5030464FF48055C0
:1044F800394605958DF818408DF819808DF81B40C0
:1045080008F01EFD3046294608F08BFD4025394647
:1045180018488DF818908DF819808DF81A908DF834
:104528001B40059508F00CFD21464FF4804009F02A
:10453800DFF80621032009F069FB0C2307A88DF892
:10454800213007958DF820908DF8224008F0ECF97D
:1045580017238DF8243009A80F238DF825308DF8FE
:1045680026308DF8274005F0F9F80AB0BDE8F08745
:1045780000040240000C024000380040014B18784B
:10458800704700BF2C0D0020024B5A889B88028080
:104598000B8070472C0D0020014B00221A707047C9
:1045A8002C0D0020F0B593B06846002148220FF08A
:1045B80015F86D46002464484FF4805108F033FD27
:1045C800002301E001339BB2002BFBD09020FFF7C2
:1045D800E3FE002301E001339BB2002BFBD0FFF781
:1045E800F5FE4FF480510746574808F01AFD00239E
:1045F80001E001339BB2002BFBD053484FF48051AC
:1046080008F011FD002301E001339BB2002BFBD021
:10461800D020FFF7C1FE002301E001339BB2002B3D
:10462800FBD0FFF7D3FE4FF480510646464808F00A
:10463800F8FC45F8047B01342E6244484021E4B27A
:1046480008F0DDFC10B9092CB5D101E0092C78D1AE
:104658009DE80C00D218029B03980699D218049B77
:10466800C018059BC018079BCB180899032490FB1A
:10467800F4F092FBF4F25B1893FBF4F3151AC11AE9
:104688009C1A002DB8BF6D420029B8BF4942002CC2
:10469800B8BF6442502D03DD502909DD502C50DC91
:1046A8008D4205DAAC424FF0020405DB111806E032
:1046B8008C424FF0020401DAD11800E0C1180A9BBD
:1046C800099A0C980F9DD2180B9BD2180D9BC018F5
:1046D8000E9BC018109BEB18119D91FBF4F103245D
:1046E80092FBF4F290FBF4F05B1993FBF4F3161AC7
:1046F800C41A9D1A002EB8BF7642002CB8BF644277
:10470800002DB8BF6D42502E89B203DD502C09DD53
:10471800502D16DCA64205DAB5424FF0020405DB3F
:10472800131806E0A5424FF0020401DAD31800E09E
:10473800C318074A93FBF4F39BB29380012351807B
:10474800137013B0F0BD00BF00040240000C02401B
:104758002C0D002000000000FFF710BFF7B505463C
:104768000C4601A80DF10601FFF70EFF1B4BBDF823
:104778000660BDF8040093E80600724301FB0022BE
:1047880099685218164992FBF1F207EE102AF8EED2
:10479800C77A40F23F17FCEEE77A17EE902A92B2FA
:1047A800B2F5207F28BF3A462A801D69DA685B691E
:1047B8006E4302FB0060C01890FBF1F107EE101A7F
:1047C800F8EEC77AFCEEE77A17EE903A9BB2B3F5AB
:1047D800F07F28BFEF232380FEBD00BF340D0020EB
:1047E80040420F00FFF7D8BE014B187E704700BF4C
:1047F800340D0020FFF7C8BE042808B505D90748BE
:10480800074A084B7D21FEF713FC054B03EB80009C
:10481800038B0B80438B138008BD00BF7CA3050866
:10482800D25904089AA3050808B5082001F0B8F978
:1048380042F69643C31A584240EB030008BD10B530
:104848000A2001F0D5F90C4C20600E2001F0D0F9B7
:104858006060122001F0CCF9A060162001F0C8F9C0
:10486800E0601A2001F0C4F920611E2001F0C0F9AF
:1048780001236061237610BD340D002010B5FFF7C9
:10488800DBFD01F057FA044601F060FA07490346D8
:104898002246202004F0D4FDFFF7C6FF28B101F01E
:1048A80063FA10B9BDE81040C9E710BDD6A30508E2
:1048B80010B5104C0A20216801F081F961680E20BA
:1048C80001F07DF9A168122001F079F9E16816205C
:1048D80001F075F921691A2001F071F961691E204A
:1048E80001F06DF9082042F69641BDE8104001F04C
:1048F80049B900BF340D00202DE9F04F0346A7B099
:10490800B0F800C01C898688DF885D89CDF810C0A2
:10491800B249B0F802C0B3F80C90B3F80E80CDF8E5
:1049280024C00FFA84FB30B201220FFA87FE0BEB8A
:10493800000C0A7629B20FFA89FACDF888C001EB83
:104948000E0C0FFA88F2CDF890C00AEB0B0CCDF8DC
:1049580030C002EB010CCDF858C0B3F810C05B8A28
:10496800CDF800C00FFA8CFC06910CEB00010A91FF
:1049780002930CEB0A011BB2239103EB0E010E917B
:1049880099182591049900FA81F0584450446044DC
:10499800DDF824C006990EFA8CFEDDF810C01FFA67
:1049A80080FB1CFB0CF08E4416FB0600964414FB9F
:1049B8000400009A19FB09009E4412FB02001FFA2A
:1049C8008EFA0AF0F5F9DDF824C0029ACDE9120151
:1049D8001CFB0CF017FB070015FB050018FB080073
:1049E80012FB02000AF0E4F9DDF824C0029ACDE9CE
:1049F800140104991CFB01F317FB063615FB04662A
:104A0800009B18FB096612FB03600AF0D1F9DDE987
:104A18001423CDE90001DDE912010AF03FFA04464A
:104A28000D46DDE9000102460B460AF037FA024658
:104A38000B46204629460AF07DF8CDE9180158466C
:104A48000AF0C6F9CDE91001DDE91023DDE900011E
:104A58000AF024FACDE9060150460AF0B9F9804671
:104A680089464246DDE912014B460AF017FADDE9AC
:104A78001023CDE91C01DDE914010AF00FFA002228
:104A880006460F46564BDDE918010AF007FA42467A
:104A980004460D464B46DDE906010AF0FFF90246D9
:104AA8000B460AF049F802460B46204629460AF00A
:104AB80043F8424604460D464B46DDE91C010AF020
:104AC800EDF902460B46204629460AF033F8DDE99F
:104AD800102304460D46304639460AF0DFF90246EF
:104AE8000B46204629460AF025F8DDF828C0CDE90E
:104AF80002014FEA8C10DDF830C000EB0C20DDF825
:104B080010C0A0241CFB04000AF052F9DDF838C0DC
:104B1800CDE90A014FEA8C10DDF858C000EB0C20F3
:104B2800DDF824C01CFB04000AF042F9CDE90C01B1
:104B380050460AF03DF9DDE91023CDE91601DDE91B
:104B48000C010AF0ABF94246CDE91E014B46DDE9FE
:104B58000A010AF0A3F94246CDE920014B46DDE9F6
:104B680000010AF09BF932463B4609F0E3FFCDE924
:104B78000E0158460AF01CF9DDE91C23CDE91A019B
:104B8800DDE9060109F0D6FFDDF88CC0C024CDE9C7
:104B9800060104FB0CF0DDF888C0302505FB0C008D
:104BA800DDF810C078261CFB06000AF001F9DDF8D4
:104BB80094C0824604FB0CF0DDF890C005FB0C00A5
:104BC800DDF824C01CFB06008B460AF0F1F8DDE98D
:104BD800102306460F460AF061F903E0340D002061
:104BE800000014404246CDE904014B465046594660
:104BF8000AF054F9DDE9142380468946DDE90A0103
:104C08000AF04CF9DDE9002304460D46DDE90C0104
:104C18000AF044F902460B462046294609F08AFF65
:104C28000022A14B0AF03AF9DDE9202304460D469B
:104C3800DDE91E0109F07EFF02460B46DDE916019B
:104C48000AF02CF902460B462046294609F074FF63
:104C5800002204460D46954BDDE90E010AF01EF9C7
:104C680002460B462046294609F066FFDDE9022385
:104C78000AF03EFA88A3D3E900230AF00FF90AF0F4
:104C8800A7FB8B490860DDE91223DDE90C010AF076
:104C980005F9DDE9002304460D46DDE90A010AF0BD
:104CA800FDF802460B462046294609F043FF00223C
:104CB8007D4B0AF0F3F8DDE91E2304460D46DDE9D5
:104CC800200109F037FF02460B46DDE91A010AF018
:104CD800E5F802460B462046294609F02DFF00223A
:104CE80004460D46714BDDE906010AF0D7F8024685
:104CF8000B462046294609F01FFFDDE902230AF08A
:104D0800F7F965A3D3E900230AF0C8F80AF060FBB5
:104D1800674A5060DDE90E23DDE90A010AF0BEF8B2
:104D2800DDE9062304460D46DDE90C010AF0B6F874
:104D380002460B462046294609F0FEFE002204469C
:104D48000D465A4BDDE918010AF0A8F802460B4651
:104D58002046294609F0F0FEDDE902230AF0C8F9E9
:104D68004DA3D3E900230AF099F80AF031FB504B20
:104D780059469860DDE9142350460AF08FF8DDE9BA
:104D8800002304460D46304639460AF087F80246A5
:104D98000B462046294609F0CDFE0022424B0AF078
:104DA8007DF8424604460D464B46DDE9040109F00C
:104DB800C1FE02460B46DDE916010AF06FF802460D
:104DC8000B462046294609F0B7FE35A3D3E9002350
:104DD80004460D46DDE90E010AF060F802460B466E
:104DE8002046294609F0A8FEDDE902230AF080F9E9
:104DF80029A3D3E900230AF051F80AF0E9FADFF809
:104E0800B0C0DDE91223CCF80C00394630460AF070
:104E180045F8DDE9002304460D46504659460AF098
:104E28003DF802460B462046294609F083FE00223B
:104E38001D4B0AF033F8DDE9042304460D464046CD
:104E4800494609F077FE02460B46DDE91A010AF0E9
:104E580025F802460B462046294609F06DFE10A3A8
:104E6800D3E9002304460D46DDE906010AF016F8E9
:104E780002460B462046294609F05EFEDDE902237C
:104E88000AF036F904A3D3E900230AF007F80AF078
:104E98009FFA074908610DE00000000080842E4158
:104EA8000000000000C0824000001440000089405B
:104EB800340D0020DDE90E235046594609F0EEFF77
:104EC800DDE9062304460D463046394609F0E6FF7B
:104ED80002460B462046294609F02EFE11A3D3E9C7
:104EE800002304460D46DDE9180109F0D7FF024604
:104EF8000B462046294609F01FFEDDE902230AF089
:104F0800F7F80AA3D3E9002309F0C8FF0AF060FA0A
:104F1800034A506127B0BDE8F04FC9E4AFF3008001
:104F2800340D00200000000000C082400000000096
:104F380080842E41AFF30080064B074A5968116000
:104F48001969064A1160D969054A11609A6A054BC0
:104F58001A60704740000020FC630020AC64002009
:104F680000640020C0630020014B1878704700BF20
:104F7800500D0020032808B505D90548054A064BF9
:104F88006E21FEF755F80C235843044B185808BDFA
:104F980011A40508FE5904082BA4050840000020A8
:104FA800032808B505D90648064A074B7321FEF7BA
:104FB8003FF8064B0C2202FB0030406808BD00BFDA
:104FC80011A405080E5A04082BA405084000002067
:104FD800034B044A1B780C2101FB03239868704794
:104FE800500D002040000020034B044A1B780C2081
:104FF80000FB032399607047500D002040000020FB
:10500800144B1B78012B10B5134B144C0ED1196897
:10501800C82000F0D4FD2168CC2000F0D0FD104B52
:10502800D020196800F0CBFDD4200DE01968D820F5
:1050380000F0C5FD2168DC2000F0C1FD084BE02030
:10504800196800F0BCFDE420064B1968BDE8104063
:1050580000F0B5BDB80E0020FC630020AC64002051
:1050680000640020C0630020144B1B78012B10B58E
:10507800134C0FD1C82000F0BBFD2060CC2000F0FD
:10508800B7FD104B1860D02000F0B2FD0E4B186031
:10509800D4200EE0D82000F0ABFD2060DC2000F02A
:1050A800A7FD084B1860E02000F0A2FD064B186031
:1050B800E42000F09DFD054B186010BDB80E0020DF
:1050C800FC630020AC64002000640020C063002062
:1050D80008B502F0C0FD10B1BDE80840C4E708BD3E
:1050E8000148FCF704B800BFDC1300200148FBF7B7
:1050F800FEBF00BFDC1300200148FBF7F8BF00BF6C
:10510800DC1300200148FBF7F2BF00BFDC130020CE
:10511800032808B505D91448144A154B4B21FDF747
:1051280087FF144B1870144B02281870134B0FD0BC
:10513800032813D0012805D0114A12681A60BDE867
:105148000840CDE70F4A12681A60BDE80840CDE76D
:105158000D4A12681A60BDE80840CDE70B4A12688C
:105168001A60BDE80840CDE711A405081F5A0408D5
:1051780055A40508500D0020F2630020CC02002041
:10518800C4020020C0020020BC020020B802002097
:10519800064B07495960C021002219721E211A7056
:1051A800D9601A745A611A76DA6170472816002095
:1051B80040787D0138B5294D294C284601224FF405
:1051C800005107F032FF0321FF22C02001F094F8BC
:1051D800102120608022C02001F08EF8112120606B
:1051E8008022C02001F088F8122120608022C0208F
:1051F80001F082F8132120608022C02001F07CF8A1
:10520800142120608022C02001F076F8152120604A
:105218008022C02001F070F8162120608022C02072
:1052280001F06AF8172120608022C02001F064F89C
:1052380020600C4CB721227AC02001F05DF80022D2
:10524800012328464FF40051227462612276E261FC
:105258002370BDE8384007F0E8BE00BF00080240F0
:10526800DC6300202816002038B5C0200321FF2267
:1052780001F042F80B4D00242B19615D5A78C020CB
:10528800023401F039F8C82CF6D1B121AC22C02083
:1052980001F032F8C0200321002201F02DF800208F
:1052A80038BD00BF335A04082DE9F34706460F46B8
:1052B80092461D461AB90C1FE401914635E005EEE9
:1052C800902A06EE903AB8EE657AF8EE667AFC0116
:1052D800C7EE277AA4F500749FED5C7A67EE877AAB
:1052E80017EE900A09F086FD41EC100B0BF018FD43
:1052F80059EC108B494640460AF092F824184FEAB8
:10530800CA1009F055FDCDE90001284609F050FD05
:105318004B46424609F0C2FD02460B46DDE9000154
:1053280009F008FC0AF07CF88146002E14BF4FF003
:1053380022084FF01A08C5F307224146C02000F0A2
:10534800DBFF08F10101EAB2C02000F0D5FFC4F389
:10535800014208F10201C02000F0CEFFC4F3072289
:1053680008F10301C02000F0C7FFE2B208F1040110
:10537800C02000F0C1FFC9F3034305F4702243EADB
:10538800123208F10501C02000F0B6FF08F106014D
:10539800C9F30722C02000F0AFFF08F107015FFA48
:1053A80089F2C02000F0A8FFC020B121A02200F09F
:1053B800A3FF07EE107A264CF8EEC77A0EBBD4EDA1
:1053C800015A06EE90AAB8EE657A05EE905AB8EE44
:1053D800666AF8EE656A0123C6EE266A237477EEDC
:1053E800A67A67EE277A17EE900A09F003FD41ECDA
:1053F800100B0BF095FC51EC100B0AF011F86061E2
:1054080020E005EE90AAD4ED016AB8EE656A05EED3
:10541800905AB8EE667AF8EE656A0123C6EE266AF7
:10542800237677EEA67A67EE277A17EE900A09F0C8
:10543800E1FC41EC100B0BF073FC51EC100B09F084
:10544800EFFFE0610020BDE8FC8700BF00000043DB
:10545800281600200022012326E7012838B50D462A
:1054680004D002280CBF3C242C2400E0342421461C
:10547800C02001F03DF805F0070200F00F0040EAF7
:1054880002122146C020BDE8384000F035BF2DE9A2
:10549800F3470A9C1D4607468A461646524B01E0CA
:1054A8006D0864089C42FBD82DB906F10076043ECD
:1054B800F601A94634E006EE905AB8EE667A06EE92
:1054C800904AF8EE667AF601C7EE277AA6F50076D6
:1054D8009FED467A67EE877A17EE900A09F08AFC04
:1054E80041EC100B0BF01CFC59EC108B4946404664
:1054F80009F096FF3618E80109F05AFCCDE90001D9
:10550800204609F055FC4B46424609F0C7FC0246C6
:105518000B46DDE9000109F00DFB09F081FF81462A
:10552800022F9BBF324BDB194FF0000893F8C8805D
:10553800C4F307224146C02000F0DEFE08F1010155
:10554800E2B2C9B2C02000F0D7FE08F10201C9B228
:10555800C6F30142C02000F0CFFE08F10301C9B232
:10556800C6F30722C02000F0C7FE08F10401C9B243
:10557800F2B2C02000F0C0FE04F47024C9F3034363
:1055880008F1050143EA1432C9B2C02000F0B4FEA4
:1055980008F10601C9B2C9F30722C02008F10708BB
:1055A80000F0AAFE5FFA89F25FFA88F1C02000F0E5
:1055B800A3FEBAF1010F0CBF2F220F220DB942F042
:1055C8004002012F06D002D3022F0AD105E0C020E5
:1055D800102104E0C020112101E0C020122100F0B8
:1055E8008BFE0020BDE8FC87FFFF0F000000004392
:1055F800335A040807B5012300930023FFF747FF38
:105608000EBD00280CBFFF22002208B5C0200321D0
:1056180000F072FE002008BD08B5C020B121AC2200
:1056280000F06AFE002008BD704708B500F050F988
:1056380000F050F9014B00221A7008BD540D0020EB
:10564800024B187880F00100704700BF540D00200D
:10565800014B1878704700BF540D002008B54FF46F
:1056680000710F4807F0CBFC0E4BD0F101005A78BF
:1056780038BF0020824201460ED05A681D2A0DDC30
:1056880001321E2A5A6009D15870074800225A6010
:10569800BDE8084003F0DEBF00225A6008BD00BF25
:1056A80000080240540D0020B1A40508014B5878A9
:1056B800704700BF540D002010B500210446012298
:1056C800302000F019FEC0B9012001F0B7F8002C15
:1056D800B8BF4034E4B210212246302000F00CFE5E
:1056E800012001F0ABF830201121224600F004FE21
:1056F8000120BDE8104001F0A1B810BD10B500218F
:1057080004460122302000F0F7FDC0B9012001F065
:1057180095F8002CB8BF4034E4B21221224630205C
:1057280000F0EAFD012001F089F83020132122461B
:1057380000F0E2FD0120BDE8104001F07FB810BD87
:10574800002810B5044603DB5F2CA8BF5F2400E0E7
:10575800002430200021012200F0CEFDA8B901204C
:10576800E4B201F06BF83B212246302000F0C4FD82
:10577800012001F063F830203C21224600F0BCFDF6
:105788000120BDE8104001F059B810BD302810B50F
:1057980004460ADC10F17F0F02DB002802DB05E07B
:1057A8006FF07E0404F5807400E03024002130207E
:1057B8000A4600F0A1FDA8B90120E4B201F03EF8C4
:1057C80041212246302000F097FD012001F036F8F3
:1057D80030204221224600F08FFD0120BDE8104014
:1057E80001F02CB810BD282810B5044609DC10F1CA
:1057F800180F02DB002802DB04E06FF017047F3487
:1058080000E02824002130200A4600F075FDA8B9E0
:105818000120E4B201F012F853212246302000F0B2
:105828006BFD012001F00AF830205421224600F0D7
:1058380063FD0120BDE8104001F000B810BD08B5B7
:1058480030200021012200F057FD60B9012000F04E
:10585800F5FF30203321402200F04EFD0120BDE845
:10586800084000F0EBBF08BD10B530200021012230
:1058780000F042FD044660B9012000F0DFFF30204F
:105888003321224600F038FD0120BDE8104000F029
:10589800D5BF10BD10B530200021012200F02CFD2D
:1058A8000446A0B9012000F0C9FF34212246302067
:1058B80000F022FD012000F0C1FF302037212246F0
:1058C80000F01AFD0120BDE8104000F0B7BF10BD80
:1058D8004020F1E6402011E708B5002101223020E0
:1058E80000F00AFD012000F0A9FF30203421024613
:1058F80000F002FD012000F0A1FF30203721024610
:1059080000F0FAFC0120BDE8084000F097BF08B598
:1059180000210122302000F0EFFC012000F08EFF72
:10592800302034210C2200F0E7FC0120BDE80840BB
:1059380000F084BF00000000704770477047704750
:10594800254B2DE9704F0024D3E900ABD3E9028938
:105958002546224E03E0C246CB4680468946A85FCC
:1059680009F036FA01341AA3D3E9002309F0C0FB81
:10597800A4B25B46524609F0DDF823B20435FF2B8A
:10598800E9DD174A144B14800025002445EC174B19
:10599800C3E9040183ED007B83ED027B02460B46DD
:1059A80009F07CFA424604460D464B4640464946B5
:1059B80009F074FA0B4602462946204609F0BCF85D
:1059C80009F006FD074B1860BDE8708FAFF3008043
:1059D800000000000040BF40600D0020A4550020DA
:1059E800D45D0020C41D00202DE9F84F2E4B2F4A0E
:1059F80019682F4B19B92F4911602F4A02E02F4916
:105A080011602F4A1A602F4BDFF8C0B0DFF8C09042
:105A180000221A80254A9846176840F2FF1A31E09A
:105A280007EB84036500B3F9023007EE103AF8EE8D
:105A3800C77A013617EE900A09F0DCF918A3D3E902
:105A4800002309F02BFA09F0C3FC29F815002BF8FC
:105A5800140037F9243007EE103AF8EEC77A01350A
:105A680017EE900A09F0C6F90DA3D3E9002309F04F
:105A780015FA09F0ADFC144B29F8150023F81400A9
:105A8800A8F80060B8F8006034B25445C8DD00F0EA
:105A98005DF800F069F801F0CFFABDE8F84F4FE77C
:105AA8009A9999999999E93FB01D0020DC1C00202A
:105AB800D01A002068260020681E00209844002084
:105AC800502F0020D45D002048400020283C0020B2
:105AD800A455002010B50B4C204606F07EFE0A4B5C
:105AE80018600A4806F079FE094B1860FFF77CFF3A
:105AF800084B0949012220461A83BDE8104006F0E8
:105B0800EDBE00BF10600240B01D0020886002405A
:105B1800601E0020600D002020800010014B1868D6
:105B2800704700BFC41D002008B5054B05481988FB
:105B3800002201230AF0E4F8034B187008BD00BFE7
:105B4800700000208C5500202C5100200348044987
:105B5800044A4FF400730AF04BB900BF74000020E8
:105B6800283C00207037002003480449044A4FF4B9
:105B780000730AF03DB900BF8000002048400020B3
:105B88004816002038B505460C460135C1F30721F3
:105B980000F062FEA8B2E1B200F05EFE00B238BDCD
:105BA80038B5044600F06CFD01340546A0B200F09B
:105BB80067FDEDB2C0B240EA052000B238BD37B586
:105BC8000B0E8DF804300B0C8DF805300B0A8DF890
:105BD80006308DF80710002400E0284601AB451C6C
:105BE800E15C013400F038FE042CADB2F5D13EBDC5
:105BF80037B5002400E02846451C00F041FD01AB04
:105C0800ADB2E0540134042CF5D19DF805009DF89F
:105C18000430000440EA03609DF8073018439DF8FB
:105C2800063040EA03203EBD38B50446642000F043
:105C380005FE25786068AD00EDB2257007F0E5F93E
:105C4800237A40FA03F000F003000543104B257057
:105C580005F00F055A5D6378D218D2B2D3B201327B
:105C6800D2B2022A637001D80022A2705BB2012B63
:105C780003DD0123A3700023637094F9013001331D
:105C880003DAFF23A3700023637094F9020038BD80
:105C9800045B0408F7B504200121234F07F0F8FC42
:105CA80002AD01214FF48040012407F021FD0026B8
:105CB8004FF4B0733846694645F8083D8DF80460DE
:105CC8008DF8074007F03CF91020214607F0E0FC6A
:105CD80078236946154800938DF804608DF80740CD
:105CE80007F02EF90420214607F0D2FC21464FF494
:105CF800804007F0FDFC1E233846694600938DF866
:105D080004608DF8074007F01BF90220214607F0D0
:105D1800BFFCB02306488DF8046069468DF807403B
:105D2800009307F00DF9FEBD000802400010024084
:105D380000040240802108B5034807F060F9D0F15B
:105D4800010038BF002008BD0004024008B54FF428
:105D58008071044807F053F9D0F1010038BF0020E2
:105D680008BD00BF0008024008B5FFF7E3FF08B10F
:105D7800FFF7ECFFC0B208BD10B5642000F05EFD6F
:105D88000F48FFF751FF044610B90E4B187009E091
:105D9800FFF7DCFF30B9002C0A4B01DD012200E0DF
:105DA800FF221A700848FFF73FFF0028074B01D170
:105DB800187010BD01DD012200E0FF221A7010BD2D
:105DC800F000002004640020FC000020A45D0020F6
:105DD80007B50220012107F05BFC012300938DF831
:105DE800043002238DF805300448002369468DF8F5
:105DF80006308DF8073007F0A3F80EBD0004024006
:105E080010B5084C01210022204607F00EF940F297
:105E1800FF4000F013FD012120460A46BDE810406E
:105E280007F003B90004024008B5FFF7E9FF0021B5
:105E38000A46302000F060FA012000F0FFFC012142
:105E48000A46302000F058FA012000F0F7FC002143
:105E58000122302000F050FA012000F0EFFC01216F
:105E68000822302000F048FA012000F0E7FC022167
:105E78000122302000F040FA012000F0DFFC002170
:105E88000A46302000F038FA012000F0D7FC1B2128
:105E9800CD22302000F030FA012000F0CFFC0421A0
:105EA8000322302000F028FA012000F0C7FC062168
:105EB8000822302000F020FA012000F0BFFC072162
:105EC8000A46302000F018FA012000F0B7FC08213B
:105ED8008022302000F010FA012000F0AFFC1E21D3
:105EE800B022302000F008FA012000F0A7FC0521BC
:105EF8009122302000F000FA012000F09FFC0D21D3
:105F08000322302000F0F8F9012000F097FC0E2160
:105F18000022302000F0F0F9012000F08FFC14215D
:105F28008022302000F0E8F9012000F087FC0B21E6
:105F38008822302000F0E0F9012000F07FFC3020BA
:105F48000C21822200F0D8F9012000F077FC122100
:105F58008822302000F0D0F9012000F06FFC1321D6
:105F68008C22302000F0C8F9012000F067FC0021E5
:105F78000122302000F0C0F9012000F05FFC0C2164
:105F88000822302000F0B8F9012000F057FC0D215C
:105F98000822302000F0B0F9012000F04FFC0E215B
:105FA8000822302000F0A8F9012000F047FC0F215A
:105FB8000822302000F0A0F9012000F03FFC002169
:105FC8000A46302000F098F9012000F037FC402103
:105FD8000222302000F090F9012000F02FFC00226E
:105FE8004121302000F088F9012000F027FC302002
:105FF8003F21D42200F080F9012000F01FFC00218D
:106008000122302000F078F9012000F017FC10215F
:106018000F22302000F070F9012000F00FFC112150
:106028000F22302000F068F9012000F007FC12214F
:106038000022302000F060F9012000F0FFFB13215E
:106048000022302000F058F9012000F0F7FB092168
:106058003C22302000F050F9012000F0EFFB002135
:106068000122302000F048F9012000F0E7FB302041
:106078003421024600F040F9012000F0DFFB302017
:106088003721024600F038F9012000F0D7FB36210D
:106098000322302000F030F9012000F0CFFB392135
:1060A8000322302000F028F9012000F0C7FB3B2133
:1060B8003C22302000F020F9012000F0BFFB3C21F9
:1060C8000A46302000F018F9012000F0B7FB002143
:1060D8000A46302000F010F9012000F0AFFB5121F2
:1060E800C022302000F008F9012000F0A7FB302082
:1060F8005221002200F000F90120BDE8084000F01C
:106108009DBB00BF2DE9F04F434E444D91B0012196
:106118004FF4001007F0BCFA304606F05FFA404B27
:106128004FF0C0628DE80C003E4B00244FF48067AE
:106138004FF400694FF400584FF4807A4FF4003B55
:106148003046694602930497069703940594CDF860
:106158001C90CDF82080CDF824A0CDF828B00B9461
:1061680006F0C8FA224630462F4906F01EFB304694
:10617800012106F024FB01210A464FF0402007F0D8
:10618800F5FC284606F02AFA284B04970193284B79
:106198000697029328464023694603930094059482
:1061A800CDF81C90CDF82080CDF824A0CDF828B0EB
:1061B8000B9406F09FFA224628461E4906F0F5FA87
:1061C8002846012106F0FBFA42F21077012202214B
:1061D800194807F0CBFC384600F030FB3046012167
:1061E80006F0C3FA0121284606F0BFFA384600F047
:1061F80025FB0B238DF83C300FA801238DF83D407B
:106208008DF83E408DF83F3003F0A8FA384600F08C
:1062180015FB11B0BDE8F08F1060024088600240A5
:106228000C40004098440020682600200C3C0040A8
:10623800502F0020681E0020003C0040024810211A
:10624800012206F009BB00BF1060024013B502200E
:10625800012107F01DFA4FF410730E4C009302232E
:106268008DF804308DF8053001238DF8063020466E
:10627800002369468DF8073006F062FE20460621A5
:10628800042206F0DDFE20460921042206F0D8FE8D
:106298001CBD00BF0004024030B5154D85B001217A
:1062A8004FF4001007F018FA284606F0DFFE002326
:1062B800ADF804304BF6FF73ADF806303323ADF874
:1062C80008304FF48063ADF80A304FF48043ADF8DE
:1062D8000C3004AC074B2846012144F8103D06F069
:1062E80067FF2846694606F0EFFE05B030BD00BFDF
:1062F80000540040801A060073B54FF49613064602
:106308000D461446019304E0019B5A1E0192002B8E
:1063180057D031484FF4003107F062F80028F3D124
:106328002D48012106F050FF4FF48053019304E0FB
:10633800019B5A1E0192002B45D02748274907F098
:106348003AF80028F4D024483146002206F054FFD9
:106358004FF48053019304E0019B5A1E0192002BD5
:1063680033D01D481E4907F026F80028F4D01A48F3
:10637800294606F0C4FF4FF48053019303E0019BC4
:106388005A1E01921BB31448164907F014F8002846
:10639800F5D01148214606F0B2FF4FF49613019349
:1063A80003E0019B5A1E01929BB10B480E4907F06E
:1063B80017F80028F5D00848012106F011FF002041
:1063C80008E0012006E0022004E0032002E00420A7
:1063D80000E005207CBD00BF005400400100030020
:1063E800820007008000070004000010F7B51F4670
:1063F8004FF4961306460D461446019304E0019B9C
:106408005A1E0192002B5ED034484FF4003106F03A
:10641800E7FF0028F3D13148012106F0D5FE4FF4FB
:106428008053019304E0019B5A1E0192002B4CD02B
:106438002A482B4906F0BFFF0028F4D027483146E8
:10644800002206F0D9FE4FF48053019304E0019B2B
:106458005A1E0192002B3AD02048224906F0ABFF81
:106468000028F4D01D48294606F049FF4FF4805310
:10647800019304E0019B5A1E0192002B29D0174872
:10648800194906F098FF0028F4D000254FF4961615
:1064980010E0615D114806F032FF019603E0019BB0
:1064A8005A1E0192BBB10D48104906F099FF002809
:1064B800F5D00135EBB2BB42EBD30848012106F019
:1064C8008FFE002008E0012006E0022004E00320FF
:1064D80002E0042000E00520FEBD00BF005400409B
:1064E800010003008200070080000700040000107C
:1064F80037B54FF4961304460D46019305E0019B0A
:106508005A1E0192002B00F09B8056484FF4003130
:1065180006F066FF0028F2D15248012106F054FE29
:106528004FF48053019305E0019B5A1E0192002B02
:1065380000F088804B484C4906F03DFF0028F3D016
:1065480048482146002206F057FE4FF48053019335
:1065580004E0019B5A1E0192002B75D04148434923
:1065680006F029FF0028F4D03E48294606F0C7FE69
:106578004FF48053019304E0019B5A1E0192002BB3
:1065880064D038483A4906F02BFF0028F4D0354843
:10659800012106F019FE4FF48053019304E0019B9A
:1065A8005A1E0192002B53D02E482F4906F003FFA4
:1065B8000028F4D02B482146012206F01DFE4FF496
:1065C8008053019304E0019B5A1E0192002B41D095
:1065D800244C2849204606F003FF0028F3D0204623
:1065E800002106F011FE20460121238B06F0F8FD5C
:1065F8004FF48053019304E0019B5A1E0192002B33
:106608002AD018481C4906F0EBFE0028F4D015489B
:1066180006F077FE4FF480530193124A03E0019B82
:10662800591E0191D3B113889B05F8D40121044662
:106638000C4806F0E9FD0B48104906F0EBFE0EE0A9
:1066480001240CE002240AE0032408E0042406E004
:10665800052404E0062402E0072400E0082420467C
:106668003EBD00BF00540040010003008200070047
:106678000400001002000010400000100004001088
:1066880013B54FF496130446019305E0019B5A1E77
:106698000192002B00F0B08061484FF4003106F001
:1066A8009FFE0028F2D15E48012106F08DFD4FF4CF
:1066B8008053019305E0019B5A1E0192002B00F0C4
:1066C8009D805748574906F076FE0028F3D0544875
:1066D800A021002206F090FD4FF48053019305E0BD
:1066E800019B5A1E0192002B00F08A804C484E49AB
:1066F80006F061FE0028F3D0C4F30521484806F0EF
:10670800FEFD4FF48053019304E0019B5A1E019251
:10671800002B77D04248454906F062FE0028F4D0A5
:10672800E1B23F4806F0EBFD4FF48053019304E0DB
:10673800019B5A1E0192002B66D039483B4906F04E
:106748004FFE0028F4D03648012106F03DFD4FF4F5
:106758008053019304E0019B5A1E0192002B55D0EF
:106768002F48304906F027FE0028F4D02C48A121F4
:10677800012206F041FD4FF48053019304E0019B90
:106788005A1E0192002B43D0254C2949204606F079
:1067980027FE0028F3D02046002106F035FD2046CC
:1067A8000121238B06F01CFD4FF48053019304E074
:1067B800019B5A1E0192002B2CD019481D4906F046
:1067C8000FFE0028F4D0164806F09BFD4FF48053C6
:1067D8000193134A03E0019B591E0191E3B1138809
:1067E8009905F8D4012104460D4806F00DFD0C4822
:1067F800114906F00FFE10E001240EE002240CE01F
:1068080003240AE0042408E0052406E0062404E042
:10681800072402E0082400E0092420461CBD00BF2C
:10682800005400400100030082000700040000102B
:1068380002000010400000100004001082B0002385
:1068480004E0019B01330193009B01330093009BFB
:106858008342F6D302B0704737B54FF480530446ED
:106868000D46019304E0019B5A1E0192002B6ED045
:106878003D484FF4003106F0B3FD0028F3D13A4803
:10688800012106F0A1FC4FF48053019304E0019B21
:106898005A1E0192002B5CD03348344906F08BFD18
:1068A8000028F4D03048A021002206F0A5FC4FF4BF
:1068B8008053019304E0019B5A1E0192002B4AD099
:1068C80029482B4906F077FD0028F4D0C4F30521A8
:1068D800254806F014FD4FF48053019304E0019B12
:1068E8005A1E0192002B38D01F48224906F063FD3A
:1068F8000028F4D0E1B21C4806F001FD4FF48053A3
:10690800019303E0019B5A1E019243B316481949AB
:1069180006F051FD0028F5D01348294606F0EFFC93
:106928004FF49613019303E0019B5A1E0192C3B1E1
:106938000D48114906F054FD0028F5D00A480121F8
:1069480006F04EFC0D48FFF779FF00200AE0012011
:1069580008E0022006E0032004E0042002E005200D
:1069680000E006203EBD00BF0054004001000300C7
:10697800820007008000070004000010A0860100C4
:1069880013B50520012106F083FE184C4FF4E0539F
:10699800009302238DF804308DF80530204600233B
:1069A80069468DF806308DF8073006F0C9FA20469A
:1069B8000A21062206F044FB20460C21062206F096
:1069C8003FFB062220460B21A4F5006406F038FBA5
:1069D8004FF4004320466946009306F0B1FA20467A
:1069E8000F21062206F02CFB1CBD00BF0008024048
:1069F8001FB50446FFF7ECF9FFF74EFCFFF714FA52
:106A0800FFF7BEFF01214FF4004006F065FE029437
:106A18000F4C1023ADF80230204600236946ADF82C
:106A28000430ADF80C30ADF80030ADF8063006F0A3
:106A380082FF69464FF0402007F051F820460121B7
:106A480007F001F84FF04020012106F0FCFF1FBDC0
:106A5800003C0040014B1860704700BF8C0D0020BF
:106A6800704710B50A4A1379262B04D80949C85427
:106A78000133137110BD074A0123591ED45C013339
:106A8800272B5454F9D1034B83F8260010BD00BFBF
:106A98008C0D0020A85D0020704710B504462078B2
:106AA800FFF7DFFF14F8013F002BF8D110BD38B510
:106AB80004460D46013D14F8010BEDB2FFF7D1FF76
:106AC800002DF7D138BD00BF014B1878704700BFC3
:106AD800940D0020014B5878704700BF940D00209A
:106AE800024B187880F00100704700BF940D002019
:106AF800024B00221A705A70704700BF940D002094
:106B0800014B01221A707047940D0020014B01229D
:106B18005A707047940D002082B0002304E0019B56
:106B280001330193009B01330093009B8342F6D30A
:106B380002B070470148024904F02ABE0C5E0020EA
:106B48000C64002007B50420012106F0A1FD0121F5
:106B58004FF4804006F0CCFD4FF4007300930023FF
:106B68008DF804300348012369468DF8073006F094
:106B7800E7F90EBD0008024038B506EE900A1E4B34
:106B8800B8EEE67AD3ED007ADFED1C6A27EE877A55
:106B98001B4B87EE267ABDEEC77A83ED007AB8EEF6
:106BA800C77A77EE877A17EE900A08F023F9154B23
:106BB80004460D46C3E9004522462B460CA1D1E9FF
:106BC800000108F095FA104BD3E9002308F066F9A4
:106BD8000E4B2246C3E900012B4600200C4908F061
:106BE80087FA0C4BC3E9000138BD00BFAFF3008042
:106BF800182D4454FB211940D81B00200024744947
:106C0800243C0020F81D0020D01C0020D01D0020AE
:106C180000003040F01B00201F4B002030B51860EA
:106C28001E4B18601E4B00240025186045EC174BBE
:106C38001C4B83ED007B1C4B4B221A601B4B3222F2
:106C48000DA5D5E900451A60194BC3E900450CA507
:106C5800D5E90045174BC3E900450BA5D5E9004523
:106C6800154BC3E900450AA5D5E90045134BC3E90F
:106C78000045BDE830407FE7182D4454FB21F93F1B
:106C8800E0F09C762F1BA43F9F14F9CFD4C2F93FA4
:106C980091458FD82181F83F243C0020DC1B00203F
:106CA800D81C0020C04C0020E01C0020981D0020AB
:106CB800D01D0020D81D002030400020183C0020A6
:106CC8002DE9F843284B294C294D012251EC100B92
:106CD8001A6023A3D3E9002308F0E0F8254BD3E991
:106CE800002308F005FA244B06460F460020002131
:106CF800C3E9006741EC170B204B83ED007B204B69
:106D08001A68204B002A0CBF282204221A601E4B46
:106D1800D3E90089304642464B46394684ED007B2C
:106D280007F00AFF194B4246C3E900014B463046BB
:106D3800394607F0FFFE00220023C5E9000108F0EC
:106D480029FB18B194ED007B85ED007B104A0023E8
:106D58001360104A1360BDE8F88300BFAFF30080EA
:106D6800182D4454FB211940E41C0020E03B00206E
:106D7800183C0020F81D0020D01D0020D03B00202A
:106D8800E01D0020083C0020D81D002030400020D5
:106D9800783B0020D83B00202DE9F843284B08B960
:106DA800186005E001241C6040F6B833984200D012
:106DB8000024244B244D1C6008F00AF81EA3D3E9D4
:106DC800002308F06BF8214BD3E9002308F090F971
:106DD8001F4B06460F46C3E900671E4BD3E9000167
:106DE8001D4BD3E9002307F0A7FE32463B468046F9
:106DF800894607F0A1FE194B3246C3E900013B461C
:106E08004046494607F096FE00220023C5E90001E6
:106E180008F0C0FA28B10022002343EC172B85EDB7
:106E2800007B00220CB10E4B00E00E4B0E49C1E96D
:106E38000023BDE8F88300BF182D4454FB211940F6
:106E48007C3B0020E01D0020183C0020F81D00209D
:106E5800D81D0020D01D0020C04C0020304000204C
:106E680000003E4000005940F83B00201249002332
:106E780001225A500433402BFBD1104B03F1A802D6
:106E880000200021E3E902019342F9D10C4B0A22C8
:106E98001A600C4A002313600B4A13600B4A04A1C2
:106EA800D1E9000113600A4BC3E90001704700BF34
:106EB8000000000000805640101E0020E81C002042
:106EC800081E0020E81B002038400020B84C002095
:106ED800003C002007EE100A38B5F8EEC77A304BB0
:106EE800C3ED007AFFF7C2FF0020FFF745FE2D4BE8
:106EF8002D492E4832221A6000220023C1E90023BE
:106F0800002101602A4801602A4801602A4801607E
:106F18002A4801602A48C0E900232A48C0E900231A
:106F28002948016029480524046029480160294846
:106F3800C0E900232848C0E900232848C0E9002305
:106F4800274815A5D5E90045C0E900232548C0E92B
:106F580000452548C0E90023C0E902232348C0E9C9
:106F68000023C0E902232248C0E900232148C0E9E0
:106F78000023214B1960214B1960214B1960214BCB
:106F880001221A60204B19602049214B002041EC56
:106F9800170B83ED007B38BD9A9999999999D93F38
:106FA800D81B0020081E002028400020641E002056
:106FB800041E0020001E002058370020B81D0020A5
:106FC800703B0020F81B0020C81D0020103C00204A
:106FD800203C0020702E0020503700204040002028
:106FE800F03B0020003C0020C81B0020B81B0020FC
:106FF800E03B0020482F0020C01D0020E83B002077
:10700800083C0020E41C0020E01D0020000059403E
:10701800F83B0020064A08B500231360054A4FF4E0
:10702800FA501360FFF756FFBDE80840F4E500BFCB
:10703800CC640020B86400202DE9F04F284B1A6872
:1070480093B0002A40D0013A002A1A60254A3EDC53
:1070580000211960244B1160D3E90067234BD3E961
:107068000045304622462B46394607F065FD204B41
:107078002246C3E900012B463046394607F05AFD3F
:107088001C4C1D4B804689461868C4E9008907F0E6
:10709800B1FE02460B463046394607F0FFFE0EA306
:1070A800D3E9002308F024F8144B0022C3E90001B7
:1070B80040464946002308F06DF928B10022002314
:1070C80043EC172B84ED007B00270D4C1AE00123BD
:1070D8001360F9E7AFF30080182D4454FB211940E1
:1070E800083C0020E41C0020D01D0020D81D0020F2
:1070F80030400020183C0020D81B0020D01C002065
:10710800980D0020844BFD5A844B2580FE5A844BF1
:107118006680D3E90001834BD3E9002307F00CFD17
:107128007BA3D3E9002307F0B9FE08F051F963689F
:107138007D4AC018011101F580610905090D6060DB
:10714800C0F30B100DF1480C32F8203032F8212032
:10715800616A238115FB02F0628115FB03F516FBBA
:1071680002F216FB03F60CEB4103E0602561C0F365
:10717800CF30C5F3CF356261A661C2F3CF32C6F313
:10718800CF3623F8200C23F8105C23F8182C23F8AA
:10719800086C664BA08301310B40002BE5832284E9
:1071A800668403DA013B63F003030133604A5362E8
:1071B800002B40F0A2805F480AA92832042309F076
:1071C800D7F85D485D4A0EA9042309F0D1F85C4858
:1071D8005C4A0CA9042309F0CBF85B4A5B480423FA
:1071E80010A909F0C5F8B4F9280007F0F1FD8046A8
:1071F800B4F92A00894607F0EBFDCDE90001B4F99E
:107208002C0007F0E5FD8246B4F92E008B4607F006
:10721800DFFD4246CDE902014B464046494607F0AC
:107228003DFECDE90401DDE9000102460B4607F009
:1072380035FE02460B46DDE9040107F07DFC41EC12
:10724800100B09F0F9FE524684ED0C0B5B465046D4
:1072580059468DED040B07F021FECDE90601DDE965
:10726800020102460B4607F019FE02460B46DDE90D
:10727800060107F061FC41EC100B09F0DDFEDDE9C9
:10728800000184ED0E0B52465B468DED060B07F0B0
:1072980005FE42464B46CDE90801DDE9020107F04B
:1072A800FDFD02460B46DDE9080107F043FC5246A6
:1072B800CDE908015B464046494607F0EFFDDDE9A8
:1072C800022380468946DDE9000107F0E7FD024612
:1072D8000B464046494607F02FFC9DED080B41EC54
:1072E800110B09F021FEDDE9040184ED100BDDE945
:1072F800062307F0FDFEC4E912010237B7F5806FD7
:107308007FF400AF13B0BDE8F08F00BFAFF300808B
:1073180039D6C56D305FC44070370020481600204C
:10732800D01D0020C04C0020285B0408030000800A
:10733800980D0020E4000020D8000020C20D002095
:10734800CC000020C40D0020C60D0020C000002085
:107358002DE9F04F8C4B1B6889B08DED000B8DED3E
:10736800021B6BB90020002141EC170B874B83ED02
:10737800007B874B83ED007B864B83ED007BE2E04F
:10738800854D864CD5E902ABD4E90023DDE900013F
:1073980007F0D0FB52465B4607F080FDD5E900892F
:1073A800D4E9022306460F46DDE9020107F0C2FBD5
:1073B80042464B4607F072FD02460B4630463946B8
:1073C80007F0B8FB9DED007B85ED007B9DED027B12
:1073D800C4E90089C4E902AB85ED027B5CA3D3E96B
:1073E800002306460F4607F0E9FF10B158A7D7E972
:1073F80000673046394658A3D3E9002307F0C0FF99
:1074080010B155A7D7E90067604C55A3D3E900230D
:10741800D4E9000107F042FD002280468946304643
:1074280039465F4B07F03AFD0B460246494640464F
:1074380007F082FB5B4B1B6806460F46C4E90067F2
:107448001BB343A3D3E9002307F0B8FF38B930468C
:10745800394641A3D3E9002307F092FF78B142A34C
:10746800D3E900233046394607F018FD4E4C024652
:107478000B46D4E9000107F05FFBC4E90001304680
:1074880039463BA3D3E9002334E0414BD3E90089D3
:1074980042464B4607F002FD0022002307F08EFF0C
:1074A80018B94FF000084FF000094046494628A394
:1074B800D3E9002307F082FF38B94046494626A39E
:1074C800D3E9002307F05CFF78B12BA3D3E90023AD
:1074D8004046494607F0E2FC334C02460B46D4E9E5
:1074E800000107F029FBC4E9000125A3D3E9002323
:1074F8004046494607F0D2FC264B2B4C254DC3E9A4
:107508000001D4E90001D5E9002307F015FB274B5A
:10751800D3E9006732463B468046894607F04EFF6E
:1075280048B9234BD3E900674046494632463B46B3
:1075380007F026FF38B10020002141EC170BC4E901
:10754800006785ED007B09B0BDE8F08FAFF30080E0
:10755800333333333333D33F333333333333D3BF1B
:10756800D7A3703D0AD7EF3F54E41071732AC93E80
:107578002D431CEBE2363A3F54E41071732AB93EAE
:10758800FCA9F1D24D62503F7C3B0020E03B00203B
:10759800D03B0020C04C0020C81B0020B81B002096
:1075A8000000D03FE41C0020D01D00203040002007
:1075B800183C0020014B93ED120B7047980D0020EA
:1075C800014B93ED100B7047980D0020014B93ED84
:1075D8000C0B7047980D0020014B93ED0E0B704774
:1075E800980D0020AFF3008010B5FDF7E3FD0020F3
:1075F800012324210246FDF757FE114B1C78002079
:10760800012C05D10146FDF728FF2046002104E0A2
:107618000721FDF722FF01200721FDF71EFF632246
:107628001221C020FEF768FE02200121FDF715FF98
:10763800FDF7F2FF0120BDE81040FDF7E2BF00BFF3
:10764800B80E0020054B1B78012B05D1044B054AC9
:10765800196812688A181A60704700BF085E00200F
:1076680008640020045E0020054B1B78012B05D11F
:10767800044B054A196812688A1A1A60704700BFD5
:10768800085E002008640020045E0020024B1A688F
:10769800024B1A60704700BFF463002008640020A2
:1076A8002DE9F04F824658488BB0B0FBF1F00C46FC
:1076B80007F07EFB41EC100B09F032FB51EC100B8C
:1076C80007F0AEFEC307074648BF471E04FB07F096
:1076D80007F06EFB46A3D3E9002307F009FD044633
:1076E8000D4645EC104B09F01BFB59EC108B20465E
:1076F80042464B46294607F01DFACDE904014946A2
:10770800404607F08DFE3CA3D3E900230990DDE94C
:10771800040107F03FFE00283DD1002401234FF06B
:107728001509224698462046DFF8E4B003E02346D0
:1077380042462C46B04600FB04355D452ED800FB7A
:107748000826DDE904012EA3D3E9002307F022FE71
:1077580030BBDDE9042300202C4907F0C9FC41ECCB
:10776800100B0390029109F0DBFA0398029953EC8D
:10777800102B8DED060B07F0DDF909F1FF39CDE986
:1077880004015FFA89F9DDE9060107F049FEB9F15C
:10779800000FCCD104E00125002601E0254646462D
:1077A800099BD9B2BAF1000F0BD132462B4650468D
:1077B800FDF77AFD01230093504651463A46534659
:1077C80009E032462B460120FDF76EFD01200090AE
:1077D80001463A460023FDF75AFEFDF71DFF01203A
:1077E8000BB0BDE8F04FFDF70CBF00BFAFF3008052
:1077F8000000000084D77741956479E17FFDA53DBD
:10780800BBBDD7D9DF7CDB3D00E9A4350000F03FE4
:10781800FFFF0F001F4B1B78022B10B539D01E4BF2
:107828001E4A19681E4B1F4C1B68CB1893422360D5
:1078380018DC0020FFF734FF01202168FFF730FF34
:10784800194B1C780020012C05D10146FDF705FED7
:107858002046002104E00721FDF7FFFD0120072154
:10786800FDF7FBFD114B1B78022B12D10A4C104B74
:1078780022681B689A420CDA0E4B1B78012B08D140
:107888000D4B186800F074F80C4B22681B68D3186D
:10789800236010BD206D00200864002080D1F0080E
:1078A800A4640020A8640020B80E0020085E002010
:1078B800E4630020E0630020C0630020045E002031
:1078C80008B5FEF737FA0A4B5A78187002435A700F
:1078D80022B99B78064A012B05D808BD9A7801324F
:1078E8009A7018B9F5E700235370937008BD00BF6C
:1078F800E80D002007B50420012105F0C9FE4FF46A
:107908006043009301238DF8043002238DF805307D
:107918000548002369468DF806308DF8073005F0D4
:107928000FFB03B05DF804FB00080240084B4FF45E
:107938007A721B68B3FBF2F3064A013B5360064BAD
:10794800F02183F823100023936007231360704706
:10795800E002002010E000E000ED00E0034B5A6870
:1079680012B15A68013A5A60704700BFE80D00200A
:10797800024B58605A68002AFCD17047E80D002075
:107988007FB55D4A5D4D06460C4610685168128900
:1079980001AB03C31A802B78032B10D8DFE803F060
:1079A8000205080B01A8564907E001A8554904E05B
:1079B80001A8554901E0554901A80BF0B7FE04ABF1
:1079C800981910F80C1C2144C9B22F2901D80A3182
:1079D80002E0392901D90A39C9B200F80C1C4FF65E
:1079E800FF70FCF753FB0020FCF746FC0DF1030683
:1079F8000F24204623345A2116F8012F0023A4B25D
:107A0800FCF754FCB4F5A57FF3D164205A212C224D
:107A18000023FCF74BFC0023CD205A212C22FCF735
:107A280045FC0020FCF732FB2B78032B62D8DFE8FB
:107A380003F002284B5601A931480BF077FE0A22C1
:107A48002F4800210CF016F8314A324B1278186092
:107A5800012A06D1304A9042DCBF01321A602F4A0F
:107A680006E0B0F5FA5FBCBF4FF4FA521A602C4A30
:107A78001B689342C4BF274B1A602A4B1A682A4BCB
:107A880020E001A91F480BF051FE0A221D480021E1
:107A98000BF0F0FF1E4A254B12781860012A06D118
:107AA8001D4A9042DCBF01321A601C4A06E0B0F55C
:107AB800FA5FBCBF4FF4FA521A60194A1B68934226
:107AC80018DD1A4B1A6015E001A90F480BF02EFEBD
:107AD8000D4800210A220BF0CDFF154B09E001A942
:107AE8000A480BF023FE094800210A220BF0C2FFC6
:107AF800104B186004B070BD66A50508F26300203D
:107B0800CE630020E863002090640020C463002056
:107B1800B80E0020FC6300203F420F0080D1F0081F
:107B280040420F00F463002008640020AC64002089
:107B380000640020C063002010B50D4B0D4C1A687E
:107B48000D4821460BF0CAFD0C4B0D481A6821461A
:107B58000BF0C4FD0B4B0C481A6821460BF0BEFD18
:107B68000A4B0B481A682146BDE810400BF0B6BD19
:107B7800FC63002070A50508CE630020AC640020DB
:107B8800E86300200064002090640020C0630020A7
:107B9800C463002008B500210A220D480BF06AFFD3
:107BA8000C4B002118600A220B480BF063FF0B4BAB
:107BB800002118600A220A480BF05CFF094B0021DB
:107BC80018600A2208480BF055FF084B186008BDDA
:107BD800CE630020FC630020E8630020AC64002032
:107BE8009064002000640020C4630020C06300206B
:107BF800014B93ED020B7047E80D0020014B93ED0C
:107C0800040B7047E80D0020034B83ED000B83ED58
:107C1800021B83ED042B7047987E0020014B1860EF
:107C2800704700BF08640020014B1868704700BF08
:107C3800FC630020014B1868704700BFAC6400204B
:107C480008B54FF49570FDF7ABFF40F26523C31AF2
:107C58005842584108BD08B5C620FDF7A1FF40F2BB
:107C68008D13C31A5842584108BD4FF4957040F21D
:107C78006521FDF787BFC62040F28D11FDF782BF51
:107C880008B5F8F78BFD51EC100B07F0C9FB01465E
:107C98004FF49670FDF793FFF8F786FD01464FF411
:107CA8009870FDF78CFFF8F785FD51EC100B07F085
:107CB800B7FBBDE8084001464FF49A70FDF77FBF57
:107CC800F8B5FFF7BDFF224CC0B14FF49670FDF731
:107CD8008FFF07F06DF8C4E906014FF49870FDF7BF
:107CE80087FF07F065F8C4E908014FF49A70FDF7BB
:107CF8007FFF07F05DF8C4E90A010EE00EA3D3E99F
:107D08000023C4E906230EA3D3E90023C4E908230A
:107D18000DA3D3E90023C4E90A23D4E90867D4E909
:107D28000A01D4E906450B4BC3E90045C3E90267DC
:107D3800C3E90401F8BD00BF8FC2F5285C8FF03F8E
:107D4800F6285C8FC2F5064011EA2D819997913D7E
:107D5800E80D0020987E002051EC110B2DE9F84326
:107D680011EE102A0B4657EC106B07F097F800221B
:107D780004460D4630463946184B06F0DDFE3246BD
:107D8800804689463B463046394607F087F8224602
:107D98002B4606F0D1FE0022104B06F0CBFE4246E1
:107DA80006460F464B464046494607F077F82246B6
:107DB8002B4606F0C1FE02460B463046394607F010
:107DC80097F90022064B07F069F80022054B06F0E8
:107DD800B3FE07F0FDFA9F30BDE8F8830000F03FDE
:107DE800000059400000E03F2DE9F84351EC100B2A
:107DF8000022194B55EC114B06F09EFE00228046DE
:107E0800894620462946154B07F048F8424606465B
:107E18000F464B464046494607F040F82246804602
:107E280089462B462046294607F038F802460B4675
:107E38004046494606F080FE02460B463046394623
:107E480007F056F90022064B06F076FE07F0C0FA56
:107E58007730BDE8F88300BF0000F03F00006940BC
:107E68000000E03F2DE9F043754C2DED048B0FCC5D
:107E780097B06D460FC594E80F00103485E80F00E1
:107E88000FCC08AD0FC50FCC0FC50FCC0FC594E8AC
:107E98000300642285E803004FF6FF739F207721D3
:107EA800F9F783FFA020772164224FF6FF73F9F7D3
:107EB8007CFF9E20772164224FF6FF73F9F775FF48
:107EC8009F20762164224FF6FF73F9F76EFF4FF675
:107ED800FF73782164229F20F9F767FF0020FBF7E2
:107EE80031FF9F2077216522FCF706F99F20772133
:107EF8006422FCF701F96C460DF12008B4EC028B02
:107F0800504F4FF4967500264BA3D3E90023304613
:107F1800394606F0C3FF00224A4B06460F4606F0D4
:107F280009FEB0EE480AF0EE680A41EC110B41EC8C
:107F3800190BFFF711FFB0EE480AF0EE680AB0EE31
:107F4800491AF0EE691A8146FFF74EFF0F2281B2F7
:107F58001FFA89F0FBF703FE013DD5D1394F002602
:107F68004FF4967534A3D3E900233046394606F01A
:107F780095FF06460F4632463B460020314906F03B
:107F8800D9FDB0EE480AF0EE680A41EC110B41EC5D
:107F9800190BFFF7E1FEB0EE480AF0EE680AB0EE02
:107FA800491AF0EE691A8146FFF71EFF0F2281B2C7
:107FB8001FFA89F0FBF7D3FD013DD3D144459DD18C
:107FC8000DF15808B4EC028B1E4F4FF4C87500260B
:107FD80019A3D3E900233046394606F05FFF002293
:107FE800184B06460F4606F0A5FDB0EE481AF0EE0F
:107FF800681A41EC100B41EC190BFFF7ADFEB0EE1F
:10800800490AF0EE690AB0EE481AF0EE681A81469D
:10801800FFF7EAFE002281B21FFA89F0FBF79FFD05
:10802800013DD5D14445CDD117B0BDEC048BBDE899
:10803800F08300BFAFF30080295C8FC2F528F03FC2
:10804800289B04080000F03FF8B50446101A0D46B6
:1080580006F0BEFE0646281B0F4606F0B9FE02468D
:108068000B463046394607F043F80022024B06F02B
:1080780015FF07F0ADF9F8BD00007440F8B50546E6
:10808800881A0C4606F0A4FE0646601B0F4606F04A
:108098009FFE02460B463046394607F029F8002273
:1080A800024B06F0FBFE07F093F9F8BD00006940AB
:1080B80070B505460E460024630704D5A0B22946CC
:1080C8003246FBF74CFD0134B4F5A07FF4D170BD06
:1080D80070B505460E460024630704D52846A1B2AC
:1080E8003246FBF73CFD0134C82CF5D170BD104B6E
:1080F80010481B78104A1149012B114BF0B51B6829
:10810800104F114D114E124C06D13B6033682B6055
:10811800236803600B6809E0DB013B603368DB011F
:108128002B602368DB0103600B68DB011360F0BD83
:10813800B80E0020045E0020A4640020D86300204C
:10814800FC630020F4630020E4630020AC6400209A
:1081580000640020024B1A68024B1A60704700BF87
:10816800F46300200864002008B5FFF7C0FFBDE8ED
:108178000840FFF7EFBF70B50024013823462022DE
:10818800303A092A264610F8015F04F101040CD898
:10819800032296FBF2F202EB4202964205D12C2210
:1081A800CA54CA180233557001E0CD540133092C62
:1081B8002A46E5D12022CA540B4448225A707A2212
:1081C8009A700022DA7070BD70B58CB005460C4606
:1081D80068460E491E460BF081FA684604A9FFF767
:1081E800CAFF04AA0A4908A80BF078FABDF84000AB
:1081F800FBF74CFF3046FBF75FFF2846214608AAED
:108208000023FCF771F80CB070BD00BF76A5050817
:1082180037A305082DE9F04FAF4B2DED048B1B78E4
:10822800022BC7B000F03E85AC4B1A78AC4B22B994
:108238001A68802392FBF3FB01E0D3F800B0DFF863
:10824800C4A2A84CA84DFFF7B5F98AED0C0BFFF7AF
:10825800B7F9DAE91001B0EE408AF0EE608ADAE99F
:108268000C678AED0E0B02460B4606F065FC32469B
:108278003B4606F061FC00229C4B06F039FFCAE938
:108288000201CAE91001D4E9000132463B46C5E9BA
:10829800000106F003FEB0EE480AF0EE680A94ED1D
:1082A800047BD4E9028906460F468DED047BC5E9B7
:1082B8000289CAE90C6708F0DBFCB0EE409AF0EEE0
:1082C800609AB0EE480AF0EE680A08F0D1FD304630
:1082D80053EC102B394606F0E1FD53EC192B0446FC
:1082E8000D463046394606F0D9FD002206460F46AF
:1082F800404649467E4B06F01FFC00227D4B06F0A7
:10830800F7FE02460B463046394606F013FC024695
:108318000B468046894606F0C1FD224606460F46B2
:108328002B462046294606F0B9FD02460B46304644
:10833800394606F001FC00226E4B06F0AFFD0646FA
:108348000F464046494632463B4606F0D1FE324685
:10835800CDE902013B46204605F1004106F0C8FE82
:10836800CDE90C01CAE90401584606F031FD50A3D5
:10837800D3E9002306F092FDDDE9042306F08EFD23
:1083880002460B46DDE90C0106F0D4FBCDE90401F9
:10839800DDE9020102460B4606F080FDCDE9080141
:1083A800DDE9040102460B4606F078FDCDE90A0135
:1083B800DDE90801DDE90A2306F0BEFB04460D46A7
:1083C80022462B46DDE9020106F092FE059BCDE927
:1083D8000601224603F1004104982B4606F088FE68
:1083E80035A3D3E900238046894606F0E7FF60B944
:1083F8004046494632A3D3E9002306F0C1FF40B105
:108408000FF2BC09D9E9008903E00FF2AC09D9E9F8
:1084180000899DED067B384B424683ED007BC3E91E
:10842800028940464B46494606F038FD002204467C
:108438000D46324BDDE9060106F07CFB02460B4691
:1084480006F02CFD22462B4606F076FB41EC100B7D
:1084580008F0F2FDDDE906010022284B57EC106B0D
:1084680006F06AFB02460B4606F018FD22462B462C
:1084780006F062FB41EC100B08F0DEFD304653ECD1
:10848800102B394606F034FE0FA3D3E90023044627
:108498000D4606F075FFB8BB204629460022184B4A
:1084A80006F08CFF98B30AA5D5E900452FE000BF78
:1084B8001F85EB51B81E1940000000008087C3409B
:1084C800000000008087C3C02D431CEBE2361A3F32
:1084D8001EA7E8482EFFEF3F206D0020B80E0020B1
:1084E80008640020987E0020D00200200000084088
:1084F8000080514000005E40106D0020000049409F
:108508000000F03FE80D0020D8A5D5E90045C04E91
:10851800C04FC6E90045DDE90401B3A3D3E9002350
:1085280006F0BCFCDDE90823C7E9020141EC180BA1
:10853800AFA1D1E9000106F0FDFADDE90A2306F052
:10854800F9FAB0EE480AF0EE680A41EC110BC7E9F7
:10855800000108F0E9FC53EC102B03F100438DED0A
:10856800080A09939DED087B002286ED027BAA4B41
:108578002046294606F0E0FA224606460F462B46D4
:108588000020A54906F0D6FA02460B463046394681
:1085980006F0AEFD98A3D3E90023CDE90A0106F061
:1085A8000DFF50B9DDE90A0195A3D3E9002306F0D0
:1085B800E7FE30B19FED927B01E09FED8F7B8DED63
:1085C8000A7B964B1B78022B33D1954F3E68002EC1
:1085D8002FDB06235E4306F57A76B6B23046594657
:1085E800FDF7EDFA00228F4B2046294606F056FC8F
:1085F80006F016FF06F1040A1FFA8AFA01B250467D
:10860800FDF7C0FA80A3D3E90023DDE9080106F0ED
:1086180045FC06F0DDFE0636B6B201B23046FDF77F
:10862800B1FA3B680133B3F5FA7FC8BF4FF0FF33A7
:108638003B60FEF7CBFF7C4E86ED120BFEF7CCFFBE
:1086480086ED140BFDF76AFA7849B0655A463EA8DC
:108658000BF044F87649D6E912232EA80BF03EF821
:108668007449D6E9142332A80BF038F87249DDE9C9
:10867800022336A80BF032F87049DDE90C233AA83A
:108688000BF02CF8DDE906236D491AA80BF026F843
:108698006C4942464B461EA80BF020F86A49224610
:1086A8002B4622A80BF01AF86849DDE9082326A80A
:1086B8000BF014F8DDE90A2365492AA80BF00EF837
:1086C80042A86449B26D0BF009F8544B1B78013B82
:1086D800012B00F2D982604B1B78072B00F2D48261
:1086E800DFE813F00800D202C8004F01A901FF011A
:1086F800A3025C020220FBF7BFFD4FF6FF70FBF7F9
:10870800DBFC1F20FBF7C2FC1921544A00232D2053
:10871800FBF7EAFD4FF6FF700024FBF7CDFC0020C5
:10872800FBF7B4FC5A4600940F20B4214FF6FF73B0
:10873800FFF74AFD2EAA23460F207721FBF7D4FD29
:1087480032AA2346A0207721FBF7CEFD22AA234692
:108758000F204121FBF7C8FD26AA2346A02041216E
:10876800FBF7C2FD36AA23460F206521FBF7BCFDA7
:108778003AAA2346A0206521FBF7B6FD1AAA23468C
:108788000F205321FBF7B0FD1EAA2346A02053213A
:10879800FBF7AAFD0F202AAA9B212346FBF7A4FD7D
:1087A800B36DB3F57A7FCCBF4FF4FC604FF47840DB
:1087B800FBF782FC42AAA0209B210023FBF794FD33
:1087C800274B1B78012B4FF48C704FF002010CBF24
:1087D800244A254A0023FBF787FD1F20FBF76CFC82
:1087E80052E200BFAFF300807B14AE47E17AA43FAA
:1087F8002D431CEBE2363A3F000000008087C3405F
:10880800000000008087C3C0CDCCCCCC0C5FC44036
:10881800F86C0020D06E00200000F03F085E0020B9
:10882800F86300200000F040E80D00207BA5050853
:1088380085A5050890A505089BA50508A5A5050813
:10884800AFA50508BAA50508C5A50508D0A505085A
:10885800DBA50508E7A50508A0640020F4A5050820
:10886800B80E002013A6050817A605082D431CEB13
:10887800E2361A3FDDE9022314A8BB490AF02EFFAD
:10888800DDE90C2317A8B9490AF028FFDDE906231A
:108898000EA8B7490AF022FF42464B4611A8B5492F
:1088A8000AF01CFF14AAE62002210023FBF71CFD96
:1088B80017AAE62016210023FBF716FD0EAA0220B0
:1088C800C8210023FBF710FD11AA0220DC21002398
:1088D800FBF70AFD0022A84B2046294606F0DEFADF
:1088E8009DED080B0D46044608F0C2F9B0EE408A2B
:1088F800F0EE608A9DED080B08F0BAFA4FF6E076C4
:10890800002059EC108BFBF7D7FB5A460A210023AD
:1089180000960520FFF758FC4FF47840FBF7B6FBAC
:1089280053EC182B2046294606F0B8FA82A3D3E95F
:10893800002306F001F906F04BFD424687B24B468C
:108948002046294606F0AAFA02460B467CA1D1E940
:10895800000106F0EFF806F03BFD81B23846F9F762
:1089680054FA9D20772105220023FBF7BFFB9F20A7
:10897800752105220123FBF7B9FB3046FBF786FB7F
:1089880082E17E4B18687E4B5A461968FFF75CFBFC
:10899800B0F59F7FC2BF7B4B02221A7004460022AB
:1089A800DDE90601784B06F0EBFCF8B1DDE90601DC
:1089B8000022002306F002FDC0B1DDE9060106F041
:1089C80007FDC0F5FA7006F003FA00226E4B06F0B8
:1089D8008FFB00226D4B06F061FA06F0F9FCA5B298
:1089E80081B24FF6FF722846FBF7B9F84046494670
:1089F8000022654B06F0C4FC002800F04581404683
:108A0800494651A3D3E9002306F0D8FC002800F01A
:108A18003B814946404606F0DBFCC0F5FA7006F09B
:108A2800D7F900225A4B06F063FB0022574BA4B239
:108A380006F034FA50E0514B1868514B5A46196801
:108A4800FFF702FBB0F59F7FC2BF4E4B02221A70A0
:108A580004460022DDE90201002306F0AFFCE0B184
:108A6800DDE902013AA3D3E9002306F089FCA0B1AD
:108A78000022484BDDE9020106F010FA02460B46D7
:108A88000020424906F056F806F0A2FCA5B281B2D1
:108A98004FF6FF722846FBF762F8DDE904012EA3C2
:108AA800D3E9002306F08AFC002800F0ED80DDE918
:108AB800040127A3D3E9002306F062FC002800F094
:108AC800E3800022324BDDE9040106F0E7F90022D9
:108AD800294BA4B206F030F806F07AFC81B22046A1
:108AE800A0E0204629461EA3D3E9002306F066FC31
:108AF800002800F0C980214B1868214B5A46196894
:108B0800FFF7A2FAB0F59F7FC4BF1E4B022245ECC7
:108B1800104BC8BF1A70064608F008FA002251EC3C
:108B2800100B1D4B06F0BAF906F052FCB6B281B232
:108B38003046A5E0AFF300800000000000E063408D
:108B48000000000000C05D400000000000407FC041
:108B58009A9999999999B93F9A9999999999B9BF6F
:108B680076711B0DE02DA03F1BA6050825A605085C
:108B78002FA6050839A6050800005940FC63002007
:108B8800AC640020206D002000407F400000694058
:108B980000408F4000409F40000054C0DDE90801BC
:108BA8000022454B06F07AF941A3D3E9002306F0E9
:108BB8009FFA424B06461868414B5A460F461968B9
:108BC800FFF742FAB0F59F7FC2BF3E4B02221A70F0
:108BD8001FFA80F800223C4B2046294606F05EF931
:108BE8000B4602463849002005F0A4FF06F0F0FBCA
:108BF8004FF6FF7281B24046FAF7B1FF3946304668
:108C080006F0E6FBC0F1B40006F0E2F800222A4BB9
:108C180006F06EFA00222C4B06F040F906F0D8FB5D
:108C280081B240464FF4FC622CE0DDE90A010022E3
:108C3800264B06F0A5FB38B3204B1868204B5A4644
:108C48001968FFF701FAB0F59F7FC4BF1D4B0222D8
:108C58009DED0A0BC8BF1A70044608F067F9002298
:108C680051EC100B194B06F019F902460B4600207F
:108C7800154905F05FFF06F0ABFBA4B281B22046B0
:108C88004FF6FF72FAF76BFF114B1B7813F0FD0FCD
:108C980008D04FF6FF7300930520DC215A460023C5
:108CA800FFF792FA47B0BDEC048BBDE8F08F00BF28
:108CB8001F85EB51B81E194000807640FC630020E8
:108CC800AC640020206D002000006940000059407D
:108CD800A0640020F7B5044600283ED0204E308816
:108CE80001210444FAF79AFE0120FAF7EBFCA4B23A
:108CF800A5B200271B4B33F817000137FAF730FDF0
:108D0800C62FF7D12046C72201214FF6FF73FBF784
:108D18009BF8154B35801C68144B1B682DB21B1B28
:108D280007EE103A07EE905AB8EEC77AF8EEE77AEF
:108D380067EE877A17EE900A06F05CF800220C4B73
:108D480006F0D6F906F044FB4FF6FF73221800939D
:108D58000520DC210023FFF737FA03B0F0BD00BF80
:108D6800F06C0020226D0020FC630020AC64002021
:108D78000000744013B5114CB4F85C30ADF80630FF
:108D8800BDF806309BB25BB1BDF806004FF6FF7325
:108D980080B20121C722FBF757F80023A4F85C3002
:108DA800074B1B78022B06D1064C94F90000FFF7FD
:108DB80091FF0023237002B010BD00BFE80D002012
:108DC800206D0020A45D002070477047FEE7FEE795
:108DD800FEE7704770477047FEF7C0BD08B5022030
:108DE80003F0FCFD48B1054BD3F880305B69984728
:108DF8000220BDE8084003F0FFBD08BD0C64002058
:108E080000F05CBA014802F0D5BA00BF0C5E002041
:108E1800704700BF414BD3F8882042F47002C3F872
:108E280088203F4B1A6842F001021A6000229A60BB
:108E3800196821F0847121F4803119603949596029
:108E4800196882B021F480211960DA6000920192D9
:108E58001A6842F480321A601A6802F400320192E9
:108E6800009A01320092019A1AB9009AB2F5A06FDD
:108E7800F2D12B4B1B6813F4003318BF0123019365
:108E8800019B012B2ED1264B1A6C42F080521A649A
:108E9800254A116841F4804111609A689A609A687D
:108EA80042F400429A609A6842F4A0529A601F4ABB
:108EB8005A601A6842F080721A601968184A890163
:108EC800FBD51B4B40F205611960936823F003033F
:108ED8009360936843F002039360936803F00C0374
:108EE800082BFAD10E4B9A6822F400029A60114AB4
:108EF800C3F884201A6842F080621A601A68120166
:108F0800FCD5064B4FF000629A60D3F8882042F4F3
:108F18007002C3F8882002B0704700BF00ED00E07F
:108F28000038024010300024007000400854400708
:108F3800003C024080400030184B194A996801F003
:108F48000C01042903D0082903D0164B19E0164B4D
:108F580017E059685A6811F4800F596814BF124B0A
:108F6800104B02F03F02B3FBF2F30C4A5268C2F313
:108F78000142C1F38811013252004B43B3FBF2F3B3
:108F8800074A1360054B9A68054BC2F303129A18F7
:108F98001968127921FA02F21A6070470038024003
:108FA800E00200200024F40000127A0008B54020F6
:108FB80003F014FD30B1FBF7F5FA4020BDE8084096
:108FC80003F01ABD08BD0000014608B5044805F0C5
:108FD800CFFC0348402105F078FD0028F9D008BDF2
:108FE80000440040F0B589B04FF4E133012001930B
:108FF80000232B4CADF808301E460146ADF80A3068
:10900800ADF80C30ADF810300C23ADF80E3004F08C
:109018003FFB4FF40030012104F05EFB2068022181
:10902800072204F00DF807226068032104F008F80D
:109038000125022704232068059305A98DF81A60E5
:109048008DF81B508DF818708DF8197003F078FFA3
:1090580008236068059305A98DF8187003F070FF60
:10906800A06801A905F0DAFB2A4640F225510D480F
:1090780005F012FD262307A88DF81C308DF81D6019
:109088008DF81E608DF81F5000F068FBA068294617
:1090980005F041FC044A054B1A6009B0F0BD00BF59
:1090A800F402002000440040D18F0008F87E002020
:1090B800024B9868002105F02EBC00BFF402002086
:1090C80010B5074C40F22551204605F008FD28B19F
:1090D800044BA2881988D2B24A401A8010BD00BF3A
:1090E80000440040480E00201FB5214B0C46186074
:1090F80000214FF0804004F02CFF012100224FF0A6
:10910800804005F056FA022C01D10B2303E0012C14
:1091180002D142F6DF6302930523ADF804304FF025
:109128008040002301A9ADF80C30ADF8063004F0FA
:109138007BFE4FF08040012105F05BFA4FF0804044
:10914800012104F0E4FE01210A464FF0804005F0B9
:1091580030FA4FF08040012104F0FBFE044B1968FF
:109168000029FCD14FF0804004F0F3FE1FBD00BF82
:109178004C0E00207047F0B5012085B02D4D0146FA
:1091880004F086FA4FF4D0530026019303270223F4
:10919800284601A98DF808308DF809708DF80A6005
:1091A8008DF80B6003F0CCFE284609210A2203F053
:1091B80047FF28460B210A2203F042FF0A222846CD
:1091C8000C2103F03DFF01244FF48063284601A9D8
:1091D80001938DF80A408DF80B408DF8097003F063
:1091E800AFFE0A210A46284603F02AFF21464FF41B
:1091F800804004F07DFA8020214604F055FA31467B
:109208004FF0006000F0DEFA4FF4A06000F09CFA26
:109218001C2303A88DF80C308DF80D608DF80E40D6
:109228008DF80F4000F09AFA2046214604F054FACF
:1092380005B0F0BD0000024007B54FF4C06000F073
:1092480083FA43238DF8043001A801238DF80530F3
:109258008DF806308DF8073000F080FA0EBD04480E
:1092680011B9012103F0DDBE012103F0DCBE00BF0E
:1092780000080240022137E7012135E737B504200D
:1092880001210D4D04F004FA022301248DF8053064
:109298002846002369468DF806308DF8073000947B
:1092A8008DF8044003F04CFE2846214603F0B9FE31
:1092B800C820FFF7E1FF3EBD0008024008B54FF0A7
:1092C8008040012105F08AF988B101214FF08040E2
:1092D80005F08FF9064B196819B11A68013A1A6036
:1092E80008BD4FF08040BDE8084004F032BE08BD1C
:1092F8004C0E00207047012070470349034A0220A2
:109308004FF4B77300F09CB843A60508989B04086F
:109318000349044A022040F2371300F091B800BF15
:1093280043A60508A89B04080349044A022040F202
:10933800011300F085B800BF43A60508C59B0408C3
:109348000249034A0220F52300F07AB843A605082B
:10935800DE9B04080249034A0220EA2300F070B8A1
:1093680043A60508F89B04080249034A0220DF23A4
:1093780000F066B843A60508109C04080249034A91
:109388000220C82300F05CB843A605082D9C0408F9
:109398000249034A0220BC2300F052B843A605083C
:1093A800529C04080249034A0220A62300F048B848
:1093B80043A60508719C04080249034A02208B232E
:1093C80000F03EB843A605088F9C04080249034AEA
:1093D8000220802300F034B843A60508AC9C04089A
:1093E8000249034A0220682300F02AB843A6050868
:1093F800C19C04080249034A0220522300F020B805
:1094080043A60508DB9C0408FDF772BBFDF778BB93
:1094180004490A6801320A6003490346022000F041
:109428000FB800BF500E002064A60508FDF76EBBFC
:1094380080F08000092801D8FDF72EBB704700BFD7
:109448000EB403B070470A2810B5044602D10D20A7
:10945800FFF7F9FF064A13681BB103F8014B1360C5
:1094680010BD044B1B680BB12046984710BD00BFC8
:10947800540E0020F87E002010B5044601E0FFF7E6
:10948800E2FF14F8010B0028F9D110BD2DE9F04FC7
:10949800044685B00D464FF00A0A00E035462078AC
:1094A800002800F0C480252801D0013467E06078E6
:1094B800302803D1A0780123033407E02D2802D0F7
:1094C8000234002302E0A078022303344FF000089E
:1094D80005E00AFB080814F8010BA8F13008A0F110
:1094E8003002D2B2092AF4D96C2801D04C2803D111
:1094F80014F8010B43F00403002800F0988060285A
:1095080086BFA0F12002D2B202464F2A3DD006D82B
:10951800432A2DD0442A09D0422A30D133E0552A93
:1095280004D0582A29D0532A29D101E00A272DE04E
:109538002E1D2F68002500E001357A5D002AFBD139
:1095480004E02020FFF77FFF4D4601E0980704D490
:10955800454505F10109F4D34D463846FFF78CFF20
:1095680003E02020FFF76FFF01354545F9D395E764
:1095780028782E1DFFF767FF90E7102706E0FFF712
:1095880062FF2E468AE7022700E008272E1D442A9C
:10959800296804D1002902DA494243F0080300226D
:1095A80000E02A46B1FBF7FE07FB1E11CDB2092DDC
:1095B800714607D9782814BF4FF0070C4FF0270CD5
:1095C8006544EDB230350DF80250551CBEF1000F60
:1095D80002D0102DE5D10F22190705D504A94D1980
:1095E8002D2105F8101C951C13F0010F0CBF4FF02E
:1095F800200B4FF0300B9B072F4604D508E0584648
:10960800FFF721FF4F46474507F10109F7D34F46BA
:10961800013D1DF80500FFF716FF002DF8D103E006
:109628002020FFF710FF01374745F9D336E705B08B
:10963800BDE8F08F70B5064D0C462E68286001E035
:10964800FFF701FF14F8010B0028F9D12E6070BD57
:10965800F87E00200FB407B504A951F8040B019156
:10966800FFF714FFBDE80E4004B070470EB417B5FD
:1096780005A9084C51F8043B206018460191FFF7F2
:1096880005FF2268002313702360BDE81E4003B065
:10969800704700BF540E00200EB433B505A9074C1F
:1096A80051F8043B2568206018460191FFF7EEFE4B
:1096B8002560BDE83C4003B0704700BFF87E00203D
:1096C80070B51E4604461C481546FFF7C3FF022E18
:1096D8001FD0042E25D0012E2AD105E0A15D174800
:1096E800FFF7B8FF013600E00026AE42F6DB202087
:1096F800FFF7A9FE002609E0A05DA0F12003DBB278
:109708005E2B88BF2E20FFF79EFE0136AE42F3DBAC
:109718000EE034F8021B0A48FFF79CFF013DF8D120
:1097280006E054F8041B0748FFF794FF013DF8D101
:109738000A20BDE8704086E687A605088EA60508BB
:1097480094A605089AA6050840F0BE60024B40F4AE
:109758002020D860704700BF00ED00E0C37810B546
:1097680003B3164B4278DB688478DB43C3F30223E8
:10977800C3F10401C9B202FA01F10F2242FA03F25D
:10978800C9B222400A430E4B01781201CB18D2B25B
:1097980083F8002303780122590903F01F0302FA12
:1097A80003F307E003780122590903F01F0302FAC3
:1097B80003F32031024A42F8213010BD00ED00E0E9
:1097C80000E100E021F0604121F07F01014B0843F6
:1097D8009860704700ED00E0044B1A6909B1104326
:1097E80001E022EA00001861704700BF00ED00E0C8
:1097F800044B1A6804280CBF42F0040222F0040249
:109808001A60704710E000E037B50023104C019350
:1098180005460320FFF72EFDEB681A69013C01920B
:1098280013D0019A002AF4DA019A42F00102019257
:10983800019A1A61064A1969013A019102D00199FF
:10984800C907F8D40320FFF715FD00203EBD00BF6F
:10985800410D030010B5C47874B900EB82000333DE
:109868009B10D0F8D000224603E051F8044C013296
:10987800046004319A42F8D1002010BD033230B59B
:109888009210D0F8D0400B46002003E02568013044
:1098980043F8045C04339042F8D101EB800030BDFA
:1098A8000122F0B50023827040220129C370828012
:1098B8000CD108230370042343704FF4A073C380B2
:1098C80002230372C1724FF0A04309E041B90C238F
:1098D8000370062343704FF4A063C3801F4BC1720B
:1098E80003F500620261C3604678044601461A46E1
:1098F800002508E002F5106C02F530620A65C1F82F
:1099080014C001353A460431B54202F12007F1D3BB
:1099180003F58062426103F58862C0F8CC200678BE
:1099280003F5A0650146002203E0C1F88C5001321E
:1099380020350431B242F8D31946002202E0C4F8B7
:10994800CC1001320434B24201F58051F7D303F54B
:109958006063C0F80C310020F0BD00BF0000044077
:1099680038B5037AC2680025012B04461FD1936BD2
:10997800417A65F3104309B143F480139363D368C4
:109988006FF386136FF396536FF351436FF3D3431B
:10999800D3602046FFF738FFE378012B19D1052360
:1099A80063F34405E36845F020059D6011E0D36842
:1099B80043F04003D360FFF727FF637AE268002B88
:1099C8000CBF4FF404134FF4441393631420FFF7B0
:1099D80053FCE378012B07D1E3689D68052262F305
:1099E800440545F020059D60002038BDC3689A688D
:1099F80042F001029A6000207047C3689A6822F01A
:109A080001029A600020704707B500230193019B6B
:109A180043F020030193019B61F38A130193019B97
:109A2800C2681361064B1169013B019102D001998B
:109A38008806F8D40320FFF71DFC00200EBD00BFE8
:109A4800410D030007B500230193019B43F0100368
:109A58000193019BC2681361064B1169013B019197
:109A680002D00199C906F8D40320FFF703FC0020AF
:109A78000EBD00BF410D030008B5C268D3680129B7
:109A88006FF35D736FF39E7302D143F0005302E0EE
:109A980009B943F080433220D360FFF7EDFB002083
:109AA80008BDC368586900F001007047C3685B6966
:109AB80013F0010F14BF002001207047C3685869D4
:109AC80000F001007047C3685A69986910407047F0
:109AD800C3685868704743699B6813F0010F14BF47
:109AE800002001207047C36800229A614FF0FF32BE
:109AF8005A615A606FF080425A610B4A9A61C27883
:109B08009969002A0CBF1022002242F0487221EA0B
:109B180002010A439A619A6922F0005222F008026F
:109B28009A610020704700BF0008008043691A68E6
:109B380061F301021A607047D0F8CC3018686FF3EF
:109B480082006FF341006FF3C3006FF34510704755
:109B580038B504460D46FFF782FB2046FFF7ECFFB9
:109B6800C0F3072303F01003DBB233B9012D04D18E
:109B7800D4F8CC3040F480501860C0F3072303F0C9
:109B88001003DBB22BB125B9D4F8CC3065F30C3017
:109B98001860C820BDE83840FFF76EBB43695869B4
:109BA800704738B50546FFF7C7FFD5F8CC3040F405
:109BB80080741C606420FFF75FFBD5F8CC306FF32E
:109BC800082414201C60FFF757FB012038BD70B52E
:109BD8000446FFF753FBD4F80C3100251D60237AA7
:109BE800012B08BF2946204618BF0121FFF79EFF19
:109BF8002046FFF7D6FF63691A686FF382021A607E
:109C0800E37A012B2E460ED1E36880225A6262F372
:109C18000F05E02262F30F06C0F26005C0F260068D
:109C28009D62C3F8006110212046FFF7EDFE204633
:109C3800FFF708FF002322464FF0FF35184604E0DF
:109C4800D2F88C1001338D60C860217804328B42C1
:109C5800F6D320460121FFF77BFF2046FFF743FF9D
:109C6800002070BD70B500EB810301F11504D3F835
:109C7800902000EB44154FF0FF339360C37895F8BC
:109C88001551012B0CBF04230023032D2BD8DFE82B
:109C980005F0021F021300EB411404F56C7443F045
:109CA8008903A57843F482637DB9247943F040039E
:109CB800CCB143F0200316E000EB411443F09903C4
:109CC80094F8B24343F4C0636CB143F480730AE080
:109CD80000EB441443F0010394F8124143F4087371
:109CE8000CB143F4C073D360436901249D6904FA3D
:109CF80001F42C439C61C3689C69153100EB411049
:109D080044F000749C6190F81011002361F39C5397
:109D180090F8111161F3CE2390F8121161F3CF334B
:109D280090F81311A1F1020CDCF1000141EB0C01D8
:109D380061F3514390F8151100F58874B0F81601D5
:109D480061F3934360F30A03032908BF43F0005308
:109D58001360002070BD70B501F11E04640186B067
:109D680003590A46002583B100EB4111013BB1F8C4
:109D7800B6135B18B3FBF1F39BB2B3F5807F05D93B
:109D8800090201514FF4807300E0012300EB4211F6
:109D980091F8B24301F56C712CB1C98800EB4214FB
:109DA8005943C4F8C01300EB4211D1F8C01361F352
:109DB800120563F3DC4500EB421393F8B84364F3F0
:109DC8005E7500EB8204D4F890402561C578012DBA
:109DD80008BFD3F8BC33456908BF63612368AE6820
:109DE80016F0010F14BF0026012666F35D7343F0D9
:109DF80000436FF39E732360C378002B31D102F1C7
:109E0800150300EB431393F8124154BB49B393F87D
:109E18001531032B1DD8DFE803F0020F020FC368CA
:109E2800DC6A03310194C1F38F01A4B28C4210D2D1
:109E3800996941F020010BE02B6903310493C1F3C8
:109E48008F019BB28B4204D2C368996941F080614B
:109E5800996100EB4211B1F8C033D1F8BC13FFF798
:109E6800F9FC002006B070BD00EB810186B0D1F886
:109E78009020136843F04043C3F3074111F00C01ED
:109E880001D0082902D1C168C96A01E0416909699C
:109E9800C1F3074109B961F3DF731360002006B00D
:109EA8007047034610B503EB81030124D3F89030C3
:109EB8004FF0004264F3DC421A611A68002042F055
:109EC800004260F39E721A6010BD43694FF0FF3183
:109ED800002210B59A610446596101460AE0D1F89A
:109EE8008C0003686FF3DF7343F080436FF3CF3365
:109EF80003600132237804319A42F0D32046FFF7F9
:109F0800A1FD20461021BDE810407DE5002310B5D5
:109F18001A460446C0F8103303F1C60044F820205E
:109F280003F1D40004EB80004260E01801330F2BEA
:109F380080F89023F0D10823A4F8B6332046FFF721
:109F4800AFFC2046FFF759FD2046FFF709FD012128
:109F58002046FFF791FD2046FFF739FE2046FFF720
:109F680045FD002010BDD0F8CC301868C0F3414042
:109F7800704708B5FFF715FE002008BDD0F810039C
:109F88007047D0F8140370474369986880B27047E7
:109F9800401890F89F037047D43100EB8100406867
:109FA8007047401890F89003704708B5FFF75AFEBD
:109FB80008BD421808B5002382F89F3301F11E023C
:109FC80000EB42125360FFF7C6FE08BD80B584B0AF
:109FD80000AF78604FF00003FB6040F24833C2F2F4
:109FE80000031B681B6878689847FB6843F0080300
:109FF800FB607B68DB68FA685A614FF0010318461A
:10A0080007F11007BD4680BD80B584B000AF786009
:10A018004FF00003FB6040F24833C2F200031B68B4
:10A028009B6878689847FB6843F00053FB607B683F
:10A03800DB68FA685A614FF00103184607F1100708
:10A04800BD4680BD80B485B000AF78607B68D3F82A
:10A0580090301B68BB60BB6843F00043BB60BB68C3
:10A0680043F08043BB607B68D3F89030BA681A60CD
:10A078004FF00003FB60FB6843F40013FB607B6850
:10A08800DB68FA685A614FF00103184607F11407B4
:10A09800BD4680BC704700BF80B588B000AF78600F
:10A0A8004FF00003FB724FF000037B617B6943F0C4
:10A0B80010037B617B68DB687A68D2689269114615
:10A0C8007A696FEA02020A409A617B68DB681B6A58
:10A0D800BB61BB69C3F30303DBB2FB72FB7ADBB280
:10A0E8007A6803F122034FEA8303D3189B681B683D
:10A0F800FB60BB69C3F34343DBB2022B40F09A8099
:10A10800BB69C3F30A139BB2002B40F39480FB7A1C
:10A11800DBB27A684FEA4313D31803F56F731B68F1
:10A12800002B00F08880FB7ADBB27A684FEA431391
:10A13800D31803F56F731A68BB69C3F30A139BB28C
:10A14800786811461A46FFF799FBBB69C3F3030306
:10A15800DBB2BA69C2F30302D2B279684FEA42129B
:10A168008A1802F56F721168BA69C2F30A1292B2BC
:10A178008A1879684FEA4313CB1803F56F731A608E
:10A18800BB69C3F30303DBB2BA69C2F30302D2B2F9
:10A19800796802F11E024FEA42128A1802F104029B
:10A1A8001168BA69C2F30A1292B28A18796803F17F
:10A1B8001E034FEA4313CB1803F104031A60FB7A1A
:10A1C800DBB27A6803F11E034FEA4313D31803F195
:10A1D80004031B68FB61FB7ADBB27A6803F1D403E2
:10A1E8004FEA8303D318FA695A60FB7ADBB27A68BC
:10A1F80003F122034FEA8303D3189B681B693B6171
:10A208003B69C3F3C9439BB2002B14DDFB6843F0E1
:10A218000043FB60FB686FF39E73FB60FB7ADBB265
:10A228007A6803F122034FEA8303D3189B68FA681C
:10A238001A6000E000E000BF7B6943F010037B6117
:10A248007B68DB687A68D268926911467A690A4342
:10A258009A614FF00103184607F12007BD4680BDFB
:10A2680080B59CB000AF786039607A683B6803F1CC
:10A2780022034FEA8303D3189B68FB66FB6E9B6837
:10A28800BB66FB6EDB687B66BA6E7B6E1340BB6693
:10A298007A683B6803F122034FEA8303D3189B686B
:10A2A8001B683B664FF000037B6697F8683003F045
:10A2B8000403DBB2002B22D04FF00003BB65BB6D5B
:10A2C80043F00403BB65BA6DFB6E9A607A683B681D
:10A2D80003F122034FEA8303D3189B68DB687B658D
:10A2E8007B6D43F002037B657A683B6803F12203C8
:10A2F8004FEA8303D3189B687A6DDA6098E097F881
:10A30800683003F02003DBB2002B0AD04FF00003C3
:10A318003B653B6D43F020033B653A6DFB6E9A60ED
:10A3280086E097F8683003F00803DBB2002B3ED0D4
:10A338007A683B6803F122034FEA8303D3189B68CA
:10A34800DB68FB64FB6C43F00203FB647A683B68E0
:10A3580003F122034FEA8303D3189B68FA6CDA608F
:10A368007A683B68D31803F564734FF005021A70D6
:10A378004FF00003BB64BB6C43F01003BB64BA6CC2
:10A38800FB6E9A604FF000037B647B6C43F008031C
:10A398007B647A6CFB6E9A60BB6E6FF30413BB66CA
:10A3A8003B68DBB278681946FFF75EFD40E097F836
:10A3B800693003F00403DBB2002B39D07A683B68BC
:10A3C80003F122034FEA8303D3189B68DB683B64DD
:10A3D8003B6C43F002033B647A683B6803F1220359
:10A3E8004FEA8303D3189B683A6CDA603B68DBB2A8
:10A3F80078681946FFF738FD4FF00003FB63FB6BE5
:10A4080043F01003FB63FA6BFB6E9A607A683B6853
:10A41800D31803F564734FF008021A704FF0000365
:10A42800BB63BB6B43F48063BB63BA6BFB6E9A6020
:10A4380097F8693003F00203DBB2002B28D07A6862
:10A448003B6803F122034FEA8303D3189B68DB6858
:10A458007B637B6B43F002037B637A683B6803F1A1
:10A4680022034FEA8303D3189B687A6BDA603B6850
:10A47800DBB278681946FFF7F7FC4FF000033B633F
:10A488003B6B43F400733B633A6BFB6E9A60DEE10F
:10A4980097F8683003F00103DBB2002B00F0A580C9
:10A4A8007B68DB78012B1DD17A683B6803F12203B6
:10A4B8004FEA8303D3189B681B69FB657A683B687E
:10A4C80003F11E034FEA4313D3181A68FB6DC3F355
:10A4D8001203D21A79683B6803F1D4034FEA830365
:10A4E800CB185A607A683B68D31803F564734FF049
:10A4F80001021A707B683A6802F1C6024FF0000147
:10A5080043F822104FF00003FB62FB6A43F001039B
:10A51800FB62FA6AFB6E9A6097F8623003F00C03EC
:10A52800DBB2002B06D097F8623003F00C03DBB2E5
:10A53800082B3BD17A683B6803F122034FEA830377
:10A54800D3189B68DB68BB62BB6A43F00203BB623B
:10A558007A683B6803F122034FEA8303D3189B68A8
:10A56800BA6ADA603B68DBB278681946FFF77CFCA8
:10A578004FF000037B627B6A43F010037B627A6AC8
:10A58800FB6E9A607A683B684FEA4313D31803F569
:10A5980072731B7883F00103DAB279683B684FEA7B
:10A5A8004313CB1803F572731A7050E197F86230B1
:10A5B80003F00C03DBB20C2B40F048813B6E43F0F8
:10A5C80000533B667A683B6803F122034FEA830332
:10A5D800D3189B683A6E1A607A683B68D31803F5FB
:10A5E80066734FF00102DA7130E197F8683003F0D2
:10A5F8000203DBB2002B00F084807A683B6803F129
:10A6080022034FEA8303D3189B68DB683B623B6AEB
:10A618006FF341033B627A683B6803F122034FEA18
:10A628008303D3189B683A6ADA607A683B68D31860
:10A6380003F564731B78DBB2012B08D17A683B6899
:10A64800D31803F566734FF00102DA714EE07A68A9
:10A658003B68D31803F564731B78DBB2052B08D16C
:10A668007A683B68D31803F566734FF00402DA7111
:10A678003CE07A683B68D31803F564731B78DBB257
:10A68800062B08D07A683B68D31803F564731B78E7
:10A69800DBB2082B10D17B683A6802F1C6024FF092
:10A6A800000143F822107A683B68D31803F56673F3
:10A6B8004FF00302DA7119E097F8623003F00C03E7
:10A6C800DBB20C2B12D17A683B684FEA4313D318DC
:10A6D80003F572731B7883F00103DAB279683B687B
:10A6E8004FEA4313CB1803F572731A704FF0000347
:10A6F800FB61FB6943F00203FB61FA69FB6E9A6038
:10A70800A5E097F8683023F07F03DBB2002B3ED03A
:10A718007A683B6803F122034FEA8303D3189B68E6
:10A72800DB68BB61BB6943F00203BB617A683B68C5
:10A7380003F122034FEA8303D3189B68BA69DA60EE
:10A748007B683A6802F1C60253F8223003F101012E
:10A758007B683A6802F1C60243F822107A683B68BF
:10A76800D31803F564734FF006021A703B68DBB226
:10A7780078681946FFF778FB4FF000037B617B6927
:10A7880043F080037B617A69FB6E9A605FE097F81B
:10A79800683003F01003DBB2002B58D097F8623012
:10A7A80003F00C03DBB20C2B1DD17A683B6803F174
:10A7B80022034FEA8303D3189B68DB683B613B693C
:10A7C80043F002033B617A683B6803F122034FEAD6
:10A7D8008303D3189B683A69DA603B68DBB2786810
:10A7E8001946FFF741FB7A683B68D31803F5647391
:10A7F8004FF003021A704FF00003FB60FB6843F050
:10A808001003FB60FA68FB6E9A6097F8623003F0F9
:10A818000C03DBB2002B06D097F8623003F00C0370
:10A82800DBB2082B13D13B6E43F000433B663B6E13
:10A838006FF39E733B667A683B6803F122034FEA25
:10A848008303D3189B683A6E1A6000E000BF4FF08C
:10A858000103184607F17007BD4680BD80B59AB060
:10A8680000AF786039607A683B6803F122034FEAE9
:10A878008303D3189B687B667B6E9B683B667B6E05
:10A88800DB68FB653A6EFB6D13403B667A683B6894
:10A8980003F122034FEA8303D3189B681B68BB6547
:10A8A80097F8603003F00403DBB2002B22D04FF09E
:10A8B80000037B657B6D43F004037B657A6D7B6EDB
:10A8C8009A607A683B6803F122034FEA8303D3183E
:10A8D8009B68DB683B653B6D43F002033B657A6828
:10A8E8003B6803F122034FEA8303D3189B683A6D50
:10A8F800DA6080E297F8603003F02003DBB2002BC7
:10A908000AD04FF00003FB64FB6C43F02003FB64A8
:10A91800FA6C7B6E9A606EE297F8613003F002037E
:10A92800DBB2002B28D07A683B6803F122034FEA98
:10A938008303D3189B68DB68BB64BB6C43F00203DA
:10A94800BB647A683B6803F122034FEA8303D31898
:10A958009B68BA6CDA603B68DBB278681946FFF727
:10A9680083FA4FF000037B647B6C43F400737B64D1
:10A978007A6C7B6E9A603EE297F8603003F00103D0
:10A98800DBB2002B38D07B683A6802F1C6024FF080
:10A99800000143F822107A683B6803F122034FEA6A
:10A9A8008303D3189B68DB683B643B6C43F002036A
:10A9B8003B647A683B6803F122034FEA8303D318A8
:10A9C8009B683A6CDA603B68DBB278681946FFF737
:10A9D8004BFA4FF00003FB63FB6B43F00103FB638F
:10A9E800FA6B7B6E9A607A683B68D31803F56473D8
:10A9F8004FF001021A70FEE197F8603003F0080387
:10AA0800DBB2002B30D04FF00003BB63BB6B43F0CD
:10AA18000803BB63BA6B7B6E9A607A683B6803F184
:10AA280022034FEA8303D3189B68DB687B637B6B45
:10AA380043F002037B637A683B6803F122034FEA21
:10AA48008303D3189B687A6BDA603B68DBB278685B
:10AA58001946FFF709FA7A683B68D31803F5647357
:10AA68004FF005021A70C6E197F8603003F0100342
:10AA7800DBB2002B38D07B683A6802F1C6024FF08F
:10AA8800000143F822107A683B6803F122034FEA79
:10AA98008303D3189B68DB683B633B6B43F002037B
:10AAA8003B637A683B6803F122034FEA8303D318B8
:10AAB8009B683A6BDA603B68DBB278681946FFF747
:10AAC800D3F94FF00003FB62FB6A43F01003FB620B
:10AAD800FA6A7B6E9A607A683B68D31803F56473E8
:10AAE8004FF003021A7086E197F8603023F07F0375
:10AAF800DBB2002B3ED07A683B6803F122034FEAB1
:10AB08008303D3189B68DB68BB62BB6A43F002030C
:10AB1800BB627A683B6803F122034FEA8303D318C8
:10AB28009B68BA6ADA603B68DBB278681946FFF757
:10AB38009BF97B683A6802F1C60253F8223003F1A8
:10AB480001017B683A6802F1C60243F822107A686C
:10AB58003B68D31803F564734FF006021A704FF080
:10AB680000037B627B6A43F080037B627A6A7B6EB8
:10AB78009A6040E197F8603003F04003DBB2002BA5
:10AB880038D07B683A6802F1C6024FF0000143F8FA
:10AB980022107A683B6803F122034FEA8303D31833
:10ABA8009B68DB683B623B6A43F002033B627A685E
:10ABB8003B6803F122034FEA8303D3189B683A6A80
:10ABC800DA603B68DBB278681946FFF74DF94FF059
:10ABD8000003FB61FB6943F04003FB61FA697B6E8C
:10ABE8009A607A683B68D31803F564734FF00402DF
:10ABF8001A7000E197F8613003F00403DBB2002B10
:10AC08003AD07A683B6803F122034FEA8303D318EA
:10AC18009B68DB68BB61BB6943F00203BB617A6870
:10AC28003B6803F122034FEA8303D3189B68BA6990
:10AC3800DA603B68DBB278681946FFF715F94FF020
:10AC480000037B617B6943F010037B617A697B6E4B
:10AC58009A607A683B68D31803F564734FF008026A
:10AC68001A704FF000033B613B6943F480633B611A
:10AC78003A697B6E9A60BEE097F8603003F0020391
:10AC8800DBB2002B00F0B7807A683B6803F122033F
:10AC98004FEA8303D3189B68DB68FB60FB686FF39C
:10ACA8004103FB607A683B6803F122034FEA8303A0
:10ACB800D3189B68FA68DA607A683B68D31803F59A
:10ACC80064731B78DBB2012B22D17A683B68D318F6
:10ACD80003F566734FF00102DA7197F85A3003F002
:10ACE8000C03DBB2082B7CD17A683B684FEA43132C
:10ACF800D31803F572735B7883F00103DAB27968CD
:10AD08003B684FEA4313CB1803F572735A7068E037
:10AD18007A683B68D31803F564731B78DBB2032B9E
:10AD280008D17A683B68D31803F566734FF00202BE
:10AD3800DA7156E07A683B68D31803F564731B78B8
:10AD4800DBB2042B1AD17A683B6803F115034FEA8A
:10AD58004313D31803F588731B79012B05D13B687E
:10AD6800DBB278681946FFF79CF87A683B68D31815
:10AD780003F566734FF00202DA7132E07A683B68D5
:10AD8800D31803F564731B78DBB2052B08D17A68F6
:10AD98003B68D31803F566734FF00402DA7120E0BC
:10ADA8007A683B68D31803F564731B78DBB2062B0B
:10ADB80017D17B683A6802F1C60253F82230032B98
:10ADC8000FD17A683B68D31803F566734FF0030216
:10ADD800DA717B683A6802F1C6024FF0000143F865
:10ADE80022104FF00003BB60BB6843F00203BB6056
:10ADF800BA687B6E9A604FF00103184607F168073E
:10AE0800BD4680BD80B588B000AF78604FF00003C4
:10AE1800FB614FF00003FB604FF000033B614FF014
:10AE28000003BB614FF000037B617B68D3F8CC3033
:10AE38001B68BB617B68D3F8CC301B687B617B697E
:10AE48006FF382037B617B696FF341037B617B69ED
:10AE58006FF3C3037B617B696FF345137B613B7EB3
:10AE680003F00203DBB2002B0FD07B6943F002032F
:10AE78007B6140F24833C2F200031B685B68786864
:10AE88009847FB6943F00103FB613B7E03F008032D
:10AE9800DBB2002B75D07B6943F008037B613B7EF6
:10AEA80003F00403DBB2002B63D0BB7E03F0060380
:10AEB800DBB2042B05D0BB7E03F00603DBB2022B0A
:10AEC80035D17B685B691B683B61BB7E03F0060379
:10AED800DBB2042B17D17B685B6941F270725A6050
:10AEE8003B7C03F00303DBB2022B24D07B681B7A84
:10AEF800022B04D178684FF00201FEF717FE78683C
:10AF0800FEF74FFE17E07B685B694BF680325A60AC
:10AF18003B7C03F00303DBB2012B0CD078684FF0C5
:10AF28000101FEF703FE7868FEF73BFE03E0786850
:10AF3800FEF737FE00E000BF40F24833C2F20003DC
:10AF48001B68DB68786898474FF00003FB60FB6874
:10AF580043F00053FB607B68DB687A68D2689269CB
:10AF68001146FA686FEA02021140FA680A439A61C8
:10AF780007E040F24833C2F200031B681B69786897
:10AF880098473B7E03F02003DBB2002B07D07B6998
:10AF980043F020037B61FB6943F00103FB617B689D
:10AFA800D3F8CC307A691A60FB69184607F1200794
:10AFB800BD4680BD80B586B000AF78607B685B69B0
:10AFC8001B69BB603B7BC3F3C303DBB27A6803F145
:10AFD8001E034FEA4313D3181B6803F103034FEA18
:10AFE8009303FB82A3E03B894FEA8303BB82BA8ABF
:10AFF8003B7BC3F3C303DBB2796803F11E034FEA5B
:10B008004313CB181B689A421DD93B7BC3F3C30378
:10B01800DBB27A6803F11E034FEA4313D3181B68A7
:10B02800BB824FF000033B613B6943F080633B61A7
:10B038007B68DB687A68D268926911463A696FEA78
:10B0480002020A409A613B7BC3F3C303DBB27A680E
:10B0580003F11E034FEA4313D3181B6803F10303DC
:10B068004FEA9303FB823B7BC3F3C303DBB27A68EB
:10B078004FEA4313D31803F56F7319683B7BC3F387
:10B08800C303DBB21A46BB8A7868FEF7E3FB3B7B57
:10B09800C3F3C303DBB23A7BC2F3C302D2B279680B
:10B0A8004FEA42128A1802F56F721168BA8A8A1832
:10B0B80079684FEA4313CB1803F56F731A603B7B2B
:10B0C800C3F3C303DBB23A7BC2F3C302D2B27968DB
:10B0D80002F11E024FEA42128A181168BA8A8A1AC5
:10B0E800796803F11E034FEA4313CB181A603B7BC0
:10B0F800C3F3C303DBB23A7BC2F3C302D2B27968AB
:10B1080002F11E024FEA42128A1802F10402116883
:10B11800BA8A8A18796803F11E034FEA4313CB18D9
:10B1280003F104031A607B685B691B69BB603B8998
:10B13800FA8A9A420DD23B7BC3F3C303DBB27A6827
:10B1480003F11E034FEA4313D3181B68002B7FF447
:10B158004AAF4FF00103184607F11807BD4680BDF6
:10B1680080B588B000AF78607B68DB68DB6AFB601D
:10B178003B7CC3F3C303DBB27A6803F11E034FEAD7
:10B188004313D3181B6803F103034FEA9303FB83AC
:10B19800A3E0BB894FEA8303BB83BA8B3B7CC3F331
:10B1A800C303DBB2796803F11E034FEA4313CB18DC
:10B1B8001B689A421DD93B7CC3F3C303DBB27A6890
:10B1C80003F11E034FEA4313D3181B68BB834FF0E8
:10B1D8000003BB61BB6943F02003BB617B68DB688C
:10B1E8007A68D26892691146BA696FEA02020A401F
:10B1F8009A613B7CC3F3C303DBB27A6803F11E0395
:10B208004FEA4313D3181B6803F103034FEA930370
:10B21800FB833B7CC3F3C303DBB27A684FEA431377
:10B22800D31803F56F7319683B7CC3F3C303DBB210
:10B238001A46BB8B7868FEF70DFB3B7CC3F3C30350
:10B24800DBB23A7CC2F3C302D2B279684FEA421247
:10B258008A1802F56F721168BA8B8A1879684FEAF2
:10B268004313CB1803F56F731A603B7CC3F3C30316
:10B27800DBB23A7CC2F3C302D2B2796802F11E0291
:10B288004FEA42128A181168BA8B8A1A796803F150
:10B298001E034FEA4313CB181A603B7CC3F3C30366
:10B2A800DBB23A7CC2F3C302D2B2796802F11E0261
:10B2B8004FEA42128A1802F104021168BA8B8A18FE
:10B2C800796803F11E034FEA4313CB1803F1040313
:10B2D8001A607B68DB68DB6AFB60BB89FA8B9A4281
:10B2E8000DD23B7CC3F3C303DBB27A6803F11E03C0
:10B2F8004FEA4313D3181B68002B7FF44AAF4FF073
:10B308000103184607F12007BD4680BD80B586B009
:10B3180000AF78604FF000037B614FF000033B61A2
:10B328007868FEF73BFC0346FB604FF000037B6147
:10B3380034E0BB891A467B6942FA03F303F0010340
:10B34800DBB2002B26D07A687B6903F122034FEA2F
:10B358008303D3189B681B68BB607B7A23F07F0349
:10B36800DBB2002B0BD04AF26923C0F600037868E1
:10B378007969984703463A6913433B610AE04AF6FC
:10B388006503C0F6000378687969984703463A6907
:10B3980013433B617B6903F101037B617B681B7885
:10B3A8001A467B699A42C4D83B69184607F11807C0
:10B3B800BD4680BD80B584B000AF78604FF0000313
:10B3C800FB604FF00003BB607868FEF777FB03462D
:10B3D800002B00F08B807868FEF775FB0346BB6096
:10B3E800BB68002B02D14FF0000380E03B7A03F0EA
:10B3F8000803DBB2002B09D049F6D573C0F6000369
:10B40800786898470346FA681343FB603B7A03F071
:10B418001003DBB2002B09D04AF2A103C0F60003E7
:10B42800786898470346FA681343FB603B7A03F051
:10B438002003DBB2002B09D04BF26913C0F60003DE
:10B44800786898470346FA681343FB60FB7A03F071
:10B458000403DBB2002B09D04AF6BD73C0F6000323
:10B46800786898470346FA681343FB60FB7A03F051
:10B478000203DBB2002B09D04BF21533C0F60003F0
:10B48800786898470346FA681343FB60FB7A03F031
:10B498000103DBB2002B09D04AF60D63C0F60003A6
:10B4A800786898470346FA681343FB60FB7A03F011
:10B4B8002003DBB2002B09D04AF21103C0F60003C7
:10B4C800786898470346FA681343FB60BB7A03F031
:10B4D8002003DBB2002B09D04AF24D03C0F600036B
:10B4E800786898470346FA681343FB60FB68184678
:10B4F80007F11007BD4680BD0123C0F810330020B6
:10B5080070470123C0F81433002070470023C0F8A7
:10B518001433184670470020704738B50446002198
:10B52800FDF79DFEE36800254FF0FF329D61204640
:10B538005A61FEF762FAC4F81053284638BD70B550
:10B548000123002540220C46CB700B778A7181F8C5
:10B55800213006460D704D708D7081F820500979A4
:10B5680000F02BFB6179304600F027FB284670BDC0
:10B578002DE9F041069F1646984604460D46FDF70C
:10B58800FAFD0020FDF77AFE31462046FFF7D7FF87
:10B598002946C6F87C80C6F880702046FEF7B6FCBF
:10B5A800D6F880301B6898472046BDE8F041FDF783
:10B5B80043BE0B1FDBB2012B10B5044606D8D0F8EA
:10B5C80080305B6C98470B23237010BD062905D18A
:10B5D8000B230370D0F880301B68984710BD0023F8
:10B5E80070B58B740B7F013B05460C460A2B00F2A5
:10B5F800C980DFE813F00B00120039004000580042
:10B608006500790080009900A900B90001F11401D2
:10B61800627900F03BFD022343E04979FEF7B8FC6C
:10B62800012819D1237D618B584A03F0800339B171
:10B6380041F2883111800BB1032307E0052305E0AF
:10B64800322111800BB1092300E007232377284614
:10B65800FEF79AFC208295E0032840F093800B23A4
:10B6680023770523A3748DE00B798A89896800F014
:10B6780044FD042315E00979FEF78AFC012802D16C
:10B688000923237703E0042823D0032808D0284679
:10B69800FEF77AFC238AC01A3C4B1B88984271D962
:10B6A8000B2323776EE04B7900EB4313012283F8D9
:10B6B800C9234B798A89896800F0FDFC0623F0E7E5
:10B6C8004979FEF765FC012801D10723E9E7042839
:10B6D80003D1637823700C23E3E7022801D1052303
:10B6E800DFE703284ED1DBE70B7900210A4600F09B
:10B6F80004FD0823D5E70979FEF74AFC0128064628
:10B7080027D00328CCD02846FEF73EFC238AC01A4F
:10B718001E4B1B889842C3D8042E33D163782370FC
:10B728000C232377032070BD4B7900EB431393F868
:10B73800C92382F0010283F8C9234B7900210A4604
:10B7480000F0B9FC0A23ACE74979FEF721FC01288F
:10B7580003D1637823700D23A3E7022801D10923BD
:10B768009FE7032810D19BE78B7B0133DBB2022BC9
:10B778008B7301D8012394E708238B744B7802203C
:10B788000B7070BD002070BD002070BD580E0020E9
:10B7980070B594B0022305460C468DF84F30FEF77D
:10B7A800EDFB18B12846FEF7ECFB28B923781BB14E
:10B7B800032B01D00323237023780B2B00F29181F4
:10B7C800DFE813F00C001F0026006D018F01580000
:10B7D80040014C01590131018F015E012846FEF7F5
:10B7E800CDFB002800F07D8101232370C820FDF7E0
:10B7F80043FD2846FEF7BDFBD4F88030DB68984748
:10B808006FE1D5F81433012B40F06B81022367E117
:10B81800D4F880309B6898470021284600F0B4F996
:10B8280080216071284600F0AFF920712846FEF7A4
:10B838009AFB0523C0B22370D4F8803084F8210025
:10B848009B699847A079217994F8202094F82130B1
:10B85800019000262846009600F048F9A079617901
:10B86800019094F8202094F821300096284600F0A2
:10B878003DF936E1A378092B00F23381DFE813F0B4
:10B888000A002800380060006B007F009800B100B3
:10B89800C9002B0128462146082200F01DFD064656
:10B8A800002840F01E8194F829306179A3710122A3
:10B8B800A2700090019332463346284600F043F9BF
:10B8C800A37921790193009628463246334634E01D
:10B8D80028462146122200F0FFFC002840F0018192
:10B8E800D4F8803004F12200DB699847022330E065
:10B8F80028462146012200F045FD0646002840F072
:10B90800F0800220FDF7B8FC012384F82030D4F839
:10B9180080301B6A98470323A370217994F820206C
:10B92800009633462846019600F00DF9617994F89F
:10B938002020009601962846334600F004F9D0E00E
:10B9480028462146092200F019FE002840F0C98047
:10B958000423A370C5E0E28E2846214600F00EFEBF
:10B96800002840F0BE80D4F8803004F134005B6ACF
:10B9780004F13E0104F1500298470523E9E794F8E1
:10B98800302072B1FF2300932846214603AB00F014
:10B998007BFC002840F0A580D4F8803003A89B6A7F
:10B9A80003E0D4F8803050489B6A98470623D0E7D4
:10B9B80094F8312072B1FF2300932846214603AB47
:10B9C80000F062FC002840F08C80D4F8803003A896
:10B9D800DB6A03E0D4F880304348DB6A98470723E2
:10B9E800B7E794F832206AB1FF230093284621462E
:10B9F80003AB00F049FC002873D1D4F8803003A8C9
:10BA08001B6B03E0D4F8803037481B6B984708233A
:10BA18009FE794F839202846214600F0C0FC00280A
:10BA28005FD1092395E7D4F880309B6B98470128AC
:10BA380057D1E36F28461B6821469847002850D104
:10BA480006234DE0E36F28469B68214698478DF80A
:10BA58004F009DF84F3043B9072341E0E36F284674
:10BA6800DB68214698478DF84F009DF84F10204617
:10BA7800FFF79FFD35E028462146FFF7B0FD30E08F
:10BA880021462846FFF75BFDD4F880305B6898476D
:10BA9800E36F04F120015B682846984721E0D4F859
:10BAA80080301B69984721462846FFF748FDD4F89F
:10BAB80080305B689847E36F04F120015B68284693
:10BAC8009847284600F085F800232370284601216E
:10BAD800FEF71CFA05E0D4F880305B6B9847092321
:10BAE800237014B070BD00BFA1A60508F8B501F514
:10BAF800327430F8146001F1150400EB441406F0B8
:10BB08007F0784F810219DF8182084F8117184F8B3
:10BB18001521BDF81C2084F81331A4F81621C6F3AA
:10BB2800C01600EB411204F5887584F812610024F0
:10BB380082F8C84382F8C9430BB901232B71FEF779
:10BB480091F80020F8BD70B5BDF814401AB100EBAB
:10BB5800411585F8B02301F1150200EB4215B5F83F
:10BB68001661A64205F5887501D004B1EC8000EB9A
:10BB7800421292F813419C4202D00BB182F8133161
:10BB8800FEF770F8002070BD10B502460023B2F928
:10BB98009045002C08DB03F532726FEA41416FEAE9
:10BBA800514120F8121006E00133DBB20232082BB3
:10BBB800EDD14FF6FF73D8B210BD072907D801F5AC
:10BBC800327130F8113023F4004320F8113000208E
:10BBD80070470023A0F89435A0F89635A0F898355A
:10BBE800A0F89A35A0F89C35A0F89E3518467047FD
:10BBF800F8B5314D95F8423006460F46052B58D812
:10BC0800DFE803F00357571309272B6D1B68984784
:10BC1800042385F842303046FDF75DFF012848D1FE
:10BC2800254B032283F8422043E095F8462095F8F7
:10BC38004030214900F0A3FA204B01221A70304607
:10BC4800052385F84230FEF79FF980B2A5F84C002D
:10BC58002FE0FEF799F9B5F84C30174C9BB2C01A93
:10BC6800B5F84A30984221D294F840103046FEF791
:10BC78008FF901280AD1114B1A78012A19D100220B
:10BC88001A70236D20465B68984712E094F84010BC
:10BC98003046FEF77DF904280BD194F8482094F833
:10BCA80040303046394600F095FB10B9032384F83C
:10BCB80042300020F8BD00BF447F00205A0E00200B
:10BCC800384B93F8453073B50446042B66D8DFE843
:10BCD80003F003320340530000F5887300930923EF
:10BCE800019301224FF4045300F0B4FA002855D10F
:10BCF8002D4B94F8102194F813111A7094F811210F
:10BD08005A7094F8122102EB01225A8094F81421F7
:10BD180094F818111A7194F815215A7194F816218B
:10BD28009A7194F8172102EB01221A811D4B012008
:10BD380083F8450035E000F5887300931A4B1B899A
:10BD4800012201934FF4085300F084FA30BB032218
:10BD58000EE0212300220B750A234B75CA820A8341
:10BD68004A83134600F06CF908B1032816D104225F
:10BD78000C4B83F8452011E0212300220B75012587
:10BD88000B234B75CD820A834A831346164600F06F
:10BD980057F928B9034B83F8456002E0012000E019
:10BDA80028467CBD447F0020987F002038B5114D7F
:10BDB80095F84010044649B1FEF756F895F840103A
:10BDC8002046FFF7FAFE002385F84030094D95F824
:10BDD800411051B12046FEF747F895F8411020462A
:10BDE800FFF7EBFE002385F84130034B00221A7061
:10BDF80038BD00BF447F00205A0E00202DE9F347CC
:10BE0800344B062283F8422091F84420012A074641
:10BE18000C4658D191F84520012A04BF2E4A1A65CC
:10BE2800002283F8422083F8452091F8522083F8B5
:10BE38004820B1F85420A3F8462091F85620092A42
:10BE4800A3F84A2003D8234B0A22A3F84A2094F8DF
:10BE580042A0204DBAF1020F28BF4FF0020A264631
:10BE68004FF000084FF0030927E096F852100B0630
:10BE780008D5384685F84410FFF786FE014685F850
:10BE8800400009E085F8431096F852103846FFF74D
:10BE98007BFE014685F84100B5F8460094F820205D
:10BEA800019094F82130CDF800903846FFF71EFE37
:10BEB80008F101085FFA88F80836D045D5D1074B54
:10BEC8000020187004E0D1F880301B6C98470120DE
:10BED800BDE8FC87447F0020700300205A0E002034
:10BEE80030B543EA02229DF80C40CA82212500237E
:10BEF800049A0D750B83092523464D754C83BDE8BF
:10BF0800304000F09DB800BF70474A4A00232DE931
:10BF1800F047137053709370D37005461A46E918AA
:10BF2800013389780139C9B2022998BF0122062B49
:10BF3800F5D1012A7CD03F4991F802C00A784B78A4
:10BF48002846022601F10A098778BFB18C18013208
:10BF58002771D2B2002406E0013409EB040A1AF86A
:10BF680001ACBA4503D05FFA84F8E045F4D3E04564
:10BF780004D1CC18877801332774DBB20136F6B2C6
:10BF88000130082EE0D12B4C012B2270637041D177
:10BF9800207CE070FDF757FA2B78102B1BD0224637
:10BFA8000AD8022B1BD003D89BB1012B1DD112E05C
:10BFB800042B16D0052B0AE0402B12D004D8142BE2
:10BFC80011D0202B11D10AE0412B0CD0502B0CD1D1
:10BFD80009E0A37509E0174B02229A7505E00123D1
:10BFE80002E0032300E004239375124A937DD1787D
:10BFF800114A012B05D803EB4103D05CFDF718FA71
:10C008000AE0032000FB013102EB8102D2F8C030C4
:10C01800984701E00023E370064A137802F10A0109
:10C02800937000230432985C58540133062BFAD1DC
:10C03800BDE8F0875B0E0020EC9C0408FDF7F6B91C
:10C04800C878012810B504D002284FF0010319D18F
:10C0580008E00C788B814C7008240C708A60087793
:10C06800022308E00A7F0D2A03D10020CB7008774D
:10C0780010BD0B2A01D1CB7010BD0C2A04D1CB7096
:10C08800032010BD184610BD184610BD00EB421322
:10C0980010B5002483F8B24300EB42130324C3F81D
:10C0A800BC130821C3F8C01383F8B8431146FDF741
:10C0B80080FFC0B210BD38B500EB4314002584F8EA
:10C0C800B2535C010519C5F8BC1300EB4311C1F864
:10C0D800C02312B9012285F8C923041900EB4312C1
:10C0E80094F8C913002914BF0221002182F8B8135B
:10C0F8001946FDF75EFF002038BD38B500EB431444
:10C10800012584F8B2530225C4F8BC1384F8B85347
:10C11800C4F8C0231946FDF74CFF002038BD38B5D8
:10C1280000EB4315002485F8B24300EB4315C5F82E
:10C13800C02395F8C923C5F8BC13A24214BF022234
:10C14800224685F8B8231946FDF733FF204638BD47
:10C1580038B500EB43140125C4F8C02394F8C8236C
:10C16800C4F8BC13002A14BF0222002284F8B25378
:10C1780084F8B8231946FDF71CFF002038BDF8B530
:10C1880004461F460E46154602201A460E49FDF77C
:10C1980057F904EB4713012283F8B22393F8C82315
:10C1A800C3F8BC63002A14BF0221002182F00102F7
:10C1B80083F8B813C3F8C05383F8C8232046394618
:10C1C800FDF7F7FE0020F8BDA5A6050838B500EB79
:10C1D8004315002485F8B24300EB4315C5F8C02386
:10C1E80095F8C823C5F8BC13A24214BF0221214602
:10C1F80082F0010285F8B81385F8C8231946FDF7BF
:10C20800D8FE204638BD38B500EB4314012584F824
:10C21800B2532546C4F8BC13C4F8C023002485F8DB
:10C22800B8431946FDF7C5FE204638BD38B500EBC2
:10C238004315002485F8B24300EB4315C5F8BC1339
:10C24800C5F8C02385F8B8431946FDF7B2FE204665
:10C2580038BD00BF10B562F07F020A750622BDF82E
:10C268000C404A75CB8240F2094203F47F43B3F590
:10C27800407F0CBF13460023029A0B8323464C834E
:10C28800BDE81040FFF7DCBE73B5BDF818601D4669
:10C2980042F4407300F588728DE844000022044699
:10C2A800FFF7D8FFB8B994F81131032B13D194F8DC
:10C2B8001031023B9E42A8BF1E46B6B2034606E0B6
:10C2C800E218023392F8122105F8012B9BB2B3420F
:10C2D800F6D300232B707CBD73B500F58873164622
:10C2E8008DE8480000224FF4807304460D46FFF79E
:10C2F800B1FF002845D194F8103185F8223094F820
:10C30800113185F8233094F8132194F8123103EB96
:10C318000223AB8494F8143185F8263094F815314B
:10C3280085F8273094F8163185F8283094F81731B5
:10C33800082E85F8293024D994F8192194F8183151
:10C3480003EB02236B8594F81B2194F81A3103EB55
:10C358000223AB8594F81D2194F81C3103EB0223CA
:10C36800EB8594F81E3185F8303094F81F3185F844
:10C37800313094F8203185F8323094F8213185F83D
:10C3880033307CBD10B500230524CA821A460B75CC
:10C398004C750B834B83BDE81040FFF751BE10B5B9
:10C3A80000230924CA821A460B754C750B834B83EC
:10C3B800BDE81040FFF744BE10B50A8301240022EF
:10C3C8000C75CB820B2413464C754A83BDE810408C
:10C3D800FFF736BE30B54FEA431302240C75C31875
:10C3E80001244C75002412F0800F0A83CC824C8300
:10C3F80014BF83F8C84383F8C9430022254613466F
:10C40800BDE83040FFF71CBE2DE9F04F93461A787F
:10C4180002705A7889B042709A780691D97802EBFE
:10C42800012242801A790271597941719979817191
:10C43800D979C171197A0172BDF84810092940F2F9
:10C448009480022A00F293804B4A092192F800C096
:10C45800548881E01A789B1889185A78042A89B276
:10C468007AD19E7893F803A0069F09254FFA86F89B
:10C47800BAF1020F05FB08726ED81D781F79009576
:10C488005D7901959D790295DD7903951D7A022FD5
:10C49800049504D9384B83F800C05C8067E04FEA04
:10C4A80048050595CDF81C800025814650E0187890
:10C4B8001B1809185878052889B249D10798844566
:10C4C80011D000989670107004205070019882F86E
:10C4D80003A050710298177190710398D071049855
:10C4E800B446107216E0187993F8058000EB08201E
:10C4F800844230DC009896701070042050700198C7
:10C5080082F803A050710298177190710398D07146
:10C5180004981072059893F8008040FA85F40BEBA4
:10C52800C4000BF834805C7844709C788470DC78A4
:10C53800C47093F805801C7904EB082484809C79E6
:10C5480084715C791879013500EB0424A4B2EDB24A
:10C5580068B2B842ABDB484642888A423FF67AAFB7
:10C56800054B00205880187002E0002000E00320EE
:10C5780009B0BDE8F08F00BF720E0020F7B54FF488
:10C58800007300F5887701921546002206460C468E
:10C598000097FFF75FFE034633B113E0F11891F8F7
:10C5A80010119954013300E0074A99B2A942F5D312
:10C5B80004F1340004F13E0104F150023B460095B9
:10C5C800FFF722FFFEBD00BFAA7F002003780A887C
:10C5D800D3180B800378C018704700BF036823F096
:10C5E800010303600023036043608360C360036149
:10C5F800212343612C4B98421CD02C4B984220D0CD
:10C608002B4B984225D02B4B98422AD02A4B984244
:10C618002FD02A4B984233D0294B984237D0294BF8
:10C62800984204D14FF03D5243F8AC2C7047264B4A
:10C63800984203D13D2243F8082C7047234B984277
:10C6480004D14FF4746243F8202C7047204B984271
:10C6580004D14FF4741243F8382C70471D4B98429C
:10C6680004D14FF0746243F8502C70471A4B98422B
:10C6780003D11A4A43F8642C7047194B984203D1E6
:10C68800184A43F87C2C7047174B984203D1174A35
:10C6980043F8942C7047164B984204BF4FF03D5214
:10C6A80043F8AC2C704700BF10600240286002407D
:10C6B800406002405860024070600240886002405A
:10C6C800A0600240B8600240106402402864024042
:10C6D8004064024058640240706402403D000020FB
:10C6E80088640240400F0020A064024000003D2002
:10C6F800B86402400268134B10B51340CC680A684E
:10C7080022434C6922438C692243CC6922430C6A38
:10C7180022434C6A22438C6A22434C6B22438C6B23
:10C7280022431343036042690C6BCB6A22F0070271
:10C738002343134343610B6943604B6883608B68F1
:10C74800C36010BD3F801CF000230360436083601A
:10C75800C360036143618361C361036243628362AF
:10C76800C3620363436383637047036811B143F093
:10C77800010301E023F0010303607047036811B16E
:10C7880043F4004301E023F4004303607047036867
:10C7980011B143F0200301E023F020030360704748
:10C7A80041607047406880B27047036812B143F433
:10C7B800002301E023F4002303600161704703684C
:10C7C80011B143F4802301E023F480230360704710
:10C7D8000AB101617047C16070470068C0F3C0408A
:10C7E8007047006800F001007047406900F03800A9
:10C7F80070470A4A0A4B10B50A4CA04288BF134634
:10C808008A004CBF5B681B6821F0F02121F082117F
:10C8180019420CBF0020012010BD00BF0064024077
:10C82800006002400F64024010B5084B084A094CEA
:10C83800A04288BF134611F0005F21F0F02121F0DB
:10C84800821114BFD960996010BD00BF006002401A
:10C85800006402400F6402400B0607D5436912B119
:10C8680043F0800301E023F080034361802909D06D
:10C8780001F01E01036812B119430160704723EAF1
:10C88800010101607047124B124A10B5124CA042C8
:10C898008CBF14461C4621F0F02323F0C3132BB1A0
:10C8A800026802F01E0202EAD12202E0426902F0A6
:10C8B800800288004CBF6368236821F0F02121F0D2
:10C8C8008210184002D0101C18BF012010BD00BFF4
:10C8D80000600240006402400F64024010B5084B3B
:10C8E800084A094CA04288BF134611F0005F21F0A6
:10C8F800F02121F0821114BFD960996010BD00BFEA
:10C9080000600240006402400F640240044B0022B1
:10C918001A605A609A60DA60024A5A61704700BF2A
:10C92800003C0140FFFF7F00837910B5002B29D020
:10C938001A4B01681C68CA4314401C605C6822409A
:10C948005A60027902F1804202F59E32146821434E
:10C95800116002689C68D1430C409C60DC682140EF
:10C96800D9604179102906D1996811439960D9682D
:10C978000A43DA6010BD01F1804303F59E3319685C
:10C988000A4308E00379016803F1804303F59E3305
:10C998001A6822EA01021A6010BD00BF003C01407B
:10C9A80000230C2203600371427183717047024BAC
:10C9B8001A6902431A617047003C0140034B5B69E6
:10C9C80018420CBF00200120704700BF003C014006
:10C9D800014B5861704700BF003C0140054B1A6885
:10C9E8005B69034004D010420CBF0020012070474F
:10C9F80018467047003C0140014B5861704700BF22
:10CA0800003C01404FF0204318B943F2DB021A60A2
:10CA180003E043F2D20243F820204FF02042411CA9
:10CA28006FF0704342F8213002F5827242F82030EC
:10CA3800704770B584684568C368C16A0268254351
:10CA48001D4303691D4343691D4383691D43C3692E
:10CA58001D43036A1D43436A1D43836A1D43036BD9
:10CA68000D431D434FF02043082C43F8225005D1B5
:10CA780053F8224044F0400443F82240436B9E6937
:10CA88001D6835435E6845EA06159E6845EA062531
:10CA9800DE6845EA06451E695B6945EA0655541C89
:10CAA80045EA03654FF02043B1F5804F43F8245021
:10CAB80010D1836B986919680143586841EA0011DD
:10CAC800986841EA002118695B6941EA005141EA26
:10CAD800036101E06FF07041014B43F8221070BD13
:10CAE800040100A0022242604FF480524262416B6E
:10CAF8004FF4005210B5826200230F22FF24036016
:10CB08008360C360036143618361C3610362C3627D
:10CB180003630A604A608C60CA600A614A618B617B
:10CB2800816B0A604A608C60CA600A614A618B61E5
:10CB380010BD4FF0204321B153F8202042F00102EC
:10CB480003E053F82010024A0A4043F820207047B7
:10CB5800FEFF0F0010280CBF064B074B4FF040029A
:10CB68004FF0180119605A604FF0FC329A60DA6091
:10CB7800704700BF600000A0800000A030B5836847
:10CB880044681C43C36844F008041C4303691C43FD
:10CB9800436944EA4324836944EA4334C36999688E
:10CBA8005A68090441EA02211A68DB68114341EA1C
:10CBB8000361036A9A685D68120442EA05221D68E7
:10CBC800DB682A4342EA03620368102B0CBF034B5D
:10CBD800034B1C609960DA6030BD00BF600000A0A4
:10CBE800800000A010230360C269002343608360B3
:10CBF800C360036143618361FC23136053609360E6
:10CC0800D360026A136053609360D360704741B188
:10CC180010280CBF074B084B1A6842F004021A6030
:10CC2800704710280CBF034A034A044B11680B4095
:10CC380013607047600000A0800000A0FBFF0F0099
:10CC480041B110280CBF084B084B1A6842F040024B
:10CC58001A60704710280CBF034A044A044B116835
:10CC68000B401360704700BF600000A0800000A068
:10CC7800BFFF0F00102802D1024B58697047024BC2
:10CC880058697047600000A0800000A0054B18227A
:10CC98001A6000225A604FF0FC329A60DA601A611A
:10CCA800704700BFA00000A00268436842F010026D
:10CCB80042EA4322836842EA4332144B10B51A60B1
:10CCC800C26891685468090441EA04211468D2686A
:10CCD800214341EA02629A60026991685468090432
:10CCE80041EA04211468D268214341EA0262DA6009
:10CCF800426991685068090441EA00211068D268C5
:10CD0800014341EA02621A6110BD00BFA00000A001
:10CD1800C2680023036043608360FC231360536090
:10CD28009360D3600269136053609360D360426973
:10CD3800136053609360D3607047054B18B11A684D
:10CD480042F0040202E01968024A0A401A60704779
:10CD5800A00000A0FBFF0F0062B1102801D10E4B0C
:10CD680003E0B0F5807F03D10C4B5A68114311E002
:10CD78000B4BFAE7102804D1074B5A6822EA010145
:10CD880008E0B0F5807F0CBF044B054B5A686FEA8A
:10CD98000101114059607047600000A0800000A0A8
:10CDA800A00000A0102801D1064B04E0B0F5807F58
:10CDB8000CBF054B054B5B680B420CBF00200120E4
:10CDC800704700BF600000A0800000A0A00000A085
:10CDD800102804D1074B5A6822EA010108E0B0F58F
:10CDE800807F0CBF044B054B5A686FEA0101114064
:10CDF80059607047600000A0800000A0A00000A05B
:10CE0800102801D1084B04E0B0F5807F0CBF074B18
:10CE1800074B5B6813EA010004D013EAD1010CBF89
:10CE280000200120704700BF600000A0800000A023
:10CE3800A00000A0102804D1084B5A6822EAD101AA
:10CE480009E0B0F5807F0CBF054B064B5A684FEAE6
:10CE5800D10122EA01015960704700BF600000A0BB
:10CE6800800000A0A00000A008B52C4B984205D176
:10CE78000120014600F048FC012048E0284B984278
:10CE880005D10220012100F03FFC02203FE0254BA4
:10CE9800984205D10420012100F036FC042036E038
:10CEA800214B984205D10820012100F02DFC0820D3
:10CEB8002DE01E4B984205D11020012100F024FCE2
:10CEC800102024E01A4B984205D12020012100F0BF
:10CED8001BFC20201BE0174B984205D14020012164
:10CEE80000F012FC402012E0134B984205D180203C
:10CEF800012100F009FC802009E0104B98420BD179
:10CF08004FF48070012100F0FFFB4FF48070002186
:10CF1800BDE8084000F0F8BB08BD00BF00000240B3
:10CF28000004024000080240000C024000100240C9
:10CF38000014024000180240001C02400020024079
:10CF48002DE9F0470023D1F800801A464FF0010C74
:10CF580003270CFA02F404EA0805A5422ED1066854
:10CF680017FA03F4E443264006600E79D0F80090DF
:10CF780006FA03FA013E4AEA0909012EC0F80090B0
:10CF880014D8866891F8059026408660866809FA64
:10CF980003F949EA06068660466826EA05054560FB
:10CFA8008D7946689540ADB235434560C5682C40DB
:10CFB800C460CC79C5689C402C43C46001320233FC
:10CFC800102AC6D1BDE8F0874FF6FF73036000232F
:10CFD800037143718371C371704782B04FF480331A
:10CFE8000193019B0B430193019BC361C161019BA9
:10CFF800C361C3690193C369019302B070470369B0
:10D0080019420CBF002001207047006980B27047A8
:10D01800436919420CBF002001207047406980B263
:10D02800704701837047418370470AB10183704795
:10D03800418370474161704743694B404361704782
:10D0480001F00703C908083130B59B0050F821509A
:10D058000F249C4025EA040440F8214050F8214060
:10D0680012FA03F31C4340F8214030BD08B5134BB6
:10D07800984207D14FF40010012100F069FB4FF4EA
:10D08800001014E00E4B984207D14FF480000121A4
:10D0980000F05EFB4FF4800009E00A4B98420BD188
:10D0A8004FF40000012100F053FB4FF40000002171
:10D0B800BDE8084000F04CBB08BD00BF005400406C
:10D0C80000580040005C00407FB5044686886846EA
:10D0D8000D4600F06DFA02992C482B6826F03F06A1
:10D0E8003604B1FBF0F0360C80B20643A6802288E5
:10D0F80022F001021204120C2280254A93420AD817
:10D108005B00B1FBF3F301309BB280B22084032BA8
:10D1180098BF042321E0EE884BF6FF72964205D1B2
:10D1280003225343B1FBF3F39BB206E019225343A6
:10D13800B1FBF3F39BB243F480431A054FF49672A4
:10D1480008BF43F0010350434FF47A7290FBF2F0AA
:10D15800013080B243F400432084A3832388698983
:10D16800AA889BB243F001032380238823F48163B8
:10D1780023F002031B040A431B0C13439BB22380B6
:10D188002A89AB8913439BB223817FBD40420F009C
:10D19800A086010041F288330360002383804BF6A8
:10D1A800FF72038143814FF48043C28083817047BB
:10D1B800038819B19BB243F0010303E023F0010394
:10D1C8001B041B0C03807047038819B19BB243F4FE
:10D1D800807303E023F480731B041B0C03807047E7
:10D1E800038819B19BB243F4007303E023F400737E
:10D1F8001B041B0C0380704712B141F0010101E0D0
:10D2080001F0FE0101827047038819B19BB243F413
:10D21800806303E023F480631B041B0C03807047C6
:10D2280083899BB201F0FE0123F0FE030B43838147
:10D238007047838919B19BB243F0010303E023F0DF
:10D2480001031B041B0C83817047038819B19BB22F
:10D2580043F0400303E023F040031B041B0C03804E
:10D268007047038829B16FEA43436FEA53439BB27F
:10D2780001E05B045B0C03807047038819B99BB21B
:10D2880043F0800303E023F080031B041B0C03809E
:10D298007047B1F5804F838B04D023F480431B047F
:10D2A8001B0C02E09BB243F4804383837047B1F5C3
:10D2B800006F038803D19BB243F4006303E023F4B7
:10D2C80000631B041B0C03807047B1F5005F0388E3
:10D2D80003D19BB243F4005303E023F400531B042F
:10D2E8001B0C03807047038819B19BB243F01003ED
:10D2F80003E023F010031B041B0C0380704701821A
:10D308007047008AC0B27047038819B19BB243F4D2
:10D31800805303E023F480531B041B0C03807047E5
:10D32800B1F5006F038803D19BB243F4006303E0B7
:10D3380023F400631B041B0C03807047038819B196
:10D348009BB243F0200303E023F020031B041B0CD3
:10D3580003807047008BC0F307207047838819B19A
:10D368009BB243F4006303E023F400631B041B0C2B
:10D3780083807047838819B19BB243F4805303E0DC
:10D3880023F480531B041B0C8380704782B0002356
:10D3980001930190019BCB180193019B188880B2DF
:10D3A80002B0704783889BB20AB1194301E023EAAF
:10D3B800010181807047838A008B9BB243EA004059
:10D3C800084020F07F40431A584240EB0300704762
:10D3D800838A008B9BB243EA004020F07F4070476D
:10D3E80082B00023009301930B0F01900093009BE0
:10D3F80021F07F4113B1019B143302E0019B090C1A
:10D4080018330193019B1B6819420CBF00200120AF
:10D4180002B07047C94389B2818270478388808A85
:10D4280080B208409BB206D001F0E06113EA1141D6
:10D438000CBF002001207047C94389B28182704720
:10D448000A4B1A6842F001021A6000229A601968B1
:10D4580021F0847121F480311960054959601968F7
:10D4680021F480211960DA60704700BF003802405B
:10D4780010300024024B00221A701870704700BF49
:10D4880002380240034B1A6822F0F80242EAC0024E
:10D498001A60704700380240014B1860704700BF9F
:10D4A80000004742064B002201281A701A7002D069
:10D4B800042804D101E01870704705221A707047DB
:10D4C80070380240014B1860704700BF800E474219
:10D4D800014341EA821200995B08013B42EA01617B
:10D4E80041EA0341014B5960704700BF00380240D0
:10D4F800014B1860704700BF600047428001034B32
:10D5080040EA0171C3F88410704700BF0038024038
:10D51800014B1860704700BF68004742014B186014
:10D52800704700BF4C004742034B9A6822F0EC62F8
:10D5380002430A439A60704700380240034B9A68D6
:10D5480022F0784202430A439A607047003802404A
:10D55800034B9A6822F0030202439A60704700BFA7
:10D5680000380240024B986800F00C00704700BF7A
:10D5780000380240034B9A6822F0F00202439A6096
:10D58800704700BF00380240034B9A6822F4E0520B
:10D5980002439A60704700BF00380240034B9A6804
:10D5A80022F4604242EAC0029A60704700380240A2
:10D5B8001E4B9A6802F00C02042A10B503D0082A00
:10D5C80003D01B4B18E01B4B16E059685A6811F43E
:10D5D800800F596814BF174B154B02F03F02B3FB7D
:10D5E800F2F3124A5268C2F30142C1F388110132C0
:10D5F8004B435200B3FBF2F30C4903608B680E4AAD
:10D608000468C3F30313D35C34FA03F343608C68F0
:10D61800C4F38224145D33FA04F484608968C1F386
:10D628004231525CD340C36010BD00BF0038024095
:10D638000024F40000127A007803002000F44073FC
:10D64800B3F5407F084B08D1996820F0704221F467
:10D65800F81122F440720A439A601A6F000542EAF0
:10D6680010501867704700BF00380240014B18601F
:10D67800704700BF3C0E4742014B1860704700BF1F
:10D68800400E4742014B1860704700BF5C0147429B
:10D69800044B1A6B09B1104301E022EA0000186339
:10D6A800704700BF00380240044B5A6B09B1104361
:10D6B80001E022EA00005863704700BF00380240CA
:10D6C800044B9A6B09B1104301E022EA0000986309
:10D6D800704700BF00380240044B1A6C09B1104370
:10D6E80001E022EA00001864704700BF00380240D9
:10D6F800044B5A6C09B1104301E022EA0000586457
:10D70800704700BF00380240044B1A6909B1104342
:10D7180001E022EA00001861704700BF00380240AB
:10D72800044B5A6909B1104301E022EA000058612C
:10D73800704700BF00380240044B9A6909B1104392
:10D7480001E022EA00009861704700BF00380240FB
:10D75800044B1A6A09B1104301E022EA000018627A
:10D76800704700BF00380240044B5A6A09B11043A1
:10D7780001E022EA00005862704700BF003802400A
:10D78800044B1A6D09B1104301E022EA0000186544
:10D79800704700BF00380240044B5A6D09B110436E
:10D7A80001E022EA00005865704700BF00380240D7
:10D7B800044B9A6D09B1104301E022EA0000986514
:10D7C800704700BF00380240044B1A6E09B110437D
:10D7D80001E022EA00001866704700BF00380240E6
:10D7E800044B5A6E09B1104301E022EA0000586662
:10D7F800704700BF00380240044B1A7809B1104343
:10D8080001E022EA00001870704700BF0D3802409E
:10D818004309012B074A01D1136803E0022B0CBF0F
:10D82800136F536F00F01F0033FA00F000F001008F
:10D83800704700BF0038024007B50023019331202C
:10D84800FFF7E6FF019B01330193019BB3F5A06F3E
:10D8580001D00028F3D03120FFF7DAFF003018BFDD
:10D8680001200EBD024B5A6F42F080725A67704712
:10D8780000380240034BDB6818420CBF002001202F
:10D88800704700BF00380240014B1870704700BF56
:10D898000E38024008B5154B98420BD101214FF4C0
:10D8A8008050FFF761FF4FF480500021BDE8084029
:10D8B800FFF75ABF0E4B984207D14FF48040012121
:10D8C800FFF746FF4FF4804009E00A4B98420BD11E
:10D8D8004FF400400121FFF73BFF4FF400400021C7
:10D8E800BDE80840FFF734BF08BD00BF0030014065
:10D8F80000380040003C00400B88028810B54C8876
:10D9080023438C882343CC8823430C8923434C89A5
:10D9180023438C892343CC8902F441522343134384
:10D928009BB20380838B23F400631B041B0C83834B
:10D938000B8A038210BD838B23F47B6323F00F03D0
:10D948001B041B0C8383022303848B68F0B5858B2F
:10D95800022BADB238D0294A8E889468002E14BFA5
:10D9680002260126240203D5946824F40004946056
:10D97800D2F88440D2F884705268DFF884C002F08C
:10D988003F02BCFBF2F2C4F388145443C7F302729B
:10D99800B4FBF2F4CA88B2F5007F4FF00A0201D155
:10D9A800240A02E07601B4FBF6F46243B2FBF3F317
:10D9B80005330A229BB2B3FBF2F303F00102120211
:10D9C800C3F34F0392B200E000229C1EA4B2FE2CC7
:10D9D80028BF0022CC8828BF0223134323439BB2CD
:10D9E80003840B884A882B4343F4006313438A88D3
:10D9F80013438A8913439BB28383F0BD00380240E6
:10DA080000127A000023038043808380C38003814F
:10DA180043818381C3810723038270470023022245
:10DA2800038043808380C38082608381704703883A
:10DA380019B19BB243F0400303E023F040031B04F9
:10DA48001B0C03807047838B19B19BB243F480632E
:10DA580003E023F480631B041B0C83837047038853
:10DA680023F400631B041B0C038003889BB20B4345
:10DA780003807047B1F5804F038803D19BB243F40C
:10DA8800804303E023F480431B041B0C038070478E
:10DA98004FF6FF639942038803D09BB243F4807327
:10DAA80003E023F480731B041B0C038070478388F6
:10DAB80019B19BB243F0040303E023F004031B04F1
:10DAC8001B0C83807047838819B19BB243F0100305
:10DAD80003E023F010031B041B0C83807047838B27
:10DAE80023F47B6323F00F031B041B0C83830223A3
:10DAF80003840B88828BB3F5007F10B592B205D0F2
:10DB0800002B0CBF4FF48073002301E04FF48073A7
:10DB18004C8822438C88898942F4006222430A4354
:10DB280092B21343838310BD808980B2704781818C
:10DB38007047038819B19BB243F4005303E023F400
:10DB480000531B041B0C0380704703889BB243F4EB
:10DB5800805303807047012902D0008B80B2704740
:10DB6800808A80B27047008A80B2704783889BB2EF
:10DB78000AB1194301E023EA0101818070470909CC
:10DB880001238B409BB21AB1828892B2134303E0FF
:10DB9800828892B222EA030383807047038919427C
:10DBA8000CBF002001207047C94389B2018170472A
:10DBB80010B584880089012301F00F0280B213FA9E
:10DBC80002F21040A4B205D009098B401C420CBFD8
:10DBD8000020012010BD01F00F0101238B40DB4321
:10DBE8009BB20381704700BF08B501214FF4804004
:10DBF800FFF7BAFD4FF480400021BDE80840FFF769
:10DC0800B3BD014B186070470038014001F00302B2
:10DC180089080A4B023130B5920053F821500F247D
:10DC2800944025EA040443F8214053F8214010FAAF
:10DC380002F2144343F8214030BD00BF00380140D0
:10DC4800014B1860704700BFDC002742014B186089
:10DC5800704700BF00042742024B186AC0F3002037
:10DC6800704700BF0038014030B5048C24F001042F
:10DC78002404240C0484058B048CADB2A4B225F0D2
:10DC8800F305154324F00A0445EA031544F001049A
:10DC9800ADB20C430583048430BD30B5048C24F048
:10DCA80010042404240C0484048B058C24F440748C
:10DCB800ADB22405240D25F0A00544EA022445F060
:10DCC800100544EA033445EA0115A4B2ADB2048351
:10DCD800058430BD08B5474B984205D1012001465F
:10DCE800FFF742FD01203DE0B0F1804F05D1012052
:10DCF8000146FFF72DFD012076E03F4B984205D104
:10DD080002200121FFF724FD02206DE03B4B9842E1
:10DD180005D104200121FFF71BFD042064E0384BE6
:10DD2800984205D108200121FFF712FD08205BE089
:10DD3800344B984205D110200121FFF709FD10202E
:10DD480052E0314B984205D120200121FFF700FD18
:10DD5800202049E02D4B984209D102200121FFF7EC
:10DD680003FD02200021BDE80840FFF7FDBC284B59
:10DD7800984207D14FF480300121FFF7F5FC4FF4AA
:10DD88008030EFE7234B984207D14FF40030012150
:10DD9800FFF7EAFC4FF40030E4E71F4B984207D145
:10DDA8004FF480200121FFF7DFFC4FF48020D9E7F2
:10DDB8001A4B984205D140200121FFF7C9FC4020A9
:10DDC80012E0174B984205D180200121FFF7C0FCD3
:10DDD800802009E0134B98420BD14FF48070012149
:10DDE800FFF7B6FC4FF480700021BDE80840FFF74C
:10DDF800AFBC08BD0000014000040040000800401E
:10DE0800000C0040001000400014004000040140D5
:10DE18000040014000440140004801400018004013
:10DE2800001C0040002000401C4A038890429BB21E
:10DE380012D002F5806290420ED0B0F1804F0BD024
:10DE4800A2F58032904207D002F58062904203D05A
:10DE580002F58062904203D14A8823F0700313438D
:10DE68000F4A904208D002F58062904204D023F411
:10DE780040730A899BB2134303804B68C3620B88C3
:10DE88000385064B984203D003F58063984201D17D
:10DE98008B7A038601238382704700BF000001400C
:10DEA800001000404FF0FF334360002303800381DC
:10DEB800438083727047018582827047038823F00C
:10DEC80070031B041B0C0B430380704741627047AF
:10DED800C1627047406A7047008D80B270470388FE
:10DEE80019B19BB243F0020303E023F002031B04C1
:10DEF8001B0C03807047038819B19BB243F00403DD
:10DF080003E023F004031B041B0C03807047038801
:10DF180019B19BB243F0800303E023F080031B0494
:10DF28001B0C03807047038823F008031B041B0C99
:10DF3800038003889BB20B4303807047038823F454
:10DF480040731B041B0C038003889BB20B430380A4
:10DF58007047038819B19BB243F0010303E023F033
:10DF680001031B041B0C03807047038C23F001037F
:10DF78001B041B0C038470B5038C8488028B0D88EA
:10DF88004E8822F073021204120C2A438D8923F062
:10DF980002031B0435431B0CADB22B430E4DA842A4
:10DFA800A4B203D005F58065A8420ED1CD894E8A6A
:10DFB80023F008032B438D8823F004032B430D8A99
:10DFC800354324F44074ADB22C43848002838A68BC
:10DFD8004263038470BD00BF00000140038C23F03E
:10DFE80010031B041B0C0384038C828830B5048B3C
:10DFF8000D8824F4E6442404240C23F0200344EA86
:10E0080005241B048D891B0C43EA05134D8843EA3C
:10E018000513134DA84292B2A4B29BB203D005F5E2
:10E028008065A84215D1CD8923F080039BB243EACD
:10E0380005134FF6BF751D408B8845EA03130D8AFB
:10E0480022F4406242EA85024D8A42EA85029BB286
:10E0580092B282808A6804838263038430BD00BFE1
:10E0680000000140038C23F480731B041B0C038401
:10E07800038C828830B5848B0D8824F073042404C3
:10E08800240C23F400731B042C438D891B0C43EAD6
:10E0980005234D8843EA0523124DA84292B29BB24C
:10E0A80003D005F58065A84215D1CD8923F4006316
:10E0B8009BB243EA05234FF6FF351D408B8845EA9E
:10E0C80003230D8A22F4405242EA05124D8A42EA9D
:10E0D80005129BB292B282808A688483C2630384E9
:10E0E80030BD00BF00000140038C23F480531B04A3
:10E0F8001B0C0384038C30B58488828B0D8822F432
:10E10800E6421204120C23F4005342EA05221B04CF
:10E118008D891B0C43EA05334D8843EA05330B4DC3
:10E12800A842A4B292B29BB203D005F58065A8427A
:10E1380005D10D8A24F4804444EA8514A4B284806D
:10E1480082838A680264038430BD00BF00000140F6
:10E15800002303804380838083608381C38103829B
:10E168004382704730B5058C0124ADB28C4025EA56
:10E17800040400F11803048409B1082907D14908E7
:10E188004FF68F70CC582040C850C8580AE0043960
:10E19800C1F34E0148F6FF70CC582040C850120217
:10E1A800C85892B20243CA5030BD41637047816378
:10E1B8007047C163704701647047038B23F0700395
:10E1C8001B041B0C0B4303837047038B23F4E043AE
:10E1D8001B041B0C43EA01239BB203837047838B08
:10E1E80023F070031B041B0C0B4383837047838B42
:10E1F80023F4E0431B041B0C43EA01239BB28383F3
:10E208007047038B23F008031B041B0C0B43038389
:10E218007047038B23F400631B041B0C43EA0123A0
:10E228009BB203837047838B23F008031B041B0CEA
:10E238000B4383837047838B23F400631B041B0CFD
:10E2480043EA01239BB283837047038B23F00403C3
:10E258001B041B0C0B4303837047038B23F480635D
:10E268001B041B0C43EA01239BB203837047838B77
:10E2780023F004031B041B0C0B4383837047838B1D
:10E2880023F480631B041B0C43EA01239BB28383A2
:10E298007047038B23F080031B041B0C0B43038381
:10E2A8007047038B09025B0441EA53439BB2038323
:10E2B8007047838B23F080031B041B0C0B43838361
:10E2C8007047838B09025B0441EA53439BB2838303
:10E2D8007047038C23F002031B041B0C0B430384BD
:10E2E8007047038C23F008031B041B0C0B430384A7
:10E2F8007047038C23F020031B041B0C43EA011313
:10E308009BB203847047038C23F080031B041B0C0F
:10E3180043EA01139BB203847047038C23F4007310
:10E328001B041B0C43EA01239BB203847047038C34
:10E3380023F400631B041B0C43EA01239BB20384F0
:10E348007047038C23F400531B041B0C43EA01336E
:10E358009BB20384704710B5048C01238B40A4B290
:10E3680024EA03030384038C12FA01F10B439BB2E2
:10E37800038410BD10B5048C04238B40A4B224EA96
:10E3880003030384038C12FA01F10B439BB2038449
:10E3980010BD00230122038043808280C380038153
:10E3A8007047406B7047806B7047C06B7047006C5C
:10E3B8007047038B23F00C031B041B0C0383038B94
:10E3C8009BB20B4303837047038B23F440631B0406
:10E3D8001B0C0383038B9BB243EA01239BB2038389
:10E3E8007047F8B50C464988A288B4F800E023893C
:10E3F800054600290CBF02270027012A14BF012661
:10E408000226BEF1000F10D1FFF72EFC2846E18846
:10E41800FFF7CFFF2846394632462389FFF73DFCF0
:10E42800E1882846BDE8F840CEE7FFF736FC2846E5
:10E43800E188FFF7C9FF2846394632462389FFF7A6
:10E4480013FCE1882846BDE8F840B2E7838B23F047
:10E458000C031B041B0C8383838B9BB20B438383AA
:10E468007047838B23F440631B041B0C8383838BCB
:10E478009BB243EA01239BB283837047F8B50D46EC
:10E488000B88AA88498804463BB92B89FFF7ECFB1F
:10E49800E9882046BDE8F8408BE7042B07D12B8993
:10E4A800FFF7FBFBE9882046BDE8F8408CE7082B1E
:10E4B800B5F808C0078C1DD127F480773F043F0CBE
:10E4C8000784868B038CB6B29BB226F0F30623F43E
:10E4D800206346EA0C1C43EA01211FFA8CFC89B22E
:10E4E8004CEA020241F4807182830184E988BDE824
:10E4F800F840ABE727F480573F043F0C0784868B2E
:10E50800038C26F4407623F4005336055B04360D5D
:10E518005B0C46EA022243EA013342EA0C329BB220
:10E52800E98892B243F4805382830384BDE8F840BB
:10E5380097E74A880B8813438A881343CA8813438A
:10E548000A8913434A8913438A8913439BB2A0F863
:10E55800443070470023038043808380C380038155
:10E56800438183817047B0F8443029B16FEA43434F
:10E578006FEA53439BB201E05B045B0CA0F84430A4
:10E588007047838819B19BB243F0040303E023F07A
:10E5980004031B041B0C83807047838819B19BB24A
:10E5A80043F0010303E023F001031B041B0C8380E9
:10E5B800704783899BB20AB1194301E023EA01013C
:10E5C8008181704781827047038A19420CBF0020FD
:10E5D80001207047C94389B201827047038A828942
:10E5E80011EA030092B203D011420CBF00200120AF
:10E5F8007047C94389B2018270470A43A0F848208E
:10E60800704783899BB20AB1194301E023EA0101EB
:10E6180081817047838819B19BB243F0080303E0F6
:10E6280023F008031B041B0C83807047038923F025
:10E6380007031B041B0C03817047038923F0700335
:10E648001B041B0C0B43038103899BB243F0070394
:10E658000381704738B50D4611460122602D0446E6
:10E6680002D1FFF71AFB01E0FFF7FEFA238923F036
:10E6780070031B041B0C1D43258123899BB243F0A7
:10E688000703238138BD038923F070031B041B0C87
:10E698000B4303817047838823F070031B041B0C12
:10E6A800838083889BB20B4383807047038923F060
:10E6B80007031B041B0C038103899BB20B430381D3
:10E6C8007047038923F080031B041B0C0381038913
:10E6D8009BB20B430381704710B50489E4B20C4325
:10E6E800144344EA0324A4B2048110BD10B50446BF
:10E6F800FFF7F2FF23899BB243F48043238110BDC7
:10E7080010B50446FFF7E8FF238923F077031B04BD
:10E718001B0C43F07703238110BD70B50489068B69
:10E72800058C26F44076ADB226F0030624F00704E3
:10E73800360425F022052404360C1543240C46F42F
:10E74800807645EA0315214346F00106ADB2018102
:10E758000683058470BD838819B19BB243F080039A
:10E7680003E023F080031B041B0C83807047A0F890
:10E778005010704708B5234B984205D1102001214D
:10E78800FEF7F2FF102037E01F4B984207D14FF4F5
:10E7980000300121FEF7DCFF4FF4003009E01B4B8D
:10E7A80098420BD14FF480200121FEF7D1FF4FF49E
:10E7B80080200021BDE80840FEF7CABF144B9842EC
:10E7C80007D14FF400200121FEF7C2FF4FF40020CB
:10E7D800EFE7104B984207D14FF480100121FEF764
:10E7E800B7FF4FF48010E4E70B4B984209D1202083
:10E7F8000121FEF7B9FF20200021BDE80840FEF7FF
:10E80800B3BF08BD0010014000440040004800406C
:10E81800004C00400050004000140140038ACA88A0
:10E828009BB223F4405330B513430D4603828389CA
:10E838000989AA8823F4B0530A43698923F00C0391
:10E848001B040A431B0C92B213438381838AAA894F
:10E858009BB223F44073134385B083820446684611
:10E86800FEF7A6FE1A4B9C4203D003F580639C4238
:10E8780001D1039B00E0029BA28912B2002A4FF04B
:10E8880019012A6801FB03F101DA520000E0920045
:10E898006423B1FBF2F1B1FBF3F21201100903FB9F
:10E8A8001011A08900B2002806DAC9003231B1FB84
:10E8B800F3F303F0070305E009013231B1FBF3F389
:10E8C80003F00F031A4392B2228105B030BD00BF96
:10E8D800001001404FF4165303600C22002383807C
:10E8E800C38003814281838170470B88028A10B5F7
:10E8F8004C8823438C88C988234392B20B4322F463
:10E9080070629BB21343038210BD002303804380CF
:10E918008380C3807047838919B19BB243F4005345
:10E9280003E023F400531B041B0C83817047038B03
:10E9380003F47F430383038B9BB20B43038370472A
:10E94800838929B16FEA43436FEA53439BB201E0DD
:10E958005B045B0C83817047838A19B19BB243F4D3
:10E96800006303E023F400631B041B0C83827047DD
:10E97800C905C90D818070478088C005C00D7047E2
:10E98800038A23F00F031B041B0C0382038A9BB228
:10E998000B4303827047838919B19BB243F002038A
:10E9A80003E023F002031B041B0C83817047838957
:10E9B80023F400631B041B0C838183899BB20B43E4
:10E9C80083817047038A23F020031B041B0C0382F6
:10E9D800038A9BB20B4303827047038A19B19BB227
:10E9E80043F4804303E023F480431B041B0C03829D
:10E9F800704783899BB243F0010383817047838A00
:10EA080019B19BB243F0080303E023F008031B0489
:10EA18001B0C83827047038BDBB20383038B9BB28F
:10EA280043EA012303837047838A19B19BB243F0F9
:10EA3800200303E023F020031B041B0C8382704790
:10EA4800838A19B19BB243F0100303E023F010034B
:10EA58001B041B0C83827047838A23F004031B0466
:10EA68001B0C8382838A9BB20B4383827047838A01
:10EA780019B19BB243F0020303E023F002031B0425
:10EA88001B0C83827047838A9BB20AB1194301E049
:10EA980023EA010181827047C1F3421310B501F0E6
:10EAA8001F01012414FA01F1A34201D10C3004E042
:10EAB800022B01D1103000E0143003680AB1194369
:10EAC80001E023EA0101016010BD038819420CBF6F
:10EAD800002001207047C94389B201807047012294
:10EAE80010B501F01F03C1F342149A40012C01D163
:10EAF800838903E0022C0CBF038A838A9BB21340EC
:10EB0800028892B243B1090A012313FA01F11142B2
:10EB18000CBF0020012010BD184610BD090A0123B2
:10EB28008B40DB439BB20380704700BF81F00041FC
:10EB380002E000BF83F0004330B54FEA41044FEADA
:10EB4800430594EA050F08BF90EA020F1FBF54EA75
:10EB5800000C55EA020C7FEA645C7FEA655C00F011
:10EB6800E2804FEA5454D4EB5555B8BF6D420CDDE2
:10EB78002C4480EA020281EA030382EA000083EA65
:10EB8800010180EA020281EA0303362D88BF30BD05
:10EB980011F0004F4FEA01314FF4801C4CEA11315B
:10EBA80002D0404261EB410113F0004F4FEA0333BA
:10EBB8004CEA133302D0524263EB430394EA050F45
:10EBC80000F0A780A4F10104D5F1200E0DDB02FAB4
:10EBD8000EFC22FA05F2801841F1000103FA0EF248
:10EBE800801843FA05F359410EE0A5F120050EF10E
:10EBF800200E012A03FA0EFC28BF4CF0020C43FA3F
:10EC080005F3C01851EBE37101F0004507D54FF04B
:10EC1800000EDCF1000C7EEB00006EEB0101B1F59B
:10EC2800801F1BD3B1F5001F0CD349085FEA3000E1
:10EC38004FEA3C0C04F101044FEA445212F5800FEC
:10EC480080F09A80BCF1004F08BF5FEA500C50F189
:10EC5800000041EB045141EA050130BD5FEA4C0C6C
:10EC6800404141EB010111F4801FA4F10104E9D1F5
:10EC780091F0000F04BF01460020B1FA81F308BFEC
:10EC88002033A3F10B03B3F120020CDA0C3208DDB8
:10EC980002F1140CC2F10C0201FA0CF021FA02F193
:10ECA8000CE002F11402D8BFC2F1200C01FA02F103
:10ECB80020FA0CFCDCBF41EA0C019040E41AA2BF28
:10ECC80001EB0451294330BD6FEA04041F3C1CDAF0
:10ECD8000C340EDC04F11404C4F1200220FA04F010
:10ECE80001FA02F340EA030021FA04F345EA0301BA
:10ECF80030BDC4F10C04C4F1200220FA02F001FA7C
:10ED080004F340EA0300294630BD21FA04F02946FD
:10ED180030BD94F0000F83F4801306BF81F4801196
:10ED28000134013D4EE77FEA645C18BF7FEA655C09
:10ED380029D094EA050F08BF90EA020F05D054EADB
:10ED4800000C04BF1946104630BD91EA030F1EBFE0
:10ED58000021002030BD5FEA545C05D140004941E4
:10ED680028BF41F0004130BD14F580043CBF01F5D7
:10ED7800801130BD01F0004545F0FE4141F47001BD
:10ED88004FF0000030BD7FEA645C1ABF1946104698
:10ED98007FEA655C1CBF0B46024650EA013406BF99
:10EDA80052EA033591EA030F41F4002130BD00BF58
:10EDB80090F0000F04BF0021704730B54FF4806415
:10EDC80004F132044FF000054FF0000150E700BF96
:10EDD80090F0000F04BF0021704730B54FF48064F5
:10EDE80004F1320410F0004548BF40424FF00001E2
:10EDF8003EE700BF42004FEAE2014FEA31014FEA25
:10EE080002701FBF12F07F4393F07F4F81F0605173
:10EE1800704792F0000F14BF93F07F4F704730B5E2
:10EE28004FF4607401F0004521F0004120E700BF75
:10EE380050EA010208BF704730B54FF000050AE0FC
:10EE480050EA010208BF704730B511F0004502D5FD
:10EE5800404261EB41014FF4806404F132045FEAFF
:10EE6800915C3FF4DCAE4FF003025FEADC0C18BFA4
:10EE780003325FEADC0C18BF033202EBDC02C2F19A
:10EE8800200300FA03FC20FA02F001FA03FE40EA2C
:10EE98000E0021FA02F11444C1E600BF70B54FF02C
:10EEA800FF0C4CF4E06C1CEA11541DBF1CEA13550E
:10EEB80094EA0C0F95EA0C0F00F0DEF82C4481EA76
:10EEC800030621EA4C5123EA4C5350EA013518BF96
:10EED80052EA033541F4801143F4801338D0A0FB83
:10EEE80002CE4FF00005E1FB02E506F00042E0FB30
:10EEF80003E54FF00006E1FB03569CF0000F18BF36
:10EF08004EF0010EA4F1FF04B6F5007F64F54074DD
:10EF180004D25FEA4E0E6D4146EB060642EAC62170
:10EF280041EA55514FEAC52040EA5E504FEACE2EDD
:10EF3800B4F1FD0C88BFBCF5E06F1ED8BEF1004FE0
:10EF480008BF5FEA500E50F1000041EB045170BD5C
:10EF580006F0004646EA010140EA020081EA0301A0
:10EF6800B4EB5C04C2BFD4EB0C0541EA045170BD9C
:10EF780041F480114FF0000E013C00F3AB8014F116
:10EF8800360FDEBF002001F0004170BDC4F100045F
:10EF9800203C35DA0C341BDC04F11404C4F12005E0
:10EFA80000FA05F320FA04F001FA05F240EA02003B
:10EFB80001F0004221F0004110EBD37021FA04F671
:10EFC80042EB06015EEA430E08BF20EAD37070BD2B
:10EFD800C4F10C04C4F1200500FA04F320FA05F08A
:10EFE80001FA04F240EA020001F0004110EBD3708C
:10EFF80041F100015EEA430E08BF20EAD37070BDFC
:10F00800C4F1200500FA05F24EEA020E20FA04F3D4
:10F0180001FA05F243EA020321FA04F001F0004183
:10F0280021FA04F220EA020000EBD3705EEA430EF4
:10F0380008BF20EAD37070BD94F0000F0FD101F023
:10F048000046400041EB010111F4801F08BF013C5C
:10F05800F7D041EA060195F0000F18BF704703F09A
:10F068000046520043EB030313F4801F08BF013D21
:10F07800F7D043EA0603704794EA0C0F0CEA1355DD
:10F0880018BF95EA0C0F0CD050EA410618BF52EA97
:10F098004306D1D181EA030101F000414FF000009D
:10F0A80070BD50EA410606BF1046194652EA4306AB
:10F0B80019D094EA0C0F02D150EA013613D195EA1F
:10F0C8000C0F05D152EA03361CBF104619460AD167
:10F0D80081EA030101F0004141F0FE4141F4700171
:10F0E8004FF0000070BD41F0FE4141F4780170BD61
:10F0F80070B54FF0FF0C4CF4E06C1CEA11541DBFC6
:10F108001CEA135594EA0C0F95EA0C0F00F0A7F8C7
:10F11800A4EB050481EA030E52EA03354FEA0131F4
:10F1280000F088804FEA03334FF0805545EA131307
:10F1380043EA12634FEA022245EA111545EA1065CF
:10F148004FEA00260EF000419D4208BF964244F166
:10F15800FD0404F5407402D25B084FEA3202B61A85
:10F1680065EB03055B084FEA32024FF480104FF459
:10F17800002CB6EB020E75EB030E22BFB61A7546CD
:10F1880040EA0C005B084FEA3202B6EB020E75EB60
:10F19800030E22BFB61A754640EA5C005B084FEAC8
:10F1A8003202B6EB020E75EB030E22BFB61A754695
:10F1B80040EA9C005B084FEA3202B6EB020E75EBA0
:10F1C800030E22BFB61A754640EADC0055EA060E61
:10F1D80018D04FEA051545EA16754FEA06164FEAA4
:10F1E800C30343EA52734FEAC2025FEA1C1CC0D150
:10F1F80011F4801F0BD141EA00014FF000004FF0DD
:10F20800004CB6E711F4801F04BF01430020B4F19D
:10F21800FD0C88BFBCF5E06F3FF6AFAEB5EB030C55
:10F2280004BFB6EB020C5FEA500C50F1000041EB52
:10F23800045170BD0EF0004E4EEA113114EB5C041F
:10F24800C2BFD4EB0C0541EA045170BD41F48011F2
:10F258004FF0000E013C90E645EA060E8DE60CEAFA
:10F26800135594EA0C0F08BF95EA0C0F3FF43BAF17
:10F2780094EA0C0F0AD150EA01347FF434AF95EACE
:10F288000C0F7FF425AF104619462CE795EA0C0FB2
:10F2980006D152EA03353FF4FDAE1046194622E77F
:10F2A80050EA410618BF52EA43067FF4C5AE50EA59
:10F2B80041047FF40DAF52EA43057FF4EBAE12E749
:10F2C8004FF0FF3C06E000BF4FF0010C02E000BF2A
:10F2D8004FF0010C4DF804CD4FEA410C7FEA6C5C0D
:10F2E8004FEA430C18BF7FEA6C5C1BD001B050EAB0
:10F2F800410C0CBF52EA430C91EA030F02BF90EA9B
:10F30800020F0020704710F1000F91EA030F58BF59
:10F31800994208BF90422CBFD8176FEAE37040F0BB
:10F32800010070474FEA410C7FEA6C5C02D150EA59
:10F33800013C07D14FEA430C7FEA6C5CD6D152EA14
:10F34800033CD3D05DF8040B704700BF84461046D9
:10F3580062468C461946634600E000BF01B5FFF7D8
:10F36800B7FF002848BF10F1000F01BD4DF808EDA8
:10F37800FFF7F4FF0CBF012000205DF808FB00BF79
:10F388004DF808EDFFF7EAFF34BF012000205DF8D3
:10F3980008FB00BF4DF808EDFFF7E0FF94BF012020
:10F3A80000205DF808FB00BF4DF808EDFFF7CEFF21
:10F3B80094BF012000205DF808FB00BF4DF808ED60
:10F3C800FFF7C4FF34BF012000205DF808FB00BF31
:10F3D8004FEA410212F5001215D211D56FF4787375
:10F3E800B3EB625212D94FEAC12343F0004343EA18
:10F3F800505311F0004F23FA02F018BF40427047F3
:10F408004FF00000704750EA013005D111F000407C
:10F4180008BF6FF0004070474FF00000704700BF12
:10F428004A0011D212F5001211D20DD56FF478737B
:10F43800B3EB62520ED44FEAC12343F0004343EAD0
:10F44800505323FA02F070474FF00000704750EA1B
:10F45800013002D14FF0FF3070474FF00000704785
:10F468004BB942B9002908BF002802D04FF0FF313C
:10F47800084600F037B882B0EC462DE9005000F09D
:10F488001BF8DDF804E002B00CBC7047F8B5144670
:10F4980006460F461D4600F027F804FB01F300FB63
:10F4A8000535A4FB0023EB18069CB21A67EB03038F
:10F4B800C4E90023F8BD00BFF8B5144606460F4658
:10F4C8001D4600F075F900FB05F5A0FB042304FBBD
:10F4D8000155EB18069CB21A67EB0303C4E9002335
:10F4E800F8BD00BF704700BF00292DE9F0071D4691
:10F4F800C0F29E800024002DC0F2958007460D467C
:10F5080016469C46002B3ED18A4254D9B2FA82F361
:10F5180043B1C3F1200620FA06F501FA03F19A4037
:10F5280029439840160CB1FBF6F597B206FB151166
:10F538004FEA104C07FB05F34CEA01418B4209D90D
:10F54800891805F1FF3C80F015818B4240F2128149
:10F55800023D8918C3EB010CBCFBF6F306FB13C193
:10F5680080B207FB03F740EA0140874207D9591EDA
:10F57800821880F00581974240F20281023B43EAFB
:10F588000542002303E08B420AD900231A4610469D
:10F59800194614B1404261EB4101BDE8F0077047DC
:10F5A800B3FA83F3002B40F087808C4501D3824265
:10F5B800ECD80122EBE712B90123B3FBF2F2B2FA5D
:10F5C80082F6002E3AD1891A150C1FFA82FC012303
:10F5D800B1FBF5F705FB17114FEA10480CFB07F6CE
:10F5E80048EA01418E4207D9891807F1FF3802D24B
:10F5F8008E4200F2DA804746891BB1FBF5F605FB1F
:10F60800161180B20CFB06FC40EA0140844507D97C
:10F61800711E821880F0B080944540F2AD80023EA1
:10F6280046EA0742B3E7E443524263EB430365E724
:10F63800404261EB41014FF0FF345CE7B240C6F154
:10F64800200521FA05F320FA05F701FA06F9150C49
:10F65800B3FBF5F847EA09091FFA82FC05FB1837DE
:10F668004FEA19410CFB08F341EA0747B040BB4297
:10F678000AD9BF1808F1FF3180F09580BB4240F2EB
:10F688009280A8F10208BF18FE1AB6FBF5F305FB35
:10F6980013611FFA89F90CFB03F649EA01418E420E
:10F6A80006D95F1E891878D28E4276D9023B89180E
:10F6B800891B43EA08438BE7C3F1200726FA07F8BA
:10F6C8000CFA03F248EA020C21FA07F105FA03FAE8
:10F6D8004FEA1C4920FA07F5B1FBF9F845EA0A0593
:10F6E80009FB18172A0C1FFA8CFA0AFB08F142EAE0
:10F6F8000747B94206FA03F609D917EB0C0708F1D0
:10F70800FF324ED2B9424CD9A8F1020867447F1A99
:10F71800B7FBF9F209FB1271ADB20AFB02FA45EA2E
:10F7280001418A4507D9551E11EB0C0137D28A458C
:10F7380035D9023A614442EA08424FEA124C1FFAAC
:10F7480086F808FB0CF7360C95B208FB05F806FBA3
:10F75800057505EB184506FB0CFCAF4288BF0CF598
:10F76800803CCAEB01010CEB1546B14212D309D01B
:10F7780000230CE76546EDE60E4646EA074206E733
:10F788000B46FCE61FFA88F800FA03F308EB054578
:10F79800AB42EDD2013A0023F9E63B4688E72A4618
:10F7A800C9E79046B3E788466EE7023F891823E722
:10F7B8002DE9F00F144605460E46002B3FD18A422C
:10F7C8004AD9B2FA82F343B1C3F1200025FA00F214
:10F7D80001FA03F69C4016439D40210CB6FBF1F25A
:10F7E8002F0CA0B201FB126C00FB02F347EA0C4697
:10F7F800B34208D9571E361980F0FF80B34240F251
:10F80800FC80023A3619F61AB6FBF1F301FB1361D4
:10F81800ADB200FB03F045EA0141884207D95E1EFC
:10F82800091980F0EC80884240F2E980023B43EA03
:10F838000242002310461946BDE8F00F70478B427C
:10F8480043D8B3FA83F4002C42D18B42234601D328
:10F8580082423BD80122EDE712B90123B3FBF2F44F
:10F86800B4FA84F2002A40F08A80091B260CA7B259
:10F878000123B1FBF6F006FB10114FEA154C07FB0C
:10F8880000F24CEA01418A4207D9091900F1FF3C0C
:10F8980002D28A4200F2D3806046C2EB010CBCFB64
:10F8A800F6F206FB12C1ADB207FB02F745EA0145C5
:10F8B800AF4207D9511E2C1980F0A380A74240F20D
:10F8C800A080023A42EA0042B4E700231A46B1E7B0
:10F8D800C4F1200722FA07F603FA04F3334321FAA6
:10F8E80007FA4FEA134C01FA04FB20FA07F141EA40
:10F8F8000B0BBAFBFCF70CFB17A61FFA83F84FEAB1
:10F908001B4508FB07F945EA0645A94502FA04FA2A
:10F9180004D97A1EED18C0F088801746C9EB050592
:10F92800B5FBFCF60CFB16521FFA8BFB08FB06F81E
:10F938004BEA0241884503D9721EC91870D316468E
:10F9480046EA0742170C1FFA8AFC0CFB07F695B229
:10F958004FEA1A430CFB05FC03FB056505EB1C4548
:10F9680003FB07F3AE4288BF03F58033C8EB010100
:10F9780003EB1543994250D347D000235AE79440EC
:10F98800C2F12008260C20FA08F721FA08F501FA36
:10F9980002F9B5FBF6F847EA090906FB1855A7B2BC
:10F9A8004FEA194C4CEA054C07FB08F3634500FA8B
:10F9B80002F509D91CEB040C08F1FF323DD263456E
:10F9C8003BD9A8F10208A444C3EB0C02B2FBF6F33E
:10F9D80006FB13201FFA89F907FB03F249EA0041E5
:10F9E8008A4206D9581E091925D28A4223D9023BD0
:10F9F8000919891A43EA08433BE73A4603E73346BD
:10FA080015E70A4642EA004214E71FFA8CF100FAA9
:10FA180004F001EB0545A842AFD2013A002309E7FB
:10FA280088458CD9023EC9188AE7A9457FF675AF83
:10FA3800023FED1872E70346DBE79046C4E7023859
:10FA480009192AE7002103E00A4B5B5843500431A7
:10FA580009480A4B42189A42F6D3094A02E00023A1
:10FA680042F8043B074B9A42F9D3F9F7D3F900F06F
:10FA78000FF87047CCAB0508000000204C0C0020A4
:10FA8800500C0020B0810020FEE7000000000000BC
:10FA98007F4B804A2DE9F3414FF4FA661E607E4B96
:10FAA800DFF858821A607D4A7D4B1A607D4B42F21E
:10FAB80010721A607C4B64241C607C4B4FF0FF3240
:10FAC8001A607B4B00251D70012788F80070F7F736
:10FAD8002DFFF6F7BBFB2046F7F71EF8F6F7DCFB21
:10FAE8002046F7F719F8F7F705FFF7F77DFDF7F761
:10FAF80029F82046F7F710F8F9F774FA2046F7F7CF
:10FB08000BF84FF4FA50F6F773FF2046F7F704F8AE
:10FB1800F6F7F8FA2046F6F7FFFF2846F7F77AFADD
:10FB28006448F6F7F9FFF3F72BFE2046F6F7F4FFE3
:10FB3800614B03F1100229468DE8240028465A68D3
:10FB48001B68F4F723F83046F6F7E6FF2846F4F783
:10FB58009DFA4FF6FF70F4F7AFFA32200321574AA7
:10FB68002B46F4F7C1FB96208C21554A2B46F4F717
:10FB7800BBFB9620534AA0212B46F4F7B5FBB421D2
:10FB8800514A2B469620F4F7AFFB3046F6F7C4FFF0
:10FB9800DC214E4A2B462846F4F7A6FB4C48F6F7DC
:10FBA800BBFF2046F6F7B8FFF6F774F82046F6F7DD
:10FBB800B3FF9FED350BF7F783F82046F6F7ACFF58
:10FBC800444B454A00933946444B4548FBF7D0FC23
:10FBD8002046F6F7A1FFF4F751FE2046F6F79CFF02
:10FBE8001420F5F7ADFD2846F5F7FDFD2046F6F79C
:10FBF80093FFF5F799FF2046F6F78EFFF6F71EFB01
:10FC08002046F6F789FFF6F795F808B188F800500E
:10FC1800344B1D70F1F754FAF4F7E6FD08B9324891
:10FC280003E0324B324800221A70F1F760FA314D86
:10FC3800314CF5F74DFAF8F75AFAF8F78BFAF8F766
:10FC48003FF8F7F779FF2F46F6F796F82B7833B198
:10FC5800012B02D1F7F7F6FC01E0F7F705FD0026C6
:10FC68003E70F7F72DFEF3F70DF8F9F783F82388C0
:10FC78001BB2012BE8D1F8F7CDFAF7F7CBFD2680B8
:10FC8800E2E700BFAFF300800000000000409F40A3
:10FC9800D8630020E0673500FC63002080C3C901F9
:10FCA800AC64002000640020C0630020F8630020DA
:10FCB800206D002000127A00987D0108C4A4050870
:10FCC800DEA40508EAA40508F6A40508FFA40508AB
:10FCD800002D3101000300200C6400206003002087
:10FCE8000C5E0020E0630020600F0020085E00200A
:10FCF8004C11002004640020780D0020B80E00206C
:10FD080010B4314C0180B1F5807F44608270C370BB
:10FD180052D00DD9B1F5806F39D017D9B1F5006F30
:10FD28002ED0B1F5805F24D0FF2040B210BC7047C0
:10FD380020293AD014D9402930D08029F4D1234938
:10FD48004FF02012C26081600020EEE7B1F5007F1D
:10FD5800EAD11F4B4FF00811C16083600020E4E72F
:10FD68001029E1D11B494FF00122C26081600020B7
:10FD7800DBE7194B4FF00111C16083600020D4E725
:10FD8800164A4FF00213C36082600020CDE7144981
:10FD98004FF00412C26081600020C6E7114B4FF09B
:10FDA8004011C16083600020BFE70F4A4FF0801305
:10FDB800C36082600020B8E70C4A4FF01013C3609C
:10FDC80082600020B1E700BFE4A30408229405087C
:10FDD800F2930508E2950508E4930508E6930508FB
:10FDE800EA93050862940508E29405080294050858
:10FDF8002DE9F00FB2B02E9030932E9B00882E9CE8
:10FE08005B68309FA4682D90451E03EB4506BF082C
:10FE1800209328942C952F911F921E96319700F0CD
:10FE28003A814FEA900A4FEACA0B00F003002F9973
:10FE3800299003F1080504EB0B00CDF884A0CDF858
:10FE4800A8B019951A921B97189617912B90179A84
:10FE5800189E13883380B2F802C0A6F802C09488AE
:10FE6800B480D788F78008361896219F199E0832E3
:10FE7800179256F8041C56F8082C4FF0000A4FF059
:10FE8800000B002F00F06982CDE904ABCDE906AB89
:10FE9800CDE902ABCDE900AB289CBC46029BDDF85E
:10FEA8000C902568C2FBC5394FF0000848EA030AE0
:10FEB800CB46CDE902AB049BDDF814B0C1FBC53BD2
:10FEC800CDF824B0CDF82080DDE908ABC1EA020006
:10FED8004AEA030ACDE904AB069BDDF81CB0326898
:10FEE800C0FBD53BCDF82CB0CDF82880DDE90AABB6
:10FEF800C2EA01074AEA030ACDE906AB9DE8010810
:10FF0800C7FBD50BCDF834B0CDF83080DDE90CABAC
:10FF18004AEA000A63680298CDE900AB0834DDF8C4
:10FF28000CB0C1FBC30BCDF83CB0CDF83880DDE98F
:10FF38000EAB4AEA000ACDE902AB71680498DDF815
:10FF480014B0C2FBC30BCDF844B0CDF84080DDE956
:10FF580010AB4AEA000ACDE904AB0698DDF81CB0FC
:10FF6800C7FBD30BCDF84CB0CDF84880DDE912AB18
:10FF7800C1EA02054AEA000ACDE906AB9DE8010894
:10FF8800C5FBD30BCDF854B0CDF85080DDE914ABE8
:10FF980008364AEA000ABCF1010CCDE900AB7FF44F
:10FFA8007DAF2A9D19982B9B2E18299F002F35D09D
:10FFB8001868039F029BC2FBC03700241D971C943E
:10FFC800DDE91C4544EA0304CDE90245049B059D8F
:10FFD800C1FBC035002723952297DDE9224544EA75
:10FFE8000304CDE90445C1EA0203079D069AC3FB51
:08FFF800D02525952497DDE9D1
:020000040801F1
:10000000244544EA02043368C3EA0101CDE9064508
:1000100053465D46C1FBD03527952697DDE926ABD3
:100020004AEA030A069A029C0499039D079FD30B90
:10003000059AE60BC90B46EA454043EA474441EAC4
:10004000424604F30F0500F30F0C199BCCEA054759
:1000500006F30F001A9D1B9E2F604FEADA3A083311
:100060004AEA4B4B0BF30F04C0EA04426A600835BE
:10007000711E19931A951B917FF4EDAE319A2F9E44
:100080001E991F9BDDF880B0D00037180D182F97F0
:100090000BEB000A1F181E951F97CDF880A0DDF806
:1000A000C0C01CF0030BCDF820B000F086802D9B63
:1000B000DDF8BC80CDF808B05808DDF880A0DDF888
:1000C000A0B00690CDF81080049A1E9E32F8025B14
:1000D000069826F8025B0492BAF80270BBF8023068
:1000E000BAF80020BBF800401E9617FB03F112FB84
:1000F00004F6451E4FEAE17711EB06082B4605F0A2
:10010000010047EBE6790AF104020BF10401002D2E
:100110003BD0A8B1B2F800C0BBF80470548848883E
:100120001CFB07F518EB050749EBE57614FB00F916
:1001300017EB090846EBE97904320431013B24D07E
:100140000F88B2F800C0568848888C8895881CFBB8
:1001500007FC18EB0C0816FB00F7D088CE8849EB9B
:10016000EC7C15FB04F518EB07084CEBE77918EB72
:10017000050710FB06FC49EBE57417EB0C0844EB94
:10018000EC7908320831023BDAD11F9A02994FEA22
:10019000D83545EA494404F30F0322F8023B4F1EC9
:1001A0000AF1020A1F9202978ED1DDF880A0DDF8D5
:1001B00020B00AEB4B0ACDF880A02C9E2E98B508F3
:1001C00040683FD0209F47EA000212F0030F00F181
:1001D000080307F1080214BF002101219F4298BFC4
:1001E000904294BF00260126314277D097E8420022
:1001F000016001216C1EA942466004EA010419D085
:1002000044B192E81200196002215C6008320833A0
:10021000A9420FD092E850001C605E60966802F11F
:10022000080BD2689E600231DA601033A9420BF1EC
:100230000802EFD1DDF880C0ED000CEB050B401992
:10024000CDF880B02C9C14F0030343D05A0854001E
:10025000002A00F08E80209D40EA050717F0030F6A
:10026000209F14BF00250125011D3E1D012B94BFB9
:10027000002505F001058F4298BFB04294BF0021D0
:1002800001210D4275D039689200BF18A342016068
:1002900020971044C4EB03011CD0209B013933F894
:1002A000024B0A4620F8024B01F0010192B129B13C
:1002B00033F8021B013A20F8021B0BD01C46014602
:1002C00034F802CB21F802CB5D88A31C4580881C42
:1002D000023AF3D132B0BDE8F00F7047B7F800C072
:1002E000A0F800C07C884480BE888680691EFE8895
:1002F0000C46BA4601F00101C680002C9AD089B1A3
:10030000B2F800B0A3F800B051885980B2F804C028
:10031000A3F804C0B2F806B00832A3F806B0083358
:10032000013C87D016881E8051885980B2F804B0ED
:10033000A3F804B0B2F806C0A3F806C016891E815F
:1003400003F1080B5189ABF802109389ABF8043024
:10035000D6891032023C0BF10803ABF80660E1D1FC
:1003600068E7289BCDE904ABCDE906ABCDE902AB4C
:100370001FE6194691E700BF2DE9F00F9CB0067803
:100380000F900F9C40880F9DA4686D681990B3FB77
:10039000F6FA471E4FEA5A0804EB4709AAEB48034E
:1003A00040460A940D951A97CDF86C800C911492E2
:1003B000CDF82C901193002800F0B5811746199ABA
:1003C000199CCDF848809108CA00159104F00303E8
:1003D000A9181792169310971891760075084FEA8E
:1003E000450C002D00F03B840B9FDDF8308047EA80
:1003F000080010F0030F14BF0021012108F10404CC
:10040000381D012E94BF002101F00101804598BFE5
:10041000A74294BF4FF000094FF0010911EA090FFC
:1004200000F01D84BB46D8F8002001236F1EAB42AC
:10043000CBF8002007EA03072146024614D237B161
:10044000246802230431021DAB4204600CD20C4626
:10045000104654F8047B40F8047B4968023351602D
:10046000211D021DAB42F2D3DDF83080DDF82CB047
:100470004FEA4C05664508EB05020BEB0503CCEB98
:1004800006001DD0013832F802CB014623F802CB1A
:1004900000F00100A1B128B132F8029B013923F824
:1004A000029B0DD014461F4634F8029B27F8029B8E
:1004B000B2F802A0A21CA3F802A0BB1C0239F1D121
:1004C0000C9ADDF83CC00B989CF800807100531822
:1004D0000A9E0C93159BCDF84C80451806EB4802FC
:1004E0000B950E92002B00F0B18300240025CDE97E
:1004F0000445CDE9024507930D9913460A9AB3F8CE
:1005000004A0B2F806B0CDF804A0B3F806A00E8897
:100510001588CDF820B0CDF824A0DDE902AB15FB9D
:1005200006F51AEB050A4BEBE57BCDE902AB1F881C
:100530004888B2F802C0B3F80290B2F804808C8800
:10054000CDF81880DDE904AB16FB07F61AEB060AB6
:100550004BEBE67BDDE902671CFB00F5761910FB2F
:1005600009F047EBE5771AEB000A4BEBE07BCDE9AE
:1005700002ABDDF818B0DDF804C0B1F80680099DC3
:100580001BFB04F016EB000A47EBE07BDDE902679A
:1005900014FB0CF4361947EBE477089C14FB08F0C5
:1005A0000831083208331AEB000418FB05F84BEB4E
:1005B000E075079816EB080A47EBE87B0138CDE9B0
:1005C0000245CDE904AB079099D1179E0E9C0A9B7A
:1005D0001899A7199A190E97169F002F73D00E9B82
:1005E00031F8020B32F8024B33F8026BDDE9028975
:1005F000DDE904AB14FB00F47D1E10FB06F618EBDE
:10060000040849EBE4791AEB060A4BEBE67B2F462C
:1006100005F00100CDE90289CDE904AB002D52D0EF
:10062000002873D031F8024B32F8020B33F8025B2A
:1006300010FB04F614FB05F0DDE90245DDE9048951
:10064000A41945EBE67518EB000849EBE079013F8A
:10065000CDE90245CDE9048935D0C246CB46DDE976
:1006600002890D4614460497214628461A4630F85A
:10067000026B31F8027B32F802CB6D8864885B88AC
:1006800017FB06F718EB070816FB0CF649EBE779A2
:100690001AEB060714FB05FA4BEBE67B15FB03FC94
:1006A0008C1C931C0499851C18EB0A0849EBEA7909
:1006B00017EB0C0A4BEBEC7B8A1ECDE90289049206
:1006C000D2D1CDE904AB029D03990498DDF828A0AE
:1006D000059BEA0B109D42EA4148129908F30F0965
:1006E000A5F80090DDF84C90C70B0AEB8908281D8F
:1006F0004A1E47EA4346CDF8288006F30F041090BF
:100700006C8012920AD00F9C267866E6DDE904AB75
:100710000D4614460497DDE90289A5E7149F1B9B4B
:1007200007EB83061496119F002F00F0A681DDF8D9
:1007300064B0DDF86480DDF834C04FEA9B09CDF881
:100740001C904FEAC90908F0030A0CEB090BCDF81D
:100750002090CDF810A0CDF824B0DDF83CC09CF876
:10076000006075084FEA450C002D00F07E820C9960
:100770000B980B9F40EA010414F0030F14BF0022F2
:1007800001220C1D0430012E94BF002202F0010250
:10079000814298BFA74294BF002301231A4200F070
:1007A0006482BA4601230F68691EAB42CAF8007022
:1007B000024601EA0307214614D237B12768022313
:1007C000211D021DAB4207600CD20C46104654F8A6
:1007D000047B40F8047B496802335160211D021DEF
:1007E000AB42F2D3DDF83090DDF82C804FEA4C05B7
:1007F000664509EB050208EB0503CCEB06001DD0AE
:10080000013832F802BB014623F802BB00F00100B8
:10081000A1B128B132F8025B013923F8025B0DD097
:1008200014461F4634F802AB27F802ABB2F802C0F8
:10083000A21CA3F802C0BB1C0239F1D1DDF82CA028
:10084000DDF830B0079876000AEB060C0BEB0608D3
:10085000CDF82CC0CDF83080002800F0F0810A9A45
:10086000DDF834805788B2F800A0DDF8289094882D
:10087000B9F80690B8F8062084460D984188058896
:10088000B8F8040017FB01F61AFB05F3B3461BEB9F
:1008900003014FEAE67714FB00F047EBE3750F180E
:1008A0000A9B19FB02F145EBE0750CF1FF3617EBE3
:1008B000010AB14606F0010008F1080203F108033D
:1008C00045EBE17B002E00F0858048B3DDF834C0B5
:1008D0001E88BCF808405888518897889D88B2F8CF
:1008E0000680B3F806C016FB04F41AEB040A10FBEA
:1008F00001F14BEBE4761AEB010415FB07FB46EB29
:10090000E17014EB0B011CFB08F640EBEB740832B2
:10091000083311EB060A44EBE67BB9F1010959D023
:10092000CDE902ABCB46B3F80080B3F80890168847
:10093000CDF8389018FB06F6DDE902895D88548809
:1009400098889188B2F806C0DF88B2F808A015FB35
:1009500004F418EB060810FB01F149EBE67918EBFB
:10096000040817FB0CF749EBE47918EB010849EB95
:10097000E17918EB070849EBE779CDE90289DDF861
:1009800038905D89548998899189B2F80EC0DE89C2
:1009900019FB0AF7DDE9028915FB04F418EB0708D7
:1009A00010FB01F149EBE77918EB040849EBE47916
:1009B00016FB0CF618EB010449EBE175103210330D
:1009C000A01945EBE671BBF1020BCDE90201AAD1FA
:1009D00082468B460DF1200898E816006318049DA6
:1009E0009DB332F802CB33F8026B16FB0CF4013DD9
:1009F0001AEB040A294605F001004BEBE47B25B312
:100A000058B132F8028B33F8020B10FB08F71AEBDF
:100A1000070A4BEBE77B691E17D01446184634F8DB
:100A2000025B30F8027B52885B8817FB05F81AEBF3
:100A300008064BEBE87713FB02FBA21C831C16EBAA
:100A40000B0A47EBEB7B0239E7D10F9DDDF85080B5
:100A500095F800C00A9A119E4FEADA3343EA4B44F4
:100A600004F30F0028F8020B02EB4C07711E0A97E3
:100A7000CDF8508011917FF470AE1A9E0F9CB5088E
:100A8000A06842D00A9F47EA000616F0030F07F15C
:100A9000080200F1080314BF002101219F4298BF02
:100AA000904294BF4FF0000A4FF0010A11EA0A0F7A
:100AB0007FD097E84200016001216C1EA942466088
:100AC00004EA010419D044B192E81200196002212D
:100AD0005C6008320833A9420FD092E850001C60D5
:100AE0005E60966802F10804D2689E600231DA60A6
:100AF0001033A94204F10802EFD1DDF828A0ED007F
:100B00000AEB05094019CDF82890DDF868A01AF025
:100B100003034AD05A085400002A00F0A480DDF8EC
:100B200028B040EA0B0515F0030F14BF002501257E
:100B30000BF10406011D012B94BF002505F00105F2
:100B40008B4598BFB04294BF4FF0000C4FF0010CA2
:100B500015EA0C0F00F08780DBF800109200934438
:100B6000A3420160CDF828B01044C4EB03011CD0AF
:100B70000A9B013933F8024B0A4620F8024B01F078
:100B8000010192B129B133F8021B013A20F8021B8E
:100B90000BD01C46014634F802CB21F802CB5D880D
:100BA000A31C4580881C023AF3D11CB0BDE8F00FAD
:100BB0007047B7F80090A0F800907C884480BE8809
:100BC0008680691EFE880C46B84601F00101C68089
:100BD000002C92D091B111881980B2F802C0A3F80C
:100BE00002C0B2F804A0A3F804A0B2F8069008323C
:100BF000A3F806900833013C3FF47FAF11881980B9
:100C0000B2F802C0A3F802C0B2F80490A3F80490AE
:100C1000B2F806A0A3F806A016891E8103F1080CFD
:100C20005189ACF802109389ACF80430D68910329F
:100C3000023C0CF10803ACF80660DFD15DE70D9AC9
:100C40000A9B4FF0000A4FF0000BC8E60026002771
:100C5000CDE904670A9A0D99CDE90267BCE43046F4
:100C60000B9B0C9A0EE4194682E730460B9B0C9ABC
:100C7000C6E500BF0000000000B553EC102B42F2A7
:100C8000FB1223F00043C3F6E972934285B026DDE0
:100C90004FF6FF72C7F6EF7293420BDD51EC100B6B
:100CA00002460B46FDF74AFF02460B4643EC102B6B
:100CB00005B000BD684600F0BFFB00F0030001284E
:100CC0009DED000B9DED021B1AD0022810D0F8B943
:100CD00000F0D2FE53EC102B10461946E4E79FEDCE
:100CE000101B00F0C9FE53EC102B10461946DBE731
:100CF00000F0C2FE53EC102B104603F10041D3E785
:100D000001F0F6FB53EC102B104603F10041CBE74A
:100D1000012001F0EDFB53EC102B10461946C3E700
:100D200000000000000000002DE9F04759EC108B96
:100D3000C9F30A56A6F57E74073C132C4D46CA46E5
:100D4000474626DC002C4FDB4FF6FF76C0F20F063D
:100D500046FA04F606EA090555EA080517D044A341
:100D6000D3E9002351EC100BFDF7EAFE002200232B
:100D7000FEF728FB00284AD0B9F1000F6EDB2AEA03
:100D8000060A4FF000085346424643EC102BBDE8DC
:100D9000F087332C0CDDB4F5806FF8D151EC100BDB
:100DA0003A460B46FDF7CCFE41EC100BBDE8F08750
:100DB000A6F58265033D4FF0FF3323FA05F515EAEA
:100DC000080FE4D02AA3D3E9002351EC100BFDF760
:100DD000B7FE00220023FEF7F5FAC0B1B9F1000F0B
:100DE0001CDB28EA050813E021A3D3E9002351EC1A
:100DF000100BFDF7A5FE00220023FEF7E3FA38B141
:100E0000B9F1000F1BDB4FF00008C24600E0CA46F4
:100E10005346424643EC102BBDE8F087142C09D012
:100E2000C6F5866303334FF0010808FA03F818EBA0
:100E30000708D6D30AF1010A28EA0508E8E729F0ED
:100E4000004848EA07084FF0000AD045CBF6F07A90
:100E500008BFCA4618BF4FF00008D9E74FF4801307
:100E600043FA04F409EB040A89E700BFAFF30080FA
:100E70009C7500883CE4377E00B553EC102B42F2A1
:100E8000FB1223F00043C3F6E972934285B027DDDD
:100E90004FF6FF72C7F6EF7293420BDD51EC100B69
:100EA00002460B46FDF74AFE02460B4643EC102B6A
:100EB00005B000BD684600F0BFFA00F0030001284D
:100EC0009DED000B9DED021B1DD0022812D008BB2A
:100ED000012001F00DFB53EC102B10461946E3E7FF
:100EE00000209FED111B01F003FB53EC102B10466B
:100EF0001946D9E7012001F0FBFA53EC102B1046FC
:100F000003F10041D0E700F0B7FD53EC102B104681
:100F10001946C9E700F0B0FD53EC102B104603F161
:100F20000041C1E7AFF300800000000000000000B6
:100F300000F0E6B8D0B52DED048BB0EE408AF0EEAF
:100F4000608A3C4C8AB000F0DBF994F90030B0EED6
:100F5000409AF0EE609A013335D0B0EE480AF0EED8
:100F6000680A01F04FFD00282DD051EC180B00222B
:100F70000023FEF713FA30B32F4B2478019300239C
:100F800008938DED028B8DED048B002C23D0002770
:100F90000026CFF6F07751EC180B00220023CDE9A4
:100FA0000667FEF7E7F9002825D002239C4200934C
:100FB00036D0684601F05EFD002831D0089B002B3A
:100FC00027D19DED069BB0EE490AF0EE690A0AB002
:100FD000BDEC048BD0BD4FF6FF774FF06046CCF2EE
:100FE000EF7751EC180B00220023CDE90667FEF7DE
:100FF000C1F90028D9D10123022C009315D06846ED
:1010000001F038FD88B10D4801F036FD8DED060B7D
:10101000D4E701F0EFFF089B9DED069B0360D2E74C
:1010200001F0E8FF22230360C8E701F0E3FF21237A
:101030000360E8E788030020CCA6050830A905086E
:1010400010B52DED048BB0EE408AF0EE608A294C8D
:101050008AB000F02DFC94F90030B0EE409AF0EE2A
:10106000609A01332BD0B0EE480AF0EE680A01F026
:10107000C9FC20B351EC180B00220023FEF784F9C1
:10108000E8B11D4B247801930123009300230893BA
:101090008DED048B8DED028BCCB10020002102463A
:1010A0000B46FEF729F8022CCDE9060115D101F017
:1010B000A1FF21230360089BABB99DED069BB0EE19
:1010C000490AF0EE690A0AB0BDEC048B10BD00229B
:1010D000002343EC172B8DED067B684601F0CAFC1C
:1010E0000028E8D1E3E701F085FF089B9DED069B12
:1010F0000360E4E788030020D4A605080000000090
:10110000F8B5B0EE407AF0EE607A53EC112B544211
:1011100010461D46002125F00047044353EC102BD8
:1011200047EAD474C7F6F0718C4216463DD8544253
:10113000344323F0004242EAD4748C4235D805F19E
:10114000404101F5801101434FD0AC1704F0020477
:10115000164344EAD37435D0384341D00021C7F652
:10116000F0718F424FD00021C7F6F0718A4237D01C
:10117000D21B12153C2A42DC002D7DDB53EC112BD7
:1011800051EC170BFDF7B8FF41EC100B01F030FCF0
:1011900001F06AFA51EC100B012C68D0022C57D0E8
:1011A000002C48D141EC170B07E051EC170B53EC26
:1011B000112BFDF7C5FC41EC170BB0EE470AF0EE22
:1011C000670AF8BD032CC7D801A151F824F000BF6D
:1011D000BB110108BB110108F9110108F311010845
:1011E000002B25DB9FED307BE7E7BDE8F84001F001
:1011F0003BBA9FED2F7BE0E79FED2F7BDDE72AA138
:10120000D1E90001C8E7BA423CD0032CABD801A118
:1012100051F824F02B12010825120108F9110108D8
:10122000F31101089FED267BC7E79FED277BC4E7FD
:101230009FED277BC1E730A3D3E90023FDF77EFCB8
:101240001DA3D3E90023FDF779FC41EC170BB4E7AC
:1012500029A3D3E90023FDF771FC02460B4616A132
:10126000D1E90001FDF76AFC41EC170BA5E701F19C
:10127000004141EC170BA0E73C32BFF67FAF0020E6
:10128000002189E7032CABD8DFE804F00B08050246
:101290009FED117B91E79FED127B8EE79FED127B17
:1012A0008BE79FED137B88E7182D4454FB21F93F12
:1012B000182D4454FB2109C0182D4454FB2109402A
:1012C000000000000000008000000000000000009E
:1012D000182D4454FB21F9BFD221337F7CD902C0A1
:1012E000D221337F7CD90240182D4454FB21E9BF21
:1012F000182D4454FB21E93F075C143326A6A13C7A
:101300002DE9F84F55EC104BB5F5801F2F4622DA2A
:1013100025F00043234368D0002D2046294670DB8A
:1013200000230022C4F25033FDF7BCFD4FF6FF73DB
:101330000F46C7F6EF739F4204460D466FF0350225
:1013400010DD2046294622462B46FDF7F9FB41ECED
:10135000100BBDE8F88F4FF6FF73C7F6EF7300224E
:101360009F42EEDC3B15A3F57E73073B9A18D60F20
:10137000901927F07F47C6F57E76FDF72DFD0736DD
:1013800027F4700747EA065545EC104B804689461E
:1013900001F00AFC4046494621A3D3E9002355EC5D
:1013A000104BFDF77FFD20A3D3E9002382468B4637
:1013B00040464946FDF776FD1DA3D3E900230646C6
:1013C0000F4620462946FDF76DFD02460B46304686
:1013D0003946FDF7B5FB02460B4650465946FDF728
:1013E000AFFB41EC100BBDE8F88F00210020CCF2E0
:1013F000503100220023FDF77FFE41EC100BBDE8C9
:10140000F88F22462B46FDF799FB00220023FDF7BB
:1014100073FE41EC100BBDE8F88F00BFAFF3008006
:1014200000609F501344D33F362BF111F3FE593D1A
:101430000EE526157BCBDB3F2DE9F04F53EC102B4F
:1014400042F2FB1223F00044C3F6E97294428FB0DB
:101450001E46074640F3AA804DF67B13C4F20203F2
:101460009C422ADC002E51EC100BDDA3D3E90023B3
:1014700040F3CA81FDF762FB42F2FB13C3F6F97336
:101480009C428046894600F0AA80D7A3D3E9002376
:10149000FDF754FB0D4604462B462246C7E900459E
:1014A00040464946FDF74AFBCFA3D3E90023FDF7A9
:1014B00045FB0125C7E9020181E042F2FB13C4F2BA
:1014C00039139C4240F3AA804FF6FF73C7F6EF73BF
:1014D0009C4278DC4FEA245AAAF5826AAAF1060AED
:1014E00051EC100BA4EB0A5319461D460446FDF7B8
:1014F00073FFFDF771FC8046894642464B46204605
:101500002946CDE90889FDF719FB00230022C4F222
:101510007013FDF7C7FC0D460446FDF75DFFFDF7B0
:101520005BFC804689462046294642464B46CDE92B
:101530000A89FDF703FB00230022C4F27013FDF7B4
:10154000B1FC002204460D460023CDE90C45FDF711
:1015500011FF002800F07B8140464946002200230D
:10156000FDF708FF03240AAD013C40B175E9020113
:1015700000220023FDF7FEFE013C0028F6D12346A1
:10158000022400949E4C08A839465246019400F06B
:10159000ABFB002E054612DA7A68FB6802F10042C6
:1015A00003F100437A60FB60454208E0002200231B
:1015B00043EC172B87ED000B80ED027B00252846BE
:1015C0000FB0BDE8F08F51EC100B02460B46FDF753
:1015D000B5FA0025C7E90201C7E90001EFE77AA3E0
:1015E000D3E90023FDF7AAFA79A3D3E900238046C3
:1015F0008946FDF7A3FA0D4604462B462246C7E965
:10160000004540464946FDF799FA71A3D3E9002306
:10161000FDF794FA0125C7E90201D0E701F0E8F9E6
:1016200059EC108B6CA3D3E9002340464946FDF7E3
:1016300039FC00230022C3F6E073FDF781FAFDF7C1
:10164000CBFE0546FDF7C8FB65A3D3E90023CDE932
:101650000201FDF727FC02460B4640464946FDF7CE
:101660006DFA61A3D3E9002382468B46DDE90201CE
:10167000FDF718FC1F2DCDE90401504659462BDC1F
:101680006A1E604B53F82230A34225D0DDE90423C3
:10169000FDF754FA02460B46C7E900238146884607
:1016A0004A46434650465946FDF748FADDE90423C9
:1016B000FDF744FA002E02460B46C7E90223BFF6A7
:1016C0007EAF08F1004301F10041C7F800907B6054
:1016D000B860F9606D4272E7DDE90423FDF72EFA88
:1016E00088462415C8F30A53E31A102B8146C7E92C
:1016F0000001D5DD34A3D3E90023DDE90201FDF7C4
:10170000D1FB8046894642464B4650465946FDF736
:1017100015FACDE90601DDE9062350465946FDF7E5
:101720000DFA42464B46FDF709FA29A3D3E90023F7
:1017300080468946DDE90201FDF7B4FB42464B468F
:10174000FDF7FCF9CDE90401DDE90423DDE906013B
:10175000FDF7F4F98846C8F30A53E41A312C8146A0
:10176000C7E9000140F3958021A3D3E90023DDE917
:101770000201FDF797FB8046894642464B46DDE96C
:101780000601FDF7DBF982468B4652465B46DDE9F2
:101790000601FDF7D3F942464B46FDF7CFF916A3F4
:1017A000D3E9002380468946DDE90201FDF77AFB93
:1017B00042464B46FDF7C2F9CDE904015046594671
:1017C00064E700BFAFF300800000601A61B4D03D51
:1017D0007370032E8A19A33B83C8C96D305FE43F41
:1017E00000004054FB21F93F3163621A61B4D03DDF
:1017F0000000002E8A19A33BC14920259A837B391A
:101800005CA70508DCA60508FDF79AF942F2FB1370
:10181000C3F6F9739C42804689461AD01EA3D3E9C9
:101820000023FDF78DF90D4604462B462246C7E9F5
:10183000004540464946FDF781F917A3D3E9002347
:10184000FDF77EF94FF0FF35C7E90201B7E6032443
:1018500095E613A3D3E90023FDF772F912A3D3E9A8
:10186000002380468946FDF76BF90D4604462B465A
:101870002246C7E9004540464946FDF75FF90AA3FD
:10188000D3E90023FDF75CF94FF0FF35C7E902010A
:1018900095E6DDE906AB03E73163621A61B4D03D3A
:1018A0000000601A61B4D03D7370032E8A19A33B07
:1018B0002DE9F84353EC102B00242546C7F6F074AD
:1018C000C7F6F0751C40AC422DED028BB0EE408A9D
:1018D000F0EE608A1946104600F0AB80002B7FDDE9
:1018E0001A1500F08980A2F57E7721F07F4323F45A
:1018F0007003073FD20743F4801366D5C20F4FF041
:10190000000C02EB43037F104200654616204FF4A3
:1019100000116C18D60F9C424FEA420202DC651897
:101920001B1B8C444908013806EB4303F1D12026E8
:1019300080464FF0004107E043D0D40F49085200E1
:10194000013E04EB43031BD0AB4208EB0104F3DD83
:1019500004F00049B9F1004F04EB01082BD0A9466F
:101960009442C5EB0303C4EB020288BF013B40185D
:10197000D40F49085200013E4D4604EB4303E3D126
:101980001A4327D146084FEA6C0101F17E511CF041
:10199000010F01F5C00118BF46F0004601EB0753E7
:1019A000324643EC182BB0EE480AF0EE680ABDEC64
:1019B000028BBDE8F883B8F1000FD0DB05F1010917
:1019C000CEE79442C4D91D46B7E7C20F02EB4303EA
:1019D000400093E7431C39D000F001031818D1E709
:1019E00023F000441443DED0002B36D11A46C10A3E
:1019F000153A40050029FAD011F4801329D1490085
:101A00000133CC02FBD5C3F10105C3F1200420FA58
:101A100004F4521921439840A2F57E7721F07F43C8
:101A200023F47003073FD20743F480133FF566AFFA
:101A3000CBE751EC100BFDF735FA02460B4651ECA3
:101A4000180BFDF77DF841EC180BACE70CF1010C1D
:101A500099E7202401250023D9E751EC100B0B4610
:101A6000FDF76CF802460B46FDF746FB41EC180B00
:101A700099E700BF000000002DE9F04F5BEC10ABD0
:101A80002DED028BB0EE418AF0EE618A2BF000441E
:101A9000B4F1795F85B071DA50465946FDF79CFC88
:101AA000002800F0FD8052465B4650465946FDF73F
:101AB000F9F981A3D3E9002306460F46FDF7F2F9B1
:101AC0007FA3D3E90023FDF73BF832463B46FDF701
:101AD000E9F97DA3D3E90023FDF730F832463B4610
:101AE000FDF7E0F97AA3D3E90023FDF729F83246A0
:101AF0003B46FDF7D7F978A3D3E90023FDF71EF89D
:101B000032463B46FDF7CEF975A3D3E90023FDF736
:101B100017F832463B46FDF7C5F980468946002353
:101B20000022C3F6E07330463946FDF7BBF9424662
:101B3000CDE900014B4630463946FDF7B3F953EC89
:101B4000182B04460D4650465946FDF7ABF90246A0
:101B50000B4620462946FCF7F1FF02460B46DDE91D
:101B60000001FCF7EBFF0B4600210246C3F6F071C3
:101B70000020FCF7E3FF41EC100B83E052465B468C
:101B800050465946FDF78EF94BA3D3E9002306468C
:101B90000F46FDF787F94AA3D3E90023FCF7D0FFEE
:101BA00032463B46FDF77EF947A3D3E90023FCF715
:101BB000C5FF32463B46FDF775F945A3D3E900233F
:101BC000FCF7BEFF32463B46FDF76CF942A3D3E972
:101BD0000023FCF7B3FF32463B46FDF763F940A311
:101BE000D3E90023FCF7ACFF3B463246FDF75AF938
:101BF00043F23233C3F6D3739C42804689468EDD6E
